:0800000038E6040001000000D5
:04000C004682000028
:040018006C820000F6
:04003400BA7C000092
:04004400827D0000B9
:04005000F07E00003E
:04006800AC82000066
:04007400A88400005C
:0401000092820000E7
:04017000A683000062
:0401880048840000A7
:100400005420EF00C3202000008041001040BA00BB
:100410000160EF0000000600535000003D25000081
:10042000642C0000544100003D250000640D0000D4
:100430000A0000005420EF006322200000804100E9
:100440001040BA000160EF000000060043680000A1
:100450003D250000642C0000535000003D250000A5
:10046000642C0000544100003D250000640D000094
:100470000A0000005420EF006324200000804100A7
:100480001040BA000160EF00000006005B5400005D
:1004900043500000536F0000636B00006574000060
:1004A0003D250000642000002D3E000000000000FB
:1004B0005420EF0043262000008041001040BA0085
:1004C0000160EF0000000600202500006428000005
:1004D0004E650000772900005D0D00000A00000055
:1004E0005420EF00C3272000008041001040BA00D4
:1004F0000160EF000000060047730000705200002A
:10050000784D0000742E00007278000053740000D3
:1005100061740000203D000047530000505F000060
:10052000525300004C5400005F4F0000464600004C
:100530000D0A0000000000005420EF00832A200074
:10054000008041001040BA000160EF00000006008A
:100550005B520000782000005374000065700000BA
:100560003D250000645D00000D0A00000000000051
:100570005420EF00E301200083015000050031000A
:10058000432D2000008041001040BA000160EF00C0
:1005900000000600402D2000838141008081410041
:1005A0001380BA00000006005B78650078782000B0
:1005B00078785B00783C780045537800433E7800BB
:1005C0002E2E78002E2E78002E2E78005D205D00D5
:1005D0002D2D0D002D3E0A0020640000656C0000EA
:1005E000657400005420EF00E32F200000804100DC
:1005F0001040BA000160EF0000000600756E0000B8
:100600006B6E00006F7700006E2000005B450000FD
:10061000534300005D2000002530000032780000C8
:100620000D0A0000000000005420EF0003322000FB
:10063000008041001040BA000160EF000000060099
:100640004773000070520000784D0000742E0000C7
:100650006C6500006E3D0000203C00002564000039
:100660003E0D00000A0000005420EF00033420007B
:10067000008041001040BA000160EF000000060059
:100680005B57000069460000695300007461000078
:10069000746500003D250000645D00000D0A000047
:1006A000000000005420EF00E335200000804100EE
:1006B0001040BA000160EF00000006004773000020
:1006C00070520000784D0000742E00007278000017
:1006D00053740000617400003D250000640D0000AB
:1006E0000A0000005420EF00E337200000804100A2
:1006F0001040BA000160EF0000000600494E000003
:10070000564100004C49000044200000494E0000C2
:1007100050550000540000005420EF0083392000A1
:10072000008041001040BA000160EF0000000600A8
:1007300044490000534300004F4E00004E45000066
:1007400043540000200000005420EF00033B200031
:10075000008041001040BA000160EF000000060078
:10076000434F00004E4E000045430000542000005F
:10077000000000005420EF00633C20000080410096
:100780001040BA000160EF00000006005B48000066
:100790006F73000074490000504100006472000053
:1007A000506500006E640000696E0000674600003E
:1007B0006C6700003D250000645D00000D0A00002C
:1007C000000000005420EF00E301200083015000EE
:1007D00005003100E33F2000008041001040BA00D6
:1007E0000160EF0000000600E03F2000838141002F
:1007F000808141001380BA00000006004773690041
:1008000070436E00686B6700436F46006D6D6C004F
:10081000616E670064412000636B4F003A484600F8
:100820006F73460074490D0050410A006472000065
:10083000506500006E6400005420EF0083422000E9
:10084000008041001040BA000160EF000000060087
:100850004773000070520000784D000074200000C3
:1008600063690000643D00003078000025780000D6
:100870002C2000006C6500006E3D00002564000027
:100880000D0A0000000000005420EF000345200086
:10089000008041001040BA000160EF000000060037
:1008A0005245000053450000542000005749000005
:1008B00046490000000000005420EF00834620005D
:1008C000008041001040BA000160EF000000060007
:1008D000526500007365000074740000696E0000CA
:1008E00067200000536F0000636B00006574000018
:1008F000730D00000A0000005420EF008348200020
:10090000008041001040BA000160EF0000000600C6
:10091000415400002B520000455300004554000094
:100920003D310000000000005420EF00034A200089
:10093000008041001040BA000160EF000000060096
:1009400057690000666900005F43000043520000E1
:10095000435B0000323600002D320000385D00009D
:100960003D2500006325000063250000630D0000A5
:100970000A0000005420EF00634C2000008041007A
:100980001040BA000160EF0000000600554400006E
:10099000502000003A0000005420EF00834D20005A
:1009A000008041001040BA000160EF000000060026
:1009B00054430000502000003A0000005420EF0093
:1009C000A34E2000008041001040BA000160EF00FB
:1009D00000000600525800005B52000078530000EF
:1009E000697A0000653D0000256400005D0D00008F
:1009F0000A0000005420EF006350200000804100F6
:100A00001040BA000160EF000000060041540000F1
:100A10002B6E000063740000637000003D25000031
:100A2000732C000025340000750000005420EF00F6
:100A300023522000008041001040BA000160EF0006
:100A4000000006004372000065610000746500004C
:100A5000642000005443000050200000736F000029
:100A6000636B0000657400003A0D00000A0000008E
:100A70005420EF0043542000008041001040BA0091
:100A80000160EF0000000600415400002B570000F9
:100A900052530000534900003D3F00000000000099
:100AA0005420EF00C3552000008041001040BA00E0
:100AB0000160EF0000000600000000005420EF007D
:100AC000A3562000008041001040BA000160EF00F2
:100AD00000000600495000003A2D00002C2D0000B7
:100AE0002C2D00002C2D00000D0A0000000000003D
:100AF0005420EF00C30120008301500005003100A5
:100B000043592000008041001040BA000160EF000E
:100B1000000006004059200083814100808141008F
:100B20001380BA000000060050697200636B200059
:100B300055706E00436F6F006E6E74004E7520002E
:100B40006D3A660020636F006F6E75006E656E0013
:100B500063746400206E0D00756D0A00626500000C
:100B60005420EF00C35B2000008041001040BA0019
:100B70000160EF000000060050690000636B000098
:100B800055700000436F00006E6E00004E7500004F
:100B90006D3A0000206300006F6E00006E6500007B
:100BA00063740000206E0000756D00006265000037
:100BB0007220000069730000203C000025640000E2
:100BC0003E0D00000A0000005420EF00035F2000EB
:100BD000008041001040BA000160EF0000000600F4
:100BE000477300007043000068650000636B0000FD
:100BF0005463000070430000494400003A200000A4
:100C000063690000643D0000256400002C200000A2
:100C1000727300006C74000043690000643D0000C2
:100C2000256400000D0A0000000000005420EF00C1
:100C3000430220008301500005003100236320009F
:100C4000008041001040BA000160EF000000060083
:100C50002063200083814100808141001380BA001D
:100C60000000060057692C00666925005F43630099
:100C700043522C00435B2500256463002D332C0078
:100C80002D2D25003E2063002B332C005D3D3000D0
:100C900030787800257825002C30780078250D00F4
:100CA000782C0A0030780000257800005420EF00EE
:100CB00023662000008041001040BA000160EF0070
:100CC0000000060050690000636B000055700000D2
:100CD00052530000534900004E7500006D20000083
:100CE000534B0000495000003A200000214700000B
:100CF000535000005F520000534C0000545F00004E
:100D00004F4B000028250000642900000D0A000058
:100D1000000000005420EF006369200000804100C3
:100D20001040BA000160EF0000000600727300007E
:100D300073690000203D0000256400002864000065
:100D4000626D0000292000003D250000642800009D
:100D50007065000072630000656E00007429000079
:100D60000D0A0000000000005420EF00036C20007A
:100D7000008041001040BA000160EF000000060052
:100D8000496E0000766100006C690000642000007C
:100D900052530000534900000D0A000000000000FB
:100DA0005420EF00C36D2000008041001040BA00C5
:100DB0000160EF000000060030300000302E00001F
:100DC00030300000302E000030300000302E0000A7
:100DD00030300000300000005420EF00836F20000E
:100DE000008041001040BA000160EF0000000600E2
:100DF000484F00005354000020490000505B0000A1
:100E0000257300005D0D00000A0000005420EF0073
:100E100023712000008041001040BA000160EF0003
:100E200000000600417400006F6D000020410000CA
:100E30002020000020200000763100002E3000002D
:100E40003120000020200000202000002020000091
:100E5000000000005420EF00637320000080410078
:100E60001040BA000160EF0000000600455200008B
:100E7000523A0000496E0000766100006C69000083
:100E80006420000054580000205400005950000015
:100E900045210000215B0000256400005D0D00007D
:100EA0000A0000005420EF00A3022000830150003C
:100EB00005003100E3762000008041001040BA00B8
:100EC0000160EF0000000600E07620008381410011
:100ED000808141001380BA00000006002A2A6F00BA
:100EE0002A207500496E7400697420006961310020
:100EF0006C6936007A6920006E67730020746500A3
:100F00006865630020576F0069466E0049206400E1
:100F10006D6F730064752E006C652E002C202E0002
:100F200074610D006B650A007320000061620000AF
:100F30005420EF00437A2000008041001040BA00A6
:100F40000160EF00000006004154000000000000B6
:100F50005420EF00437B2000008041001040BA0085
:100F60000160EF0000000600415400004530000021
:100F7000000000005420EF00637C2000008041004E
:100F80001040BA000160EF0000000600415400006C
:100F900026570000300000005420EF00837D200021
:100FA000008041001040BA000160EF000000060020
:100FB000436D0000643A0000257300000D0A000034
:100FC000000000005420EF00E37E2000008041007C
:100FD0001040BA000160EF000000060072630000DC
:100FE000762000007761000069740000205B00003B
:100FF000256400002F310000305D00000D0A000064
:10100000000000005420EF00E38020000080410039
:101010001040BA000160EF00000006005B430000D2
:1010200068650000636B0000534300004C530000F0
:1010300054430000747200003D250000645D000010
:101040000D0A0000000000005420EF008302200081
:10105000830150000500310003842000008041001E
:101060001040BA000160EF0000000600008420007C
:1010700083814100808141001380BA000000060096
:1010800047735D0070542C006370200054786D002D
:1010900053746F00617264007420650074634200D1
:1010A000705369006F636E006B655B00743D2500D3
:1010B000256464002C205D0054782C00506B0D00DA
:1010C00074530A00697A0000655B00002564000023
:1010D0005420EF004302200083015000050031003E
:1010E00043882000008041001040BA000160EF00FA
:1010F000000006004088200083814100808141007B
:101100001380BA00000006005B456900525273006C
:101110005D47200073706E0054636F00705474005C
:10112000785320007461490072744400203A4C00E6
:101130002063450075725B00726525006E74640063
:1011400020735D0074610D0074750A007320000047
:101150005420EF00230220008301500005003100DD
:10116000438C2000008041001040BA000160EF0075
:1011700000000600408C20008381410080814100F6
:101180001380BA00000006005B4520005252730035
:101190005D47690073707A005463650070542000E5
:1011A00078536F007461760072746500203A7200A3
:1011B00020475B00737025005F54640063705D001E
:1011C00054780D00576F0A00726B00005420EF0036
:1011D00043022000830150000500310023902000CD
:1011E000008041001040BA000160EF0000000600DE
:1011F0002090200083814100808141001380BA004B
:101200000000060047735D0070542C0063704700B7
:1012100054787300537470006172430074206F003F
:101220003A486D0045414D00445B6F00282564003D
:101230007829650025433D002543250025436400AA
:1012400025430D0025430A00254300005420EF00EC
:1012500023932000008041001040BA000160EF009D
:10126000000006005B740000785200006571000009
:10127000536900007A6500003D250000642C0000E1
:101280007478000044610000746100005750000051
:101290006F7300003D250000645D00000D0A000032
:1012A000000000005420EF000302200083015000E2
:1012B00005003100E3962000008041001040BA0094
:1012C0000160EF0000000600E096200083814100ED
:1012D000808141001380BA00000006005B454F008A
:1012E000525276005D4765007370720054635B0074
:1012F000705425007844640061743C00613A250014
:101300002054640078205D0064610D0074610A005F
:1013100020730000697A0000652000005420EF006F
:10132000C30120008301500005003100A39A200072
:10133000008041001040BA000160EF00000006008C
:10134000A09A200083814100808141001380BA006F
:10135000000006004773650070546D006370610003
:101360005478690044616E00746164003A2065003D
:101370007478720052653D0071532500697A6400EB
:10138000653D0D0025640A002C7200005420EF001A
:10139000239D2000008041001040BA000160EF0052
:1013A000000006005564000070420000756C0000EB
:1013B0006B540000785B0000000000005420EF0038
:1013C000A39E2000008041001040BA000160EF00A1
:1013D0000000060047730000704300006F6D0000BE
:1013E0004D6F0000646500003D250000640D0000A5
:1013F0000A0000005420EF0063A02000008041009C
:101400001040BA000160EF0000000600464C0000EA
:1014100041530000485F0000455200004153000066
:10142000455F0000534900005A4500003D2500007B
:10143000640D00000A0000005420EF0083A2200089
:10144000008041001040BA000160EF00000006007B
:10145000464C000041530000485F00005752000016
:1014600049540000455F0000534900005A45000000
:101470003D250000640D00000A0000005420EF002C
:10148000A3A42000008041001040BA000160EF00DA
:1014900000000600505200004F470000524100007B
:1014A0004D5F00004D4500004D4F000052590000B7
:1014B0003D250000640D00000A0000005420EF00EC
:1014C000A3A62000008041001040BA000160EF0098
:1014D0000000060064620000675F000053610000C6
:1014E0006D7000006C6500005074000072200000F8
:1014F00020200000203D0000256400000D0A0000AF
:10150000000000005420EF00E3A82000008041000C
:101510001040BA000160EF000000060064620000A5
:10152000675F0000415200004E530000616D0000F3
:10153000706C00006550000074720000203D0000D7
:10154000256400000D0A0000000000005420EF0098
:1015500023AB2000008041001040BA000160EF0082
:10156000000006004773000070440000626700003E
:10157000506600004C7600006C3D000025640000C1
:101580000D0A0000000000005420EF0003AD200011
:10159000008041001040BA000160EF00000006002A
:1015A0004F4E0000000000005420EF0003AE20006A
:1015B000008041001040BA000160EF00000006000A
:1015C0004F460000460000005420EF0003AF20000B
:1015D000008041001040BA000160EF0000000600EA
:1015E0004773000070530000706100006346000004
:1015F0006C61000067200000256400000D0A0000F7
:10160000000000005420EF00E3B020000080410003
:101610001040BA000160EF000000060041540000D5
:101620002B42000044410000544100003D300000C6
:10163000000000005420EF0063B220000080410051
:101640001040BA000160EF000000060041540000A5
:101650002B42000044410000544100003D31000095
:10166000000000005420EF00E3B3200000804100A0
:101670001040BA000160EF00000006004475000051
:101680006D7000005B250000645D00003E200000DE
:101690005B0000005420EF0063B520000080410093
:1016A0001040BA000160EF00000006005278000010
:1016B0005B250000645D00003E2000005B00000030
:1016C0005420EF00C3B62000008041001040BA0053
:1016D0000160EF0000000600414300004B5B00008A
:1016E000256400005D3E0000205B0000000000005B
:1016F0005420EF0043B82000008041001040BA00A1
:101700000160EF00000006005D0D00000A0D000002
:101710000A0000005420EF0063B92000008041005F
:101720001040BA000160EF00000006003C450000D8
:10173000736300003E0000005420EF0083BA2000D5
:10174000008041001040BA000160EF000000060078
:101750003C540000616200003E0000005420EF0095
:10176000A3BB2000008041001040BA000160EF00E0
:10177000000006005769000046690000527800002A
:101780005374000061720000743D00002564000085
:101790002C200000000000005420EF0083BD20003A
:1017A000008041001040BA000160EF000000060018
:1017B0005769000046690000527800005369000034
:1017C0007A6500003D250000642C00002000000028
:1017D0005420EF0043BF2000008041001040BA00B9
:1017E0000160EF0000000600486F00007374000005
:1017F0004950000041640000724600006C67000020
:101800003D250000642C0000200000005420EF0063
:1018100023C12000008041001040BA000160EF00A9
:1018200000000600736500007420000039300000DD
:10183000304B000062700000730D00000A200000B1
:10184000000000005420EF00E3C2200000804100AF
:101850001040BA000160EF00000006002A2A0000D4
:101860002A200000477300007054000065730000D8
:10187000742000007374000061720000742A00007C
:101880002A2A00000D0A0000000000005420EF008A
:1018900023C52000008041001040BA000160EF0025
:1018A00000000600415400002B570000413D00009D
:1018B000617400006F6D00003030000030330000B4
:1018C0002C2C000031310000000000005420EF00FB
:1018D00023C72000008041001040BA000160EF00E3
:1018E00000000600415400002B4E00004448000058
:1018F000435000003D310000000000005420EF0084
:10190000A3C82000008041001040BA000160EF0031
:1019100000000600415400002B4E0000535500000B
:10192000445000003D35000035300000310000001B
:101930005420EF0043CA2000008041001040BA004C
:101940000160EF00000006004F5900004F3E00000C
:10195000205300004B49000050200000534E00006F
:10196000415000005F53000075700000706C000073
:10197000795F00004F6E00000D0A000000000000BB
:101980005420EF00C3CC2000008041001040BA007A
:101990000160EF00000006002A2A00002046000037
:1019A000696C00006520000053790000737400002A
:1019B000656D000020450000727200006F7200002B
:1019C00020200000200D00000A0000005420EF003D
:1019D00023CF2000008041001040BA000160EF00DA
:1019E000000006004E6F000045720000726F00009C
:1019F000720D00000A0000005420EF0083D0200088
:101A0000008041001040BA000160EF0000000600B5
:101A10004D65000064690000612000004E6F000009
:101A2000742000005265000061640000790D000020
:101A30000A0000005420EF0063D220000080410023
:101A40001040BA000160EF00000006004669000087
:101A50006C650000204E00006F74000020460000FE
:101A60006F7500006E6400000D0A000000000000A9
:101A70005420EF0043D42000008041001040BA0001
:101A80000160EF0000000600202000002049000057
:101A90006E760000616C0000696400002050000058
:101AA00061740000680D00000A0000005420EF007F
:101AB00023D62000008041001040BA000160EF00F2
:101AC00000000600496E0000766100006C690000AD
:101AD000642000004E6100006D6500000D0A0000EA
:101AE000000000005420EF00E3D7200000804100F8
:101AF0001040BA000160EF000000060041630000E2
:101B0000636500007373000020440000656E0000F0
:101B100069650000640D00000A0000005420EF0019
:101B2000A3D92000008041001040BA000160EF00FE
:101B30000000060044690000736B000020460000AE
:101B4000756C00006C0D00000A0000005420EF00CE
:101B500023DB2000008041001040BA000160EF004C
:101B60000000060052650000616400002F5700006D
:101B70007269000074650000204500007272000068
:101B80006F7200000D0A0000000000005420EF00FA
:101B900023DD2000008041001040BA000160EF000A
:101BA000000006004E6F000074200000456E00002B
:101BB000616200006C650000640D00000A00000016
:101BC0005420EF00C3DE2000008041001040BA0026
:101BD0000160EF00000006004E6F0000204600008C
:101BE000696C0000652000005379000073740000E8
:101BF000656D00000D0A0000000000005420EF0099
:101C0000830220008301500005003100A3E1200081
:101C1000008041001040BA000160EF0000000600A3
:101C2000A0E1200083814100808141001380BA003F
:101C30000000060047452000545F540043536F00E6
:101C400044206B0045726500726F6E0072202E009A
:101C5000657820007065520063743100696E200061
:101C600067203D00436F20006D6D2500616E3000E0
:101C7000642032004163580063650D0070740A00EF
:101C8000656400005420EF008302200083015000AF
:101C900005003100E3E52000008041001040BA005B
:101CA0000160EF0000000600E0E5200083814100B4
:101CB000808141001380BA000000060047452000E3
:101CC000545F540043496F0044206B004572650027
:101CD000726F6E0072202E006578200070655200D1
:101CE00063743100696E200067203D00436F20005F
:101CF0006D6D2500616E3000642032004163580034
:101D000063650D0070740A00656400005420EF00E4
:101D100023E92000008041001040BA000160EF007C
:101D20000000060043720000656100007469000055
:101D30006E67000020660000696C0000653A0000D4
:101D400020730000616D0000706C0000652E0000C3
:101D500074780000740D00000A0000005420EF00A9
:101D6000A3EB2000008041001040BA000160EF00AA
:101D700000000600736100006D7000006C650000DB
:101D80002E74000078740000000000005420EF0062
:101D900023ED2000008041001040BA000160EF00F8
:101DA000000006007772000069740000655F0000A3
:101DB000746500007374000020460000532000008A
:101DC00045520000524F0000522000006F6E00008C
:101DD00020660000696C0000655F00006F70000005
:101DE000656E00000D0A0000000000005420EF00A6
:101DF00023F02000008041001040BA000160EF0095
:101E000000000600486500006C6C00006F200000B8
:101E100064610000726B00006E6500007373000067
:101E2000206D0000792000006F6C0000642000002D
:101E300066720000696500006E640000000000002A
:101E40005420EF00C3F22000008041001040BA008F
:101E50000160EF000000060041740000746500009E
:101E60006D700000696E000067200000746F000054
:101E7000207700007269000074650000202D0000CA
:101E80003E250000733C00002D0D00000A000000FC
:101E90005420EF0043F52000008041001040BA00BC
:101EA0000160EF0000000600777200006974000016
:101EB000655F000074650000737400002046000038
:101EC0005320000045520000524F000052200000F5
:101ED0006F6E0000206600006972000073740000DD
:101EE000206600005F7700007269000074650000E2
:101EF0000D0A0000000000005420EF0083F82000CD
:101F0000008041001040BA000160EF0000000600B0
:101F10002C200000492700007665000020630000A7
:101F20006F6D000065200000746F000020620000EB
:101F300065200000776900007468000020790000C7
:101F40006F7500002061000067610000696E00008D
:101F50000D0A0000000000005420EF0083FB200069
:101F6000008041001040BA000160EF000000060050
:101F70007772000069740000655F000074650000FE
:101F800073740000204600005320000045520000FA
:101F9000524F0000522000006F6E000020730000BE
:101FA000656300006F6E000064200000665F000043
:101FB0007772000069740000650D00000A000000DF
:101FC0005420EF00C3FE2000008041001040BA0002
:101FD0000160EF0000000600616200006F75000004
:101FE00074200000746F00002074000072790000FB
:101FF00020730000796E0000636900006E670000C6
:10200000207400006865000020660000696C000014
:10201000650D00000A0000005420EF00830121003C
:10202000008041001040BA000160EF00000006008F
:102030007772000069740000655F0000746500003D
:10204000737400003A20000045720000726F0000B7
:10205000722000007265000074750000726E00004E
:102060006564000020660000726F00006D200000B3
:10207000665F0000737900006E6300000D0A0000C7
:10208000000000005420EF00E30421000080410024
:102090001040BA000160EF0000000600616200001D
:1020A0006F75000074200000746F00002063000052
:1020B0006C6F00007365000020740000686500000C
:1020C00020660000696C0000650D00000A00000039
:1020D0005420EF0043072100008041001040BA0067
:1020E0000160EF0000000600466900006C6500001A
:1020F000202D00003E250000733C00002D20000034
:1021000063720000656100007465000064200000D7
:102110007375000063630000657300007366000060
:10212000756C00006C7900000D0A000000000000D2
:102130005420EF00430A2100008041001040BA0003
:102140000160EF000000060045720000726F0000A1
:10215000722000006F700000656E0000696E000064
:1021600067200000736F0000757200006365000057
:1021700020660000696C0000652000002D20000032
:10218000257300000D0A0000000000005420EF003D
:10219000230D2100008041001040BA000160EF00D3
:1021A0000000060045720000726F000072200000FF
:1021B0006F700000656E0000696E0000672000000F
:1021C0006465000073740000696E000061740000B3
:1021D000696F00006E200000666900006C650000F9
:1021E000202D000020250000730D00000A000000D3
:1021F0005420EF0043102100008041001040BA003D
:102200000160EF0000000600436F00006D6D0000EC
:10221000656E0000636900006E67000020660000C4
:10222000696C000065200000636F00007079000099
:102230000D0A0000000000005420EF00831221006E
:10224000008041001040BA000160EF00000006006D
:1022500050610000737300003A250000640D000017
:10226000000000005420EF00E31321000080410033
:102270001040BA000160EF00000006000A430000B1
:102280006F70000079200000636F00006D70000027
:102290006C650000746500000D0A0000000000007D
:1022A0005420EF00C3152100008041001040BA0007
:1022B0000160EF00000006004D6F0000756E000029
:1022C000746900006E670000204D00006564000026
:1022D0006961000020700000726900006F720000E8
:1022E000207400006F200000466F0000726D000037
:1022F00061740000746900006E6700000D0A000040
:10230000000000005420EF00E3182100008041008D
:102310001040BA000160EF0000000600436C0000AE
:1023200065610000726900006E67000020460000D1
:102330004154000025640000207300006563000024
:10234000746F0000723A000020250000756C0000D8
:102350000D0000005420EF00631B210000804100AD
:102360001040BA000160EF0000000600436C00005E
:1023700065610000726900006E6700002044000083
:102380006972000065630000746F000072790000DC
:10239000204500006E740000726900006573000043
:1023A0003A200000257500006C0D000000000000C0
:1023B0005420EF00431E2100008041001040BA006D
:1023C0000160EF0000000600476C00006F62000033
:1023D000616C0000204200006C6F0000636B000025
:1023E000204C0000656E000067740000682000004B
:1023F0003D200000256C0000750D00000A00000063
:102400005420EF00C3202100008041001040BA009A
:102410000160EF00000006000D0A00004D610000A1
:102420007374000065720000204200006F6F0000AE
:102430007420000052650000636F000072640000A9
:102440003A0000005420EF00E32221000080410008
:102450001040BA000160EF00000006000D0A000005
:10246000204200006F6F00007420000053650000E0
:10247000637400006F720000206C00006F63000046
:102480006174000065640000206100007420000099
:102490004D420000520000005420EF00832521002F
:1024A000008041001040BA000160EF00000006000B
:1024B0000D0A000050610000727400006974000091
:1024C000696F00006E20000054610000626C000023
:1024D0006520000061740000204D000042520000A1
:1024E000206F000066660000736500007420000025
:1024F0003078000030310000424500003A00000012
:102500005420EF0023022000830150000500310019
:10251000C3292100008041001040BA000160EF0093
:1025200000000600C0292100838141008081410014
:102530001380BA00000006000D0A530053656500C1
:10254000637463006F727400206F6F0066667200C0
:102550007365200074203D006F6620002050250028
:1025600061726C007469750074690D006F6E0A0009
:10257000204200006F6F0000742000005420EF0024
:10258000A32C2100008041001040BA000160EF0040
:1025900000000600506100007274000069740000C1
:1025A000696F00006E200000426F00006F74000031
:1025B0002053000065630000746F0000723A000051
:1025C000000000005420EF00E32E210000804100B5
:1025D0001040BA000160EF0000000600496E0000E4
:1025E000766100006C690000642000004641000034
:1025F000542000007379000073740000656D0000C2
:1026000020640000657400006563000074650000CC
:10261000640D00000A0000005420EF008331210007
:10262000008041001040BA000160EF000000060089
:1026300047450000545F000043490000442000006B
:1026400045720000726F0000722000002D20000013
:1026500052650000737000006F6E0000736500002B
:10266000203D00002025000030320000580D000001
:102670000A0000005420EF00633421000080410074
:102680001040BA000160EF00000006000D0A0000D3
:102690000D0A0000000000005420EF00630220003B
:1026A0008301500005003100833621000080410085
:1026B0001040BA000160EF000000060080362100E3
:1026C00083814100808141001380BA000000060030
:1026D0002A2A2A002A2A2A002A2A2A002A2A2A0002
:1026E0002A2A2A002A2A2A002A2A2A002A2A2A00F2
:1026F0002A2A2A002A2A2A002A2A2A0020432A00D3
:1027000049442A00202A2A002A2A2A002A2A0D00BF
:102710002A2A0A002A2A00002A2A00005420EF0050
:10272000A3392100008041001040BA000160EF0091
:10273000000006000D0A00004D6100006E750000EB
:10274000666100006374000075720000657200002D
:1027500020490000443A00002025000058000000F5
:102760005420EF00C33B2100008041001040BA001C
:102770000160EF00000006000D0A00004F45000058
:102780004D2F000041700000706C00006963000074
:1027900061740000696F00006E2000004944000071
:1027A0003A200000256300002563000000000000BF
:1027B0005420EF00433E2100008041001040BA0049
:1027C0000160EF00000006000D0A00004F45000008
:1027D0004D2F000041700000706C00006963000024
:1027E00061740000696F00006E2000004944000021
:1027F0003A200000256300002563000025630000E7
:102800002563000025630000000000005420EF0055
:1028100023412100008041001040BA000160EF0018
:10282000000006000D0A0000507200006F640000F6
:102830007563000074200000526500007669000096
:10284000736900006F6E00003A20000025580000F8
:10285000000000005420EF0063432100008041008D
:102860001040BA000160EF00000006000D0A0000F1
:102870005365000072690000616C0000204E00008A
:10288000756D000062650000723A000020250000AE
:102890005825000058250000582500005800000069
:1028A0005420EF00C3452100008041001040BA00D1
:1028B0000160EF00000006000D0A00004D610000FD
:1028C0006E750000666100006374000075720000A0
:1028D0006572000020440000617400006520000063
:1028E000436F0000646500003A2000002558000096
:1028F00025580000000000005420EF00834821000C
:10290000008041001040BA000160EF0000000600A6
:102910000D0A000043520000432D00003720000044
:1029200043680000656300006B730000756D000074
:102930003A20000025580000000000005420EF005D
:10294000A34A2100008041001040BA000160EF005E
:102950000000060047450000545F0000435300009C
:102960004420000045720000726F000072200000D9
:102970002D20000052650000737000006F6E000093
:1029800073650000203D000020250000303200006B
:10299000580D00000A0000005420EF0063022000E0
:1029A0008301500005003100834E2100008041006A
:1029B0001040BA000160EF0000000600804E2100C8
:1029C00083814100808141001380BA00000006002D
:1029D0002A2A2A002A2A2A002A2A2A002A2A2A00FF
:1029E0002A2A2A002A2A2A002A2A2A002A2A2A00EF
:1029F0002A2A2A002A2A2A002A2A2A0020432A00D0
:102A000053442A00202A2A002A2A2A002A2A0D00B2
:102A10002A2A0A002A2A00002A2A00005420EF004D
:102A2000A3512100008041001040BA000160EF0076
:102A3000000006000D0A000043530000445F000040
:102A400053540000525500004354000055520000FA
:102A5000453A000020250000580000005420EF00F7
:102A6000A3532100008041001040BA000160EF0034
:102A7000000006000D0A0000544100004143000020
:102A80003A20000025580000000000005420EF000C
:102A900023552100008041001040BA000160EF0082
:102AA000000006000D0A00004E53000041430000E4
:102AB0003A20000025580000000000005420EF00DC
:102AC000A3562100008041001040BA000160EF00D1
:102AD000000006000D0A000054520000414E0000A4
:102AE0005F53000050450000454400003A200000BC
:102AF00025580000000000005420EF0083582100FA
:102B0000008041001040BA000160EF0000000600A4
:102B10000D0A000043430000433A00002025000056
:102B20006C580000000000005420EF00035A210000
:102B3000008041001040BA000160EF000000060074
:102B40000D0A000052450000414400005F420000B1
:102B50004C5F00004C4500004E3A0000202500006C
:102B6000580000005420EF00E35B2100008041008A
:102B70001040BA000160EF00000006000D0A0000DE
:102B800052450000414400005F4200004C5F0000DD
:102B90005041000052540000494100004C3A0000EE
:102BA00020250000580000005420EF00035E2100A3
:102BB000008041001040BA000160EF0000000600F4
:102BC0000D0A00005752000049540000455F000004
:102BD000424C00004B5F00004D4900005341000093
:102BE0004C490000474E00003A20000025580000E4
:102BF000000000005420EF006360210000804100CD
:102C00001040BA000160EF00000006000D0A00004D
:102C100052450000414400005F4200004C4B000060
:102C20005F4D000049530000414C0000494700003F
:102C30004E3A000020250000580000005420EF000C
:102C4000A3622100008041001040BA000160EF0043
:102C5000000006000D0A000044530000525F00000F
:102C6000494D0000503A00002025000058000000A7
:102C70005420EF0043642100008041001040BA005E
:102C80000160EF00000006000D0A0000435F000035
:102C9000534900005A4500003A200000256C00000E
:102CA000580000005420EF00E3652100008041003F
:102CB0001040BA000160EF00000006000D0A00009D
:102CC00056440000445F0000525F0000435500007E
:102CD000525200005F4D0000494E00003A200000B3
:102CE00025580000000000005420EF000368210078
:102CF000008041001040BA000160EF0000000600B3
:102D00000D0A000056440000445F0000525F0000BE
:102D100043550000525200005F4D00004158000032
:102D20003A20000025580000000000005420EF0069
:102D3000236A2100008041001040BA000160EF00CA
:102D4000000006000D0A000056440000445F000029
:102D5000575F000043550000525200005F4D0000D5
:102D6000494E00003A2000002558000000000000F5
:102D70005420EF00436C2100008041001040BA0055
:102D80000160EF00000006000D0A0000564400003C
:102D9000445F0000575F000043550000525200009E
:102DA0005F4D0000415800003A2000002558000007
:102DB000000000005420EF00636E210000804100FD
:102DC0001040BA000160EF00000006000D0A00008C
:102DD000435F0000534900005A4500005F4D00006A
:102DE000554C0000543A0000202500005800000017
:102DF0005420EF0043702100008041001040BA00D1
:102E00000160EF00000006000D0A000045520000BE
:102E100041530000455F0000424C00004B5F000042
:102E2000454E00003A200000255800000000000038
:102E30005420EF0043722100008041001040BA008E
:102E40000160EF00000006000D0A0000534500007D
:102E5000435400004F5200005F530000495A0000E5
:102E6000453A000020250000580000005420EF00E3
:102E700023742100008041001040BA000160EF007F
:102E8000000006000D0A0000575000005F470000D8
:102E9000525000005F530000495A0000453A0000BC
:102EA00020250000580000005420EF000376210088
:102EB000008041001040BA000160EF0000000600F1
:102EC0000D0A0000575000005F47000052500000FC
:102ED0005F4500004E410000424C0000453A0000B2
:102EE00020250000580000005420EF000378210046
:102EF000008041001040BA000160EF0000000600B1
:102F00000D0A000052320000575F000046410000E9
:102F1000435400004F5200003A20000025580000A2
:102F2000000000005420EF00E37921000080410000
:102F30001040BA000160EF00000006000D0A00001A
:102F40005752000049540000455F0000424C000009
:102F50005F4C0000454E00003A200000255800005C
:102F6000000000005420EF00E37B210000804100BE
:102F70001040BA000160EF00000006000D0A0000DA
:102F80005752000049540000455F0000424C0000C9
:102F90005F5000004152000054490000414C0000C5
:102FA0003A20000025580000000000005420EF00E7
:102FB000237E2100008041001040BA000160EF0034
:102FC000000006000D0A0000464900004C450000C4
:102FD0005F4600004F5200004D410000545F00006A
:102FE00047520000503A0000202500005800000021
:102FF0005420EF0043802100008041001040BA00BF
:103000000160EF00000006000D0A0000434F0000C1
:10301000505900003A200000255800000000000030
:103020005420EF00C3812100008041001040BA000D
:103030000160EF00000006000D0A0000504500008E
:10304000524D00005F5700005249000054450000F7
:103050005F500000524F00005445000043540000F0
:103060003A20000025580000000000005420EF0026
:1030700023842100008041001040BA000160EF006D
:10308000000006000D0A0000544D0000505F0000D3
:103090005752000049540000455F000050520000A4
:1030A0004F54000045430000543A00002025000022
:1030B000580000005420EF0063862100008041008A
:1030C0001040BA000160EF00000006000D0A000089
:1030D000464900004C4500005F4600004F5200008A
:1030E0004D410000543A0000202500005800000027
:1030F0005420EF0043882100008041001040BA00B6
:103100000160EF00000006000D0A000043520000BD
:10311000433A000020250000580000005420EF0032
:10312000A3892100008041001040BA000160EF0037
:10313000000006000D0A00000D0A00000D0A000044
:10314000000000005420EF00E38A210000804100CD
:103150001040BA000160EF0000000600566F00004A
:103160006C7500006D650000206900007320000090
:103170004641000054310000320D00000A000000FA
:103180005420EF00C38C2100008041001040BA00A1
:103190000160EF0000000600566F00006C75000033
:1031A0006D650000206900007320000046410000AA
:1031B00054310000360D00000A0000005420EF00DA
:1031C000A38E2100008041001040BA000160EF0092
:1031D00000000600566F00006C7500006D65000071
:1031E00020690000732000004641000054330000B5
:1031F000320D00000A0000005420EF0083902100EF
:10320000008041001040BA000160EF00000006009D
:1032100042790000746500007320000070650000B2
:103220007220000053650000637400006F7200009C
:10323000203D0000202500006C7500000D0A0000F4
:10324000000000005420EF00E392210000804100C4
:103250001040BA000160EF00000006005265000057
:103260007365000072760000656400002053000062
:1032700065630000746F000072730000203D000061
:10328000202500006C7500000D0A00000000000001
:103290005420EF0043952100008041001040BA0007
:1032A0000160EF0000000600536500006374000039
:1032B0006F72000073200000706500007220000033
:1032C000436C0000757300007465000072200000FC
:1032D0003D200000257500000D0A000000000000E0
:1032E0005420EF00C3972100008041001040BA0035
:1032F0000160EF00000006004279000074650000E4
:10330000732000007065000072200000436C000014
:103310007573000074650000722000003D200000FD
:10332000256C0000750D00000A0000005420EF001D
:10333000239A2100008041001040BA000160EF0094
:1033400000000600546F0000746100006C20000053
:1033500053650000637400006F720000732000006A
:103360003D200000256C0000750D00000A000000E3
:103370005420EF00439C2100008041001040BA001F
:103380000160EF0000000600536500006374000058
:103390006F72000073200000666F00007220000052
:1033A00046410000542000003D200000256C000034
:1033B000750D00000A0000005420EF00839E2100DC
:1033C000008041001040BA000160EF0000000600DC
:1033D00046410000542000003120000061640000DC
:1033E0006472000065730000732000003D2000003F
:1033F00030780000253800006C5800000D0A0000ED
:10340000000000005420EF00E3A0210000804100F4
:103410001040BA000160EF000000060046410000C5
:10342000542000003220000061640000647200003B
:1034300065730000732000003D200000307800001C
:10344000253800006C5800000D0A00000000000044
:103450005420EF0043A32100008041001040BA0037
:103460000160EF0000000600526F00006F74000062
:10347000206400006972000065630000746F000042
:103480007279000020610000646400007265000031
:1034900073730000203D00002030000078250000FC
:1034A000386C0000580D00000A0000005420EF00A6
:1034B00023A62100008041001040BA000160EF0007
:1034C00000000600446100007461000020610000FB
:1034D00072650000612000006164000064720000F9
:1034E00065730000732000003D200000307800006C
:1034F000253800006C5800000D0A00000000000094
:103500005420EF00C3A82100008041001040BA0001
:103510000160EF0000000600526F00006F740000B1
:10352000206400006972000065630000746F000091
:10353000727900002073000065630000746F000062
:1035400072730000203D000020250000750D000072
:103550000A0000005420EF0063AB2100008041000E
:103560001040BA000160EF00000006005365000043
:10357000637400006F72000073200000666F00002B
:10358000722000006461000074610000203D0000B2
:10359000202500006C7500000D0A000000000000EE
:1035A0005420EF00C3AD2100008041001040BA005C
:1035B0000160EF0000000600546F0000746100001D
:1035C0006C200000436C00007573000074650000FF
:1035D00072730000203D0000202500006C75000083
:1035E0000D0A0000000000005420EF0003B021008D
:1035F000008041001040BA000160EF0000000600AA
:103600004869000064640000656E000020530000FB
:1036100065630000746F000072730000203D0000BD
:10362000202500006C7500000D0A0000000000005D
:103630005420EF0043B22100008041001040BA0046
:103640000160EF000000060045720000726F00008C
:10365000722000005265000061640000696E000085
:1036600067200000746800006520000046410000EB
:10367000540D00000A0000005420EF0083B4210024
:10368000008041001040BA000160EF000000060019
:103690000D0A000053650000637400006F720000A3
:1036A000206F000066660000736500007420000053
:1036B0006F660000204600004154000020310000E9
:1036C000203D0000202500006C7500000D0A000060
:1036D000000000005420EF0063B72100008041008B
:1036E0001040BA000160EF000000060046410000F3
:1036F0005420000031200000456E0000747200006C
:1037000069650000733A0000000000005420EF00DB
:1037100023B92100008041001040BA000160EF0091
:103720000000060045720000726F00007220000069
:103730005265000061640000696E000067200000AF
:103740007468000065200000726F00006F74000054
:10375000206400006972000065630000746F00005F
:10376000727900000D0A0000000000005420EF00F4
:10377000C3012000830150000500310023BD21005A
:10378000008041001040BA000160EF000000060018
:1037900020BD210083814100808141001380BA0057
:1037A000000006000D0A63005365740063746F0027
:1037B0006F727200206F79006666200073653D00AD
:1037C000742020006F66250020526C006F6F75001A
:1037D00074200D0044690A00726500005420EF0057
:1037E000A3BF2100008041001040BA000160EF003B
:1037F00000000600526F00006F74000020440000BB
:103800006972000065630000746F00007279000047
:10381000204500006E7400007269000065730000AE
:103820003A0000005420EF00E3C121000080410075
:103830001040BA000160EF0000000600447500006F
:103840006D700000204300006F6D00006D6100008E
:103850006E64000020450000525200004F520000EC
:10386000203100000D0A0000000000005420EF008D
:1038700023C42100008041001040BA000160EF0025
:1038800000000600447500006D7000002043000039
:103890006F6D00006D6100006E6400002045000047
:1038A000525200004F520000203200000D0A00006A
:1038B000000000005420EF0063C62100008041009A
:1038C0001040BA000160EF000000060054590000EB
:1038D00050450000206300006F6D00006D61000026
:1038E0006E64000020450000525200004F5200005C
:1038F0000D0A0000000000005420EF0083C82100E2
:10390000008041001040BA000160EF000000060096
:10391000417400006F6D000020760000312E000021
:103920003031000020450000525200003A250000CE
:1039300030340000752C0000204200006F78000039
:103940003A25000030340000752C000020490000AA
:10395000503A0000253000003375000000000000E0
:103960005420EF00C3CB2100008041001040BA007A
:103970000160EF0000000600417400006F6D000060
:1039800020760000312E00003031000020200000A1
:103990004F4B00003A25000030330000752C00002A
:1039A00025300000347500002C2500007300000055
:1039B0005420EF0043CE2100008041001040BA00A7
:1039C0000160EF00000006003C4400004952000086
:1039D0003E200000000000005420EF0083CF2100B3
:1039E000008041001040BA000160EF0000000600B6
:1039F0002020000020200000202000000000000007
:103A00005420EF00E3012000830150000500310045
:103A1000C3D12100008041001040BA000160EF00D6
:103A200000000600C0D12100838141008081410057
:103A30001380BA000000060025340D006C750A00E2
:103A400020462500696C340065286C0073297500D8
:103A50002C202000253944006C756900206272001A
:103A60007974280065737300207429006F74000056
:103A7000616C00005420EF0063D4210000804100FD
:103A80001040BA000160EF00000006002C2000008A
:103A900020250000396C0000752000004B4200001A
:103AA00079740000657300002066000072650000F4
:103AB000650D00000A0000005420EF0083D62100AD
:103AC000008041001040BA000160EF0000000600D5
:103AD0004469000072650000637400006F720000AA
:103AE00079200000437200006561000074650000E9
:103AF00064200000537500006363000065730000DC
:103B000073660000756C00006C7900000D0A0000FF
:103B1000000000005420EF0063D921000080410024
:103B20001040BA000160EF0000000600556E000072
:103B3000616200006C650000207400006F200000CE
:103B400043720000656100007465000020440000BD
:103B50006972000065630000746F000072790000F4
:103B60000D0A0000000000005420EF0003DC2100DB
:103B7000008041001040BA000160EF000000060024
:103B80004469000072650000637400006F720000F9
:103B900079200000456E000074720000792000005A
:103BA000446500006C65000074650000640D000051
:103BB0000A0000005420EF0063DE21000080410075
:103BC0001040BA000160EF000000060044650000EC
:103BD0006C650000746900006E67000020660000DC
:103BE000696C0000653A000020250000730D00009C
:103BF0000A0000005420EF0063E021000080410033
:103C00001040BA000160EF000000060044650000AB
:103C10006C650000746500006420000025640000ED
:103C200020660000696C0000657300000D0A00004A
:103C3000000000005420EF0063E2210000804100FA
:103C40001040BA000160EF00000006004E6F000057
:103C500020450000727200006F720000000000003A
:103C60005420EF00C3E32100008041001040BA005F
:103C70000160EF0000000600494C00004C450000C8
:103C8000474100004C200000464900004C45000020
:103C9000204E0000414D0000450000005420EF0080
:103CA000A3E52100008041001040BA000160EF0050
:103CB000000006004D45000044490000412000007E
:103CC0004E4F0000542000005245000041440000C7
:103CD000590000005420EF0063E7210000804100FC
:103CE0001040BA000160EF000000060046490000E5
:103CF0004C450000204E00004F54000020460000BC
:103D00004F5500004E440000000000005420EF001A
:103D100023E92100008041001040BA000160EF005B
:103D2000000006005041000054480000204E0000F2
:103D30004F540000204600004F5500004E44000044
:103D4000000000005420EF00E3EA21000080410061
:103D50001040BA000160EF0000000600414300007F
:103D6000434500005353000020440000454E00002E
:103D700049450000440000005420EF0083EC21007E
:103D8000008041001040BA000160EF000000060012
:103D90004D45000044490000412000004655000008
:103DA0004C4C0000000000005420EF0003EE210006
:103DB000008041001040BA000160EF0000000600E2
:103DC000522F00005720000045520000524F0000C3
:103DD000520000005420EF0063EF210000804100FA
:103DE0001040BA000160EF0000000600494E0000DC
:103DF000434F000052520000454300005420000091
:103E00004D450000444900004120000043480000A7
:103E1000414E000047450000000000005420EF0024
:103E2000A3F12100008041001040BA000160EF00C2
:103E300000000600575200004954000045200000D1
:103E4000505200004F54000045430000544500000C
:103E5000440000005420EF0063F321000080410083
:103E60001040BA000160EF00000006004653000059
:103E7000204E00004F540000204500004E4100003D
:103E8000424C000045440000000000005420EF00B8
:103E900023F52100008041001040BA000160EF00CE
:103EA000000006004E4F000020460000494C000074
:103EB000452000005359000053540000454D0000B8
:103EC000000000005420EF00E3F6210000804100D4
:103ED0001040BA000160EF0000000600554E0000DF
:103EE0004B4E00004F5700004E200000455200008E
:103EF000524F0000520000005420EF0083F82100D0
:103F0000008041001040BA000160EF000000060090
:103F1000464900004C450000205300005953000062
:103F2000544500004D20000045520000524F000053
:103F3000522000002D200000257300000D0A000013
:103F4000000000005420EF00E3FA2100008041004F
:103F50001040BA000160EF00000006004C4F000066
:103F60004144000048450000582000004F4B00002D
:103F70000D0A0000000000005420EF0083FC210027
:103F8000008041001040BA000160EF000000060010
:103F90003D3D00003D3D0000204200006F6F0000ED
:103FA000744C00006F610000646500007220000026
:103FB0003D3D00003D3D00000D0A000000000000F6
:103FC0005420EF00C3FE2100008041001040BA00E1
:103FD0000160EF000000060020200000202000000B
:103FE00020420000544C0000204400006174000096
:103FF000653A000020250000730D00000A00000053
:104000005420EF00C3002200008041001040BA009D
:104010000160EF00000006002020000020200000CA
:1040200020200000425400004C2000005265000097
:10403000763A000020250000730D00000A00000001
:104040005420EF00C3022200008041001040BA005B
:104050000160EF00000006004E470000205B0000FA
:10406000257800002C250000785D00000D0A000076
:10407000000000005420EF00630422000080410093
:104080001040BA000160EF00000006004F4B000036
:10409000205B000025300000385800005D4500001E
:1040A0004F4600000D0A0000000000005420EF0001
:1040B00023062200008041001040BA000160EF009A
:1040C000000006004F4B0000205B00002530000080
:1040D000385800005D0D00000A0000005420EF0079
:1040E000A3072200008041001040BA000160EF00E9
:1040F000000006003D3D00003D3D00003D3D00004C
:104100003D3D00003D3D000020540000657300006F
:1041100074200000436F00006D6D0000616E0000B0
:1041200064730000203D00003D3D00003D3D000067
:104130003D3D00000D0A0000000000005420EF008B
:10414000A30A2200008041001040BA000160EF0085
:1041500000000600205400004553000054200000D9
:104160004C450000445300002020000020200000A7
:1041700020200000202000002D200000466C0000C0
:1041800061730000682000004C450000447300008B
:104190000D0A0000000000005420EF00830D2200F3
:1041A000008041001040BA000160EF0000000600EE
:1041B000204C000045440000532000004F46000002
:1041C00046200000202000002020000020200000C9
:1041D000202000002D20000054750000726E0000A9
:1041E000204C000045440000732000006F66000072
:1041F000660D00000A0000005420EF00831022002A
:10420000008041001040BA000160EF00000006008D
:104210002054000045530000542000004255000087
:104220005A5A0000455200002020000020200000C3
:10423000202000002D200000536F0000756E00004C
:1042400064200000427500007A7A00006572000068
:104250000D0A00000D0A0000000000005420EF00CD
:10426000C30120008301500005003100A314220087
:10427000008041001040BA000160EF00000006001D
:10428000A014220083814100808141001380BA0084
:10429000000006003D3D6E003D3D64003D3D730065
:1042A0003D3D20003D3D3D0020413D0063713D000E
:1042B00075693D0073693D0074693D006F6E3D0096
:1042C00020430D006F6D0A006D6100005420EF0067
:1042D00023172200008041001040BA000160EF0067
:1042E000000006002053000054530000202000006E
:1042F00020200000202000002020000020200000BE
:1043000020200000202000002D200000426F00002F
:104310007820000053740000617400007573000081
:104320000D0A0000000000005420EF00031A2200D4
:10433000008041001040BA000160EF00000006005C
:10434000204E0000454F0000204F00004E2000008E
:10435000202000002020000020200000202000005D
:10436000202000002D2000004E6500006F2000007E
:1043700052650000636F000072640000696E000007
:10438000672000004F6E00000D0A000000000000D2
:104390005420EF00431D2200008041001040BA006D
:1043A0000160EF0000000600204E0000454F0000B5
:1043B000204F000046460000202000002020000082
:1043C0002020000020200000202000002D200000E0
:1043D0004E6500006F20000052650000636F000012
:1043E00072640000696E0000672000004F660000E4
:1043F000660D00000A0000005420EF006302200058
:10440000830150000500310083212200008041001B
:104410001040BA000160EF00000006008021220079
:1044200083814100808141001380BA0000000600B2
:10443000204E7000454F650020536400544F20000B
:10444000502054002020650020206D0020207000A6
:1044500020206F002D2072004E6561006F207200D9
:1044600052656900636F6C0072647900696E0D00BB
:1044700067200A00537400006F7000005420EF00A2
:10448000630220008301500005003100A3252200B3
:10449000008041001040BA000160EF0000000600FB
:1044A000A025220083814100808141001380BA0051
:1044B0000000060020486D0055442000444C610077
:1044C00045206E005445640053542000204F4F0097
:1044D0004E206600202066002D20200054756600C6
:1044E000726E6F0073207200626F200078203100BE
:1044F0004F6E6D0020660D006F720A0020360000BE
:104500005420EF00E301200083015000050031003A
:10451000C3292200008041001040BA000160EF0072
:1045200000000600C02922008381410080814100F3
:104530001380BA000000060020484800554475006A
:10454000444C64004520640054456C00535465009D
:10455000204F200046465400202065002D20730087
:1045600054757400726E0D0073200A006F660000AF
:10457000662000005420EF00E3012000830150007A
:1045800005003100632D2200008041001040BA0078
:104590000160EF0000000600602D220083814100D1
:1045A000808141001380BA000000060020416300B2
:1045B00044206F0053546E00415276005420650031
:1045C00020207200202073002020690020206F002E
:1045D0002D206E0053740D0061720A0074200000DB
:1045E000412F0000442000005420EF00E30220008F
:1045F000830150000500310003312200008041009A
:104600001040BA000160EF000000060000312200F7
:1046100083814100808141001380BA0000000600C0
:104620002053200045542E002053350052206D00A9
:104630003C327300352C2C00352C2000312C3100FD
:10464000322C6D00343E7300202D2C0020532000AE
:104650006574320020536D00616D7300706C2C0026
:10466000652020005261340074656D003A207300AB
:104670002E320D00356D0A00732C00005420EF001F
:10468000C30220008301500005003100A335220041
:10469000008041001040BA000160EF0000000600F9
:1046A000A035220083814100808141001380BA003F
:1046B00000000600205320004554310020503200F5
:1046C000472064003C3062002C312C00322C20004A
:1046D000323432002C333400363E6400202D620028
:1046E00020532C0065742000205033007265360082
:1046F000616D64007020620047610D00696E0A0000
:104700003A20000030640000622C00005420EF00CA
:10471000E30220008301500005003100233A22000B
:10472000008041001040BA000160EF000000060068
:10473000203A220083814100808141001380BA0029
:10474000000006002053650045542C00205720002F
:10475000532072003C44750044206E0048482000FD
:104760003A4D740020486900483A6D004D206500BC
:1047700052522C003E2020002D207200536565000F
:1047800074207000576165006B65610020737400D0
:1047900074610D0072740A0020740000696D0000DD
:1047A0005420EF0003032000830150000500310076
:1047B000C33E2200008041001040BA000160EF00BB
:1047C00000000600C03E220083814100808141003C
:1047D0001380BA00000006002047200045547200F4
:1047E0002057750053206E002020200020207400E8
:1047F0002020690020206D00202065002D202C0045
:104800004765200074207200637565007272700045
:10481000656E650074206100776174006B650D0042
:1048200020730A0074610D0072740A002074000085
:10483000696D0000652C00005420EF0083422200C7
:10484000008041001040BA000160EF000000060047
:104850003D3D00003D3D00003D3D00003D3D000070
:104860003D3D00002057000069460000692000001F
:10487000436F00006D6D0000616E00006473000006
:10488000203D00003D3D00003D3D00003D3D00005D
:104890000D0A0000000000005420EF004302200039
:1048A0008301500005003100834622000080410052
:1048B0001040BA000160EF000000060080462200B0
:1048C00083814100808141001380BA00000006000E
:1048D000205728004320540020204300202043007C
:1048E000202020002020740020206F0020202000A5
:1048F000202065002D207800576969004669740002
:10490000206329006F6E0D00736F0A006C65000054
:10491000206F00006E2000005420EF008349220029
:10492000008041001040BA000160EF000000060066
:10493000205700004F4E00002020000020200000E3
:104940002020000020200000202000002020000067
:10495000202000002D20000057690000466900005B
:10496000204F00006E0D00000A0000005420EF00F0
:10497000234C2200008041001040BA000160EF008B
:1049800000000600205700004F46000020200000D5
:104990002020000020200000202000002020000017
:1049A00020200000202000002D200000576900007A
:1049B00046690000204F0000666600000D0A0000F6
:1049C000000000005420EF00C301200083015000CC
:1049D00005003100E34F2200008041001040BA0082
:1049E0000160EF0000000600E04F220083814100DB
:1049F000808141001380BA0000000600205720008B
:104A00004F4E6F0020536E0054412000525453000B
:104A100020207400202061002020720020207400DB
:104A20002D2075005769700046690D00204F0A005F
:104A30006E2C00005420EF00E301200083015000A1
:104A40000500310063532200008041001040BA008D
:104A50000160EF00000006006053220083814100E6
:104A6000808141001380BA000000060020576F00CB
:104A70004F466E002053200054415300525474009E
:104A8000202061002020720020207400202075006A
:104A90002D20700057690D0046690A00204F000064
:104AA000666600002C2000005420EF00E301200087
:104AB00083015000050031000357220000804100AF
:104AC0001040BA000160EF0000000600005722000D
:104AD00083814100808141001380BA0000000600FC
:104AE000205772004F4E690020446E004348670013
:104AF0004720200020204300202068002020610063
:104B0000202072002D2067005769650046690D005E
:104B1000204F0A006E200000647500005420EF0052
:104B2000E30120008301500005003100A35A220058
:104B3000008041001040BA000160EF000000060054
:104B4000A05A220083814100808141001380BA0075
:104B500000000600205775004F467200204469008F
:104B600043486E004720670020202000202043009B
:104B700020206800202061002D2072005769670006
:104B800046696500204F0D0066660A00206400003B
:104B90005420EF00435D2200008041001040BA0025
:104BA0000160EF000000060020570000544F000095
:104BB0004E200000202000002020000020200000C7
:104BC0002020000020200000202000002D200000D8
:104BD000576900004669000020540000696D00001C
:104BE000656F000075740000204F00006E0D00001E
:104BF0000A0000005420EF006360220000804100A2
:104C00001040BA000160EF000000060020570000CD
:104C1000544F00004620000020200000202000000B
:104C20002020000020200000202000002020000084
:104C30002D20000057690000466900002054000044
:104C4000696D0000656F000075740000204F000062
:104C5000666600000D0A0000000000005420EF000E
:104C6000230220008301500005003100A3642200CC
:104C7000008041001040BA000160EF000000060013
:104C8000A064220083814100808141001380BA002A
:104C90000000060020573100544F2D002020320024
:104CA00020203500202034002020200020206D000E
:104CB0002020690020206E002D20750057697400A7
:104CC0004669650020547300696D2900656F0D0009
:104CD00075740A00202800005420EF00A302200071
:104CE00083015000050031008368220000804100EC
:104CF0001040BA000160EF0000000600806822004A
:104D000083814100808141001380BA0000000600C9
:104D1000205774004F4E74002049690050416E00C6
:104D20002020670020202000202049002020500063
:104D3000202020002D20410057696400466964004E
:104D4000205372007461650079737300206F7300E3
:104D50006E200D0061660A0074650000722000007C
:104D6000676500005420EF0083022000830150009B
:104D700005003100E36C2200008041001040BA00C1
:104D80000160EF0000000600E06C2200838141001A
:104D9000808141001380BA000000060020576500A2
:104DA0004F4663002049650050416900202076008D
:104DB0002020690020206E00202067002020200095
:104DC0002D20610057696E0046692000207549005A
:104DD0006E6150006666410065630D0074650A00EF
:104DE0006420000062790000207200005420EF006F
:104DF00023702200008041001040BA000160EF00E3
:104E0000000006002057000049460000492000002D
:104E1000494E0000495400002020000020200000DE
:104E200020200000202000002D20000057690000F5
:104E300046690000206D00006F640000756C000082
:104E400065200000494E0000495400000D0A000092
:104E5000000000005420EF00830220008301500076
:104E60000500310063742200008041001040BA0048
:104E70000160EF00000006006074220083814100A1
:104E8000808141001380BA000000060020572000F6
:104E90005353430049446800203C61004D7972003F
:104EA0005F53610053496300443E74002020650055
:104EB0002D2072005769200046696D002043610073
:104EC000686178006E67290065200D0053530A0061
:104ED0004944000020280000323000005420EF0038
:104EE000A3772200008041001040BA000160EF006B
:104EF00000000600205700005445000053540000F5
:104F0000204F00004E200000202000002020000044
:104F100020200000202000002D2000005769000004
:104F200046690000205400006573000074200000F2
:104F30006F6E00000D0A0000000000005420EF001A
:104F4000A37A2200008041001040BA000160EF0007
:104F50000000060020570000544500005354000094
:104F6000204F0000464600002020000020200000C6
:104F700020200000202000002D20000057690000A4
:104F80004669000020540000657300007420000092
:104F90006F660000660D00000A0000005420EF005C
:104FA000A37D2200008041001040BA000160EF00A4
:104FB000000006003D3D00003D3D00003D3D00007D
:104FC0003D3D00003D3D0000204F000074680000A2
:104FD00065720000204300006F6D00006D610000ED
:104FE0006E640000732000003D3D00003D3D000068
:104FF0003D3D00003D0D00000A0000005420EF0080
:10500000830220008301500005003100A3812200AB
:10501000008041001040BA000160EF00000006006F
:10502000A081220083814100808141001380BA0069
:105030000000060020572000524936005445200049
:1050400020536E004E2075003C316D0032336500F8
:1050500034357200363E69002D20630057722000FF
:1050600069746400652069005365670072696900AE
:10507000616C7400204E7300756D0D0062650A004E
:10508000723A00005420EF00E384220000804100C7
:105090001040BA000160EF0000000600205200003E
:1050A0004541000044200000534E00002020000035
:1050B00020200000202000002020000020200000F0
:1050C0002D200000526500006164000020530000A4
:1050D00065720000696100006C2000004E750000E0
:1050E0006D620000657200000D0A00000000000003
:1050F0005420EF00430220008301500005003100DE
:1051000043892200008041001040BA000160EF0096
:105110000000060040892200838141008081410017
:105120001380BA000000060020576E005249750037
:1051300054456600204D6100414E630020447400D8
:105140004154750045207200202065002D2020006C
:1051500057724D0069744D0065202F00446159005D
:1051600074655900206F0D0066200A004D61000033
:105170005420EF000302200083015000050031009D
:10518000438D2200008041001040BA000160EF0012
:1051900000000600408D2200838141008081410093
:1051A0001380BA00000006002052200045414D0047
:1051B000442061004D416E004E2075004441660060
:1051C0005445610020206300202074002D207500CC
:1051D000526572006164650020440D0061740A002C
:1051E000652000006F6600005420EF0023022000BD
:1051F000830150000500310003912200008041002E
:105200001040BA000160EF0000000600009122008B
:1052100083814100808141001380BA0000000600B4
:10522000204D6900432063005245720053456F00D2
:105230005420630020206F0020206E002020740086
:10524000202072002D206F0052656C0073656C0089
:10525000742065007468720065200D004D430A00DB
:10526000204D00005420EF00230220008301500055
:1052700005003100E3942200008041001040BA0094
:105280000160EF0000000600E094220083814100ED
:10529000808141001380BA0000000600205469009C
:1052A000432063005245720053456F005420630051
:1052B00020206F0020206E0020207400202072002B
:1052C0002D206F0052656C0073656C0074206500C2
:1052D0007468720065200D0054430A00204D0000E0
:1052E0005420EF00C3972200008041001040BA0014
:1052F0000160EF0000000600204200004F5800004F
:10530000204F000046460000202000002020000022
:105310002020000020200000202000002D20000080
:10532000506F00007765000072200000646F00007D
:10533000776E0000207400006865000020620000A5
:105340006F7800000D0A0000000000005420EF00FC
:10535000030220008301500005003100239C22003D
:10536000008041001040BA000160EF00000006001C
:10537000209C220083814100808141001380BA007B
:105380000000060020436E00414E200043456700A8
:105390004C206F002020690020206E002020670034
:1053A00020202000202074002D2065004361730020
:1053B0006E637400656C0D0020610A006E79000058
:1053C000206F00005420EF000302200083015000F2
:1053D00005003100E39F2200008041001040BA0028
:1053E0000160EF0000000600E09F22008381410081
:1053F000808141001380BA0000000600204D61004A
:105400004320720052456500562020002020720083
:1054100020206500202076002020690020207300D5
:105420002D20690047656F0074206E004D430D000C
:1054300020660A00697200006D7700005420EF00BA
:10544000230220008301500005003100A3A32200A5
:10545000008041001040BA000160EF00000006002B
:10546000A0A3220083814100808141001380BA0003
:1054700000000600204720004554740020546500B9
:10548000454D6D00502070004F20650020207200B7
:1054900020206100202074002D20750047657200D7
:1054A000742065006F730D0063690A006C6C000066
:1054B000617400006F7200005420EF0003022000AE
:1054C000830150000500310083A7220000804100C5
:1054D0001040BA000160EF000000060080A7220023
:1054E00083814100808141001380BA0000000600E2
:1054F000204772004554200020547400454D65003B
:1055000050206D0052207000202065002020720085
:10551000202061002D207400476575007420720002
:105520007265650067750D006C610A00746F00009C
:105530005420EF0043AA2200008041001040BA002E
:105540000160EF0000000600204700004554000005
:1055500020530000434100004E4E0000445800001C
:105560002020000020200000202000002D2000002E
:10557000476500007420000053630000616E000066
:105580004E640000780D00000A0000005420EF0077
:1055900023AD2200008041001040BA000160EF00FE
:1055A0000000060020550000504400004154000057
:1055B000452000004E560000202000002020000062
:1055C00020200000202000002D2000005570000049
:1055D00064610000746500002074000068650000CC
:1055E000204E000056200000526500007673000037
:1055F0000D0A0000000000005420EF0083B02200DC
:10560000008041001040BA000160EF000000060079
:1056100020430000484B000020410000455200009C
:105620005220000020200000202000002020000048
:10563000202000002D200000416E00007920000095
:1056400065720000726F0000727300003F0D000071
:105650000A0000005420EF00E30120008301500005
:105660000500310063B42200008041001040BA0000
:105670000160EF000000060060B422008381410059
:10568000808141001380BA000000060020472000FE
:1056900045546100204174004552200052204700CB
:1056A000202065002020740020204E00202064006F
:1056B0002D20780053680D006F770A0020650000E8
:1056C000727200006F7200005420EF00030220008D
:1056D000830150000500310003B822000080410022
:1056E0001040BA000160EF000000060000B8220080
:1056F00083814100808141001380BA0000000600D0
:105700002047740045542000204147004552650061
:105710005220740030204E002020640020207800A9
:10572000202020002D203D00536820006F7730009E
:1057300020650D0072720A006F7200002061000087
:105740005420EF00C3BA2200008041001040BA008C
:105750000160EF00000006002047000045540000F3
:10576000204100004552000052200000414C000042
:105770004C20000020200000202000002D200000F0
:10578000536800006F770000206100006C6C00001F
:1057900020650000727200006F720000730D00003F
:1057A0000A0000005420EF00E3BD22000080410009
:1057B0001040BA000160EF00000006002052000017
:1057C00045530000455400002041000045520000B0
:1057D0005220000020200000202000002020000097
:1057E0002D20000052650000736500007420000049
:1057F00041450000727200000D0A00000000000028
:105800005420EF00C3C02200008041001040BA00C5
:105810000160EF0000000600205200004147000038
:105820004E2000002020000020200000202000004A
:105830002020000020200000202000002D2000005B
:1058400052650000736500007420000041450000AF
:10585000727200002047000065740000204E0000B6
:10586000647800000D0A0000000000005420EF00E2
:1058700023C42200008041001040BA000160EF0004
:105880000000060020520000415300004E2000009E
:105890002020000020200000202000002020000008
:1058A00020200000202000002D2000005265000074
:1058B0007365000074200000414500007272000012
:1058C0002053000065740000204E00006478000042
:1058D0000D0A0000000000005420EF0083C72200E2
:1058E000008041001040BA000160EF000000060097
:1058F00020530000414700004E20000020200000FF
:105900002020000020200000202000002020000097
:10591000202000002D2000005365000074200000AE
:1059200041450000727200002047000065740000CD
:10593000204E0000647800000D0A00000000000006
:105940005420EF00230220008301500005003100A5
:10595000C3CB2200008041001040BA000160EF007C
:1059600000000600C0CB22008381410080814100FD
:105970001380BA0000000600205279004553200031
:105980002044440045466500202066002020610038
:105990002020750020206C00202074002D20730032
:1059A00052650D0073740A006F720D0065200A00C5
:1059B00046610000637400006F7200005420EF0025
:1059C000230220008301500005003100A3CF2200F4
:1059D000008041001040BA000160EF0000000600A6
:1059E000A0CF220083814100808141001380BA0052
:1059F000000006000D0A6D003D3D61003D3D6E005A
:105A00003D3D64003D3D73003D3D200020543D0080
:105A1000696D3D00696E3D0067203D00436F3D00AC
:105A20006E743D00726F3D006C6C0D0065720A0073
:105A3000204300006F6D00005420EF00E3012000C0
:105A4000830150000500310083D322000080410013
:105A50001040BA000160EF000000060080D3220071
:105A600083814100808141001380BA00000006005C
:105A700020547200432020004D4F56004E2043001A
:105A800056434F004F202000285453004D567400B9
:105A90002920610020207400202075002D20730033
:105AA0004D6F0D006E690A00746F00005420EF0006
:105AB000E3012000830150000500310023D72200BC
:105AC000008041001040BA000160EF0000000600B5
:105AD00020D7220083814100808141001380BA00D9
:105AE0000000060020547200432020004D4F470064
:105AF0004E205000475053005320200020205300D8
:105B000020207400202061002020740020207500D7
:105B10002D2073004D6F0D006E690A00746F000038
:105B20005420EF00030220008301500005003100E3
:105B3000C3DA2200008041001040BA000160EF008B
:105B400000000600C0DA220083814100808141000C
:105B50001380BA000000060020546F0043206E003E
:105B6000474520005420660052456F0041537200A3
:105B70004F4E2000202077002020610020206B0065
:105B8000202065002D2075004765700074200D00F1
:105B900072650A00617300005420EF0023022000A8
:105BA000830150000500310083DE220000804100A7
:105BB0001040BA000160EF000000060080DE220005
:105BC00083814100808141001380BA0000000600FB
:105BD0002054720043207300474565005420640040
:105BE0004750200053204700202050002020530021
:105BF0002020200020206400202061002D2074003F
:105C00004765610074200D0074680A00652000007B
:105C1000706100005420EF00E30220008301500077
:105C20000500310063E22200008041001040BA000C
:105C30000160EF000000060060E222008381410065
:105C4000808141001380BA000000060020542C001F
:105C50004320320047452D00542052004D534D0043
:105C6000472043003C312C002D3433003E202D00D2
:105C700020204700202053002D20560047652C008F
:105C80007420340072612D00772047004750530084
:105C9000532041006D730D00673A0A002031000067
:105CA0002D470000474100005420EF004302200030
:105CB000830150000500310003E72200008041000D
:105CC0001040BA000160EF000000060000E722006B
:105CD00083814100808141001380BA0000000600EA
:105CE00020544700432050004745530054202000D3
:105CF00052546400432061004441740054456500DF
:105D000020542000494D2600452020002D207400FD
:105D10004765690074206D006375650072720D003F
:105D2000656E0A00742000005420EF00630220001A
:105D3000830150000500310003EB22000080410088
:105D40001040BA000160EF000000060000EB2200E6
:105D500083814100808141001380BA000000060069
:105D600020542000432048004745720054202C0056
:105D7000414C200041524D004D20690020206E0012
:105D800020202C0020202000202052002D20650003
:105D90005365700074206500416C6100617274008D
:105DA0006D200D0044610A00792C00005420EF00A2
:105DB00003032000830150000500310023EF22007F
:105DC000008041001040BA000160EF0000000600B2
:105DD00020EF220083814100808141001380BA00BE
:105DE00000000600205461004320790053452C0038
:105DF00054202000414C4800415272004D202C009C
:105E00003C64200064204D0068686900206D6E00CD
:105E100020722C00723E2000202D52002047650089
:105E200065747000206365007572610072657400AE
:105E30006E740D0020410A006C610000726D00005C
:105E4000204400005420EF00230220008301500072
:105E500005003100E3F32200008041001040BA0049
:105E60000160EF0000000600E0F3220083814100A2
:105E7000808141001380BA000000060020544F00CA
:105E80004320200053454400542041004441430036
:105E900043202000203C28007878300078782D00BE
:105EA000783E3400202030002D2039005365350025
:105EB0007420290074680D0065200A005643000014
:105EC0005420EF0023022000830150000500310020
:105ED000C3F72200008041001040BA000160EF00CB
:105EE00000000600C0F7220083814100808141004C
:105EF0001380BA000000060020547400432065009F
:105F00004745670054207200564361004F497400B2
:105F10002020650020202000202076002020610025
:105F200020206C002D2075004765650074200D0051
:105F300056430A004F200000496E00005420EF0035
:105F4000230220008301500005003100A3FB220042
:105F5000008041001040BA000160EF000000060020
:105F6000A0FB220083814100808141001380BA00A0
:105F7000000006002054740043206500534567006C
:105F800054207200564361004F4974002020650080
:105F900020202000202076002020610020206C009E
:105FA0002D2075005365650074200D0056430A00CE
:105FB0004F200000496E00005420EF00C302200073
:105FC000830150000500310083FF22000080410062
:105FD0001040BA000160EF000000060080FF2200C0
:105FE00083814100808141001380BA0000000600D7
:105FF00020544F004320200057527600495461003E
:1060000045206C00564375004F2065004545200033
:10601000505274004F4D6F00202020002D2045006D
:1060200057724500697450006520520063754F0037
:1060300072724D00656E0D0074200A00444100002C
:10604000435F0000564300005420EF00630220002D
:10605000830150000500310003042300008041004B
:106060001040BA000160EF000000060000042300A9
:1060700083814100808141001380BA000000060046
:106080002054610043206C00524575004144650076
:1060900020562000434F66002045720045506F0097
:1060A000524F6D004D202000202045002D2045003E
:1060B000526550006164520020444F0041434D003E
:1060C0005F560D00434F0A00207600005420EF0079
:1060D0000302200083015000050031002308230043
:1060E000008041001040BA000160EF00000006008F
:1060F0002008230083814100808141001380BA0081
:10610000000006002054200043206C0047456F002B
:10611000542063004C4F6B00434B2000205373000E
:106120005441740054556100532074002854750084
:10613000474C730053290D00202D0A002047000012
:10614000657400005420EF002302200083015000FA
:1061500005003100E30B2300008041001040BA002D
:106160000160EF0000000600E00B23008381410086
:10617000808141001380BA000000060020546D00A9
:1061800043207700524561005620720020206500B0
:106190002020200020207200202065002020760092
:1061A00020206900202073002D20690047656F00C2
:1061B00074206E0054430D0020660A0069720000CE
:1061C0005420EF00E301200083015000050031005E
:1061D000C30F2300008041001040BA000160EF00AF
:1061E00000000600C00F2300838141008081410030
:1061F0001380BA0000000600205443004320200012
:10620000444152004320610054456D0053547000D6
:106210002020200020207400202065002020730012
:10622000202074002D200D0056430A004F2000004E
:10623000444100005420EF0043022000830150003D
:106240000500310063132300008041001040BA00B4
:106250000160EF000000060060132300838141000D
:10626000808141001380BA000000060020545500D0
:1062700043205300434154004E432000454C7400DA
:1062800020207900202070002020650020202000A0
:1062900020205400202043002D204300436129008A
:1062A0006E630D00656C0A00202800006F7200000C
:1062B000204A00005420EF002302200083015000F8
:1062C0000500310063172300008041001040BA0030
:1062D0000160EF0000000600601723008381410089
:1062E000808141001380BA000000060020546C0039
:1062F00043207900454E200054457700522061002C
:10630000534C6B004545650050597300204D2000EB
:106310004F44620045206F002D20780050650D002D
:1063200072690A006F64000069630000616C00001C
:106330005420EF00A302200083015000050031002B
:10634000431B2300008041001040BA000160EF00B1
:1063500000000600401B2300838141008081410032
:106360001380BA000000060020547400432065002A
:1063700053453A0054202000534C350045452C002D
:10638000505931002020300020202C0020203100E6
:10639000202035002D202C0053653300747330000D
:1063A00020742C0068653600205330006C650D00A9
:1063B00065700A0079200000726100005420EF002F
:1063C000030220008301500005003100A31F2300B9
:1063D000008041001040BA000160EF00000006009C
:1063E000A01F230083814100808141001380BA00F7
:1063F00000000600205420004320530047456C0055
:1064000054206500534C6500454570005059790093
:106410002020200020207200202061002020740015
:106420002D20650047650D0074730A00207400007C
:10643000686500005420EF00C30220008301500073
:106440000500310063232300008041001040BA00A2
:106450000160EF00000006006023230083814100FB
:10646000808141001380BA000000060020546800BB
:10647000432065004745200054206E0031327500EE
:1064800033346D002020620020206500202072003F
:1064900020207300202020002D20310069322C00A4
:1064A0006320320074652C0073743300202D2C009F
:1064B0002072340065740D0075720A006E7300005E
:1064C000207400005420EF000302200083015000DC
:1064D00005003100E3272300008041001040BA008E
:1064E0000160EF0000000600E027230083814100E7
:1064F000808141001380BA00000006002054200073
:10650000432054005445430053542000204969005F
:10651000324332002020630020202000202062002F
:1065200020207500202073002D200D0045780A00E2
:106530006572000063690000736500005420EF007D
:10654000630220008301500005003100A32B2300CB
:10655000008041001040BA000160EF00000006001A
:10656000A02B230083814100808141001380BA0069
:10657000000006002054200043206500494E6E00B4
:1065800049547400204169004C4C7200204565005C
:1065900045202000202045002020450020205000DC
:1065A0002D205200496E4F0069744D0069610D0045
:1065B0006C690A007A6500002074000068650000BC
:1065C0005420EF00430220008301500005003100F9
:1065D000C32F2300008041001040BA000160EF008B
:1065E00000000600C02F230083814100808141000C
:1065F0001380BA00000006002054680043206500A4
:10660000494E200049546C00204C6F004F577700D2
:10661000455265002045720045202000202045009D
:10662000202045002D205000496E520069744F0013
:1066300069614D006C690D007A650A0020740000E4
:106640005420EF0083022000830150000500310038
:10665000C3332300008041001040BA000160EF0006
:1066600000000600C0332300838141008081410087
:106670001380BA000000060020544500432050005B
:10668000494E520049544F0020564D00434F2000C0
:1066900020545600414243004C454F002045200005
:1066A000452074002D206100496E620069746C0001
:1066B000696165006C690D007A650A00207400004C
:1066C00068650000204500005420EF008302200090
:1066D0008301500005003100033823000080410091
:1066E0001040BA000160EF000000060000382300EF
:1066F00083814100808141001380BA0000000600C0
:1067000020546300432069005354700041526C00D0
:106710005420690044496E005343670049502000EB
:106720004C4974004E4568002028650054532000F1
:1067300054446F00292073002D20630052650D0022
:1067400073750A006D650000206400006973000025
:106750005420EF0063022000830150000500310047
:10676000433C2300008041001040BA000160EF006C
:1067700000000600403C23008381410080814100ED
:106780001380BA0000000600205463004320690013
:10679000535470004F506C002044690049536E0000
:1067A00043496700504C2000494E74004520680062
:1067B000202865005453200050446F0029207300A6
:1067C0002D20630053740D006F700A0020640000D8
:1067D000697300005420EF00230320008301500060
:1067E0000500310063402300008041001040BA00E2
:1067F0000160EF000000060060402300838141003B
:10680000808141001380BA0000000600205435004A
:1068100043202000464C28005320410078204400AB
:1068200078202C007820460078204C0020202C0076
:1068300020204100202044002D2045005365720097
:106840007420720046692C006E655000204C500088
:106850006F6353006B20450053634100616C290056
:10686000696E0D0067200A00302D000032350000EF
:106870005420EF0083022000830150000500310006
:1068800043452300008041001040BA000160EF0042
:1068900000000600404523008381410080814100C3
:1068A0001380BA00000006002054200043206F002F
:1068B000524573005345630054206900444F6C00F7
:1068C00020206C00202061002020740020206F0018
:1068D000202072002D20200052656C0073656F002F
:1068E00074206F006469700073630D0069700A00A2
:1068F0006C6900006E6500005420EF00A3022000C8
:1069000083015000050031008349230000804100CD
:106910001040BA000160EF0000000600804923002B
:1069200083814100808141001380BA00000006008D
:1069300020542000432066004745720054206F0019
:1069400045456D00205720004F52740044206800D8
:106950002861650064722000292045002D20450033
:10696000526550006164520020614F0020774D0055
:106970006F720D0064200A00617400002041000065
:10698000647200005420EF00830220008301500055
:1069900005003100E34D2300008041001040BA00A3
:1069A0000160EF0000000600E04D230083814100FC
:1069B000808141001380BA0000000600205441008D
:1069C0004320640053457200542020004545740064
:1069D00020576F004F522000442074002861680047
:1069E00064726500292020002D2045005772450063
:1069F000697450006520520061204F00776F4D0090
:106A000072640D0020610A00742000005420EF0021
:106A100003022000830150000500310023522300AF
:106A2000008041001040BA000160EF000000060045
:106A30002052230083814100808141001380BA00ED
:106A400000000600205472004320610047456D009D
:106A5000542020004F504F00544970004F4E740096
:106A60005320690020206F0020206E00202073003A
:106A70002D200D0047650A007420000050720000B0
:106A80006F6700005420EF00830220008301500054
:106A900005003100E3552300008041001040BA009A
:106AA0000160EF0000000600E055230083814100F3
:106AB000808141001380BA0000000600205463006A
:106AC00043206F0047457200542064004C41690028
:106AD00053546E00205067004F53200049547000FB
:106AE000494F6F004E537300202D690020477400FA
:106AF0006574690020746F0068656E00206C730017
:106B000061730D0074200A00726500005420EF00CC
:106B1000E30220008301500005003100235A2300C6
:106B2000008041001040BA000160EF000000060044
:106B3000205A230083814100808141001380BA00E4
:106B4000000006002054310043202E005050370032
:106B5000532020005445610053547400202020002D
:106B60002020320020202C00202031002020350061
:106B70002D202C0054433300206330007265200028
:106B8000617426006573200020703500756C30003C
:106B90007365730073200D0061740A00204A0000C1
:106BA0005420EF00830220008301500005003100D3
:106BB000C35E2300008041001040BA000160EF0076
:106BC00000000600C05E23008381410080814100F7
:106BD0001380BA00000006002054650043206700BF
:106BE00047456900542073005254740043206500E7
:106BF000414C7200415220004D207300202065005E
:106C0000202074002D2074004765690074206E00F8
:106C1000746867006520730054430D0020520A0019
:106C200054430000207200005420EF00A302200013
:106C30008301500005003100036323000080410000
:106C40001040BA000160EF0000000600006323005E
:106C500083814100808141001380BA00000006005A
:106C60002054700043206F00474577005420650092
:106C7000534E720041502000205075005752700052
:106C80002020200020206600202072002D206F0090
:106C900047656D0074202000534E5400415043005E
:106CA000206F0D006E2F0A00666600002061000054
:106CB000742000005420EF002302200083015000C4
:106CC0000500310063672300008041001040BA00D6
:106CD0000160EF000000060060672300838141002F
:106CE000808141001380BA000000060020546E002D
:106CF000432020005345610054207400534E20006F
:106D000041507000204F6F004E207700202065001A
:106D100020207200202020002D2075005365700077
:106D200074200D00534E0A0041500000206F0000F7
:106D30005420EF00230220008301500005003100A1
:106D4000436B2300008041001040BA000160EF0057
:106D500000000600406B23008381410080814100D8
:106D60001380BA000000060020546600432066002D
:106D70005345200054206100534E740041502000C0
:106D8000204F700046466F002020770020206500CD
:106D9000202072002D2020005365750074207000A3
:106DA000534E0D0041500A00206F00005420EF00A8
:106DB000230220008301500005003100236F2300CF
:106DC000008041001040BA000160EF0000000600A2
:106DD000206F230083814100808141001380BA002D
:106DE0000000060020546400432065004143200059
:106DF000512066004D4F720044456F0020206D0009
:106E00002020200020207400202068002020650021
:106E10002D202000476554007420430061630D005D
:106E200071200A006D6F00005420EF0083022000E3
:106E300083015000050031000373230000804100EE
:106E40001040BA000160EF0000000600007323004C
:106E500083814100808141001380BA000000060058
:106E600020546F0043202000534554005420430019
:106E700041432000512077004D4F69004445740084
:106E8000202068002020200020204E002D206500BA
:106E900057726F006974200065206F0041636600BF
:106EA000712066006D6F0D0064650A00207400009B
:106EB0005420EF00A30220008301500005003100A0
:106EC00043772300008041001040BA000160EF00CA
:106ED000000006004077230083814100808141004B
:106EE0001380BA00000006002054540043204300E1
:106EF000534520005420770041436900512074001D
:106F00004D4F680044452000204E4E00454F65001F
:106F100020206F002D20200057726F0069746E00D2
:106F200065200D0041630A0071200D006D6F0A009D
:106F300064650000207400006F2000005420EF0002
:106F4000030220008301500005003100A37B2300D1
:106F5000008041001040BA000160EF000000060010
:106F6000A07B230083814100808141001380BA000F
:106F7000000006003D3D61003D3D6E003D3D64006A
:106F80003D3D73003D3D200020533D0069673D00BD
:106F90006E613D006C203D0047653D006E653D0023
:106FA00072613D00746F0D0072200A00436F000093
:106FB0006D6D00005420EF00637E230000804100CF
:106FC0001040BA000160EF000000060020530000EE
:106FD00047200000534900004E45000020200000DB
:106FE00020200000202000002020000020200000A1
:106FF00020200000202000002D2000005369000008
:107000006E65000020770000617600006566000074
:107010006F7200006D0D00000A0000005420EF00A8
:10702000630220008301500005003100A382230089
:10703000008041001040BA000160EF00000006002F
:10704000A082230083814100808141001380BA0027
:107050000000060020536E0047206300534579006E
:10706000542020003C462600464620002041410096
:1070700041416D003E20700020206C0020206900FE
:107080002D207400536575007420640074686500D9
:1070900065200D0046720A006571000075650000EC
:1070A0005420EF00C3852300008041001040BA0047
:1070B0000160EF00000006002053000047200000A0
:1070C00053510000554100005245000020200000AF
:1070D00020200000202000002020000020200000B0
:1070E000202000002D200000537100007561000079
:1070F000726500002077000061760000650D0000D9
:107100000A0000005420EF00E388230000804100C3
:107110001040BA000160EF0000000600205300009C
:1071200047200000524100004D5000002020000088
:10713000202000002020000020200000202000004F
:1071400020200000202000002D20000052610000BF
:107150006D7000000D0A0000000000005420EF00D8
:10716000A38B2300008041001040BA000160EF00B3
:10717000000006002053000047200000505500008A
:107180004C5300004520000020200000202000007B
:1071900020200000202000002020000020200000EF
:1071A0002D200000507500006C730000650D00007C
:1071B0000A0000005420EF00638E2300008041008D
:1071C0001040BA000160EF000000060020530000EC
:1071D000472000004E4F00004953000045200000AA
:1071E000202000002020000020200000202000009F
:1071F00020200000202000002D2000004E6F000005
:1072000069730000650D00000A0000005420EF00C3
:107210002302200083015000050031002392230047
:10722000008041001040BA000160EF00000006003D
:107230002092230083814100808141001380BA00A5
:107240000000060020536D00472077005245610082
:10725000562072002020650020202000202072008F
:107260002020650020207600202069002020730067
:107270002D20690047656F0074206E0053470D0094
:1072800020660A00697200005420EF00030220000B
:107290008301500005003100039623000080410067
:1072A0001040BA000160EF000000060000962300C5
:1072B00083814100808141001380BA0000000600F4
:1072C00020532000472053005445470053542000CA
:1072D0002049690032433200202063002020200032
:1072E0002020620020207500202073002D200D003A
:1072F00045780A006572000063690000736500004C
:107300005420EF00C301200083015000050031002C
:10731000C3992300008041001040BA000160EF00D3
:1073200000000600C0992300838141008081410054
:107330001380BA0000000600205353004720470086
:10734000534C20004545740050206F002020200041
:107350002020730020206C00202065002020650084
:10736000202070002D200D0050750A0074200000B0
:107370005420EF00439C2300008041001040BA00DD
:107380000160EF00000006000D0A00003D3D000016
:107390003D3D00003D3D00003D3D00003D3D000005
:1073A00020460000696C000065200000436F00006B
:1073B0006D6D0000616E000064730000203D0000F0
:1073C0003D3D00003D3D00003D3D00000D0A000038
:1073D000000000005420EF00430220008301500011
:1073E0000500310063A02300008041001040BA0076
:1073F0000160EF000000060060A0230083814100CF
:10740000808141001380BA0000000600204327005D
:107410004F5073005920720073726300632027007D
:10742000647320007420740020206F00202020004E
:107430002D202700436F640070697300657374002A
:107440002074270068650D0020660A00696C000042
:10745000652000005420EF00E3012000830150006C
:107460000500310063A42300008041001040BA00F1
:107470000160EF000000060060A42300838141004A
:10748000808141001380BA000000060020432000E4
:10749000524566004154690045206C006E616500EC
:1074A0006D6520002020270020206E002020610034
:1074B0002D206D00437265006561270074650D0025
:1074C00020740A00686500005420EF00E3012000EA
:1074D000830150000500310003A823000080410013
:1074E0001040BA000160EF000000060000A8230071
:1074F00083814100808141001380BA0000000600B2
:1075000020442000454C6600206E6900616D6C00CF
:1075100065206500202020002020270020206E000C
:10752000202061002D206D00446565006C652700FA
:1075300074650D0020740A00686500005420EF0097
:10754000A3AA2300008041001040BA000160EF00B0
:1075500000000600204400004952000020200000E6
:10756000202000002020000020200000202000001B
:1075700020200000202000002D2000004C69000089
:1075800073740000206400006972000065630000ED
:10759000746F0000727900000D0A00000000000006
:1075A0005420EF0003022000830150000500310049
:1075B000C3AE2300008041001040BA000160EF001C
:1075C00000000600C0AE230083814100808141009D
:1075D0001380BA000000060020446600554D690083
:1075E00050206C006E6165006D6520002020270032
:1075F00020206E002020610020206D002D206500DD
:107600004865270078200D0064750A006D70000041
:10761000206F0000662000005420EF00830220004D
:10762000830150000500310083B223000080410037
:107630001040BA000160EF000000060080B2230095
:1076400083814100808141001380BA000000060060
:1076500020452000585064004C4F61005245740092
:1076600020206100202020002020730020207400B2
:10767000202072002D20750045786300706C740026
:107680006F727500657372002074650068650D0087
:1076900020530A004420000063610000726400006F
:1076A0005420EF0023032000830150000500310027
:1076B000C3B62300008041001040BA000160EF0013
:1076C00000000600C0B62300838141008081410094
:1076D0001380BA0000000600205373004420740099
:1076E000494E650049546D00202020002020640090
:1076F0002020610020207400202061002D20200027
:10770000496E730069747400696172006C69750078
:1077100073656300207474006865750020537200FF
:10772000442065006361730072640D0020660A00E6
:10773000696C000065200000737900005420EF00A0
:10774000030220008301500005003100A3BB230089
:10775000008041001040BA000160EF000000060008
:10776000A0BB230083814100808141001380BA00C7
:1077700000000600204D740044206F006E6172000E
:107780006D657900202020002020270020206E0039
:107790002020610020206D002D206500437227000D
:1077A00065610D0074650A002064000069720000C4
:1077B000656300005420EF00230320008301500084
:1077C0000500310063BF2300008041001040BA0073
:1077D0000160EF000000060060BF230083814100CC
:1077E000808141001380BA00000006002046780026
:1077F000494C7400452020005752610049546E00E6
:1078000045206400544520005354630020206C0040
:107810002D206F004372730065616500746573000D
:107820007320200061207400666968006C65650043
:107830002C202000777266006974690065736C0003
:10784000207365006F6D0D0065200A0074650000EF
:107850005420EF0063022000830150000500310036
:1078600043C42300008041001040BA000160EF00D3
:107870000000060040C42300838141008081410054
:107880001380BA00000006002054650059507800AB
:10789000452074006E6120006D656600202069003F
:1078A00020206C0020206500202020002D202700B3
:1078B0004C696E007374610020636D006F6E65002B
:1078C000746527006E740D0073200A006F66000057
:1078D000207400005420EF00C303200083015000F7
:1078E0000500310063C82300008041001040BA0049
:1078F0000160EF000000060060C8230083814100A2
:10790000808141001380BA0000000600205320004F
:1079100045437300544F6500522063003C78740067
:1079200078786F003E20720020202C00202020005C
:107930002D20530044697000737061006C61630016
:10794000792065007365200063746B006F726500B9
:1079500020787900787820002E20740050726F0013
:107960006573200073207100456E750074656900B1
:1079700072207400666F0D0072200A006E650000B0
:10798000787400005420EF0043022000830150006F
:1079900005003100E3CD2300008041001040BA0013
:1079A0000160EF0000000600E0CD2300838141006C
:1079B000808141001380BA0000000600205172004F
:1079C000464F7900524D20004154610020206E0046
:1079D000202064002020200020204600202041009C
:1079E0002D2054005A653100726F2000207426004B
:1079F000686520002044320069720D0065630A004A
:107A0000746F00005420EF00C30320008301500076
:107A100005003100E3D12300008041001040BA008E
:107A20000160EF0000000600E0D1230083814100E7
:107A3000808141001380BA000000060020446800E5
:107A4000454C650045546E004520200044496400C3
:107A50005220650020206C0020206500202074004A
:107A60002D206500446573006C652000746574000A
:107A700073206800616C65006C20200066696400FA
:107A80006C65690073207200696E65002074630084
:107A90006865740020646F00697272006563790024
:107AA000746F0D0072790A0020610D006E640A0087
:107AB000207400005420EF00E301200083015000F7
:107AC0000500310063D72300008041001040BA0058
:107AD0000160EF000000060060D7230083814100B1
:107AE000808141001380BA00000006003D3D610026
:107AF0003D3D6E003D3D64003D3D73003D3D200039
:107B000020423D0061743D0074653D0072793D0086
:107B10002F433D0068613D0072673D0065200D0008
:107B2000436F0A006D6D00005420EF0003DA23005C
:107B3000008041001040BA000160EF000000060024
:107B40002042000041540000542000005354000023
:107B50004154000055530000202000002020000068
:107B6000202000002D2000002842000053290000A2
:107B70002042000061740000742000005374000073
:107B800061740000757300000D0A00000000000021
:107B90005420EF0043DD2300008041001040BA0074
:107BA0000160EF0000000600204200004154000088
:107BB000542000005354000041540000555300006D
:107BC0003120000020200000202000002D20000097
:107BD00028420000533100002920000042610000CB
:107BE000747400002053000074610000747500007C
:107BF000733100000D0A0000000000005420EF0067
:107C0000E30120008301500005003100A3E12300BF
:107C1000008041001040BA000160EF000000060043
:107C2000A0E1230083814100808141001380BA00DC
:107C300000000600204220004154520054204D0014
:107C4000434820004152740047456F0020532000F4
:107C5000594E4600432043002D20430028420D008A
:107C600043530A002920000053650000747300008C
:107C70005420EF00C30220008301500005003100B2
:107C800043E52300008041001040BA000160EF008E
:107C90000000060040E5230083814100808141000F
:107CA0001380BA00000006002042410041546200E7
:107CB0005420730046412000535473002043740045
:107CC000484161005247740045206500544520003A
:107CD000524D6F00494E660041542000494F6300E9
:107CE0004E2068002D206100284272004643670044
:107CF0005429650020530D0065740A0073200000AC
:107D00005420EF00430320008301500005003100A0
:107D1000C3E92300008041001040BA000160EF0079
:107D200000000600C0E923008381410080814100FA
:107D30001380BA0000000600204268004154200071
:107D400054204200534561004C46740020447400A6
:107D50004953650043487200415269004745650038
:107D60002052730041542000452028004C4F2E0023
:107D7000202D300020283500425325004452250094
:107D8000204C2F004F296400206661006F7279003B
:107D9000204C290053440D00204E0A00694D00007C
:107DA0005420EF00630320008301500005003100E0
:107DB000C3EE2300008041001040BA000160EF00D4
:107DC00000000600C0EE2300838141008081410055
:107DD0001380BA00000006002042690041544D00A3
:107DE00054206800534520004C4642002044610066
:107DF000495374004348740041526500474572007E
:107E00002052690041546500452073004849200014
:107E1000202D2800202831004253250044522500FF
:107E200020482F0049296400206661006F727900A4
:107E30002072290065670D00756C0A0061720000F0
:107E4000204E00005420EF00A302200083015000C8
:107E500005003100E3F32300008041001040BA0028
:107E60000160EF0000000600E0F323008381410081
:107E7000808141001380BA000000060020536E008C
:107E800045547300204274004154610054206C003A
:107E900044416C005445610020207400202069009A
:107EA0002D206F0028536E004244200029204400FA
:107EB00057726100697474006520650074680D0074
:107EC00065200A004241000054540000204900008F
:107ED0005420EF0003022000830150000500310010
:107EE00043F82300008041001040BA000160EF0019
:107EF0000000060040F8230083814100808141009A
:107F00001380BA00000006002047660045546F0049
:107F10002042200041543C005420430052456D0053
:107F2000472064003C782000783E4300202D6F00FD
:107F3000204764006574650020423E0061740D00B6
:107F400074200A00696E00005420EF00A302200094
:107F5000830150000500310003FC23000080410034
:107F60001040BA000160EF000000060000FC230092
:107F700083814100808141001380BA000000060027
:107F8000204968004E4965005420200042414200CB
:107F9000545461002045740045507400524F6500F0
:107FA0004D20720034417900482D200031314500C8
:107FB00041484500202050002D205200496E4F00BE
:107FC00069744D0069610D006C690A007A650000F2
:107FD000207400005420EF00A30320008301500010
:107FE0000500310063002400008041001040BA0009
:107FF0000160EF0000000600600024008381410062
:10800000808141001380BA000000060020202C006F
:108010002020490020204200202045002020390057
:108020002020350020202C00202049002020420064
:10803000202045002849310042453000342C2C00D6
:108040004942490045344200352C4500494231003F
:10805000453530002C49350042452C003735490064
:108060002C49420042454500382C3100494231003C
:1080700045382900352C0D0049420A0045390000D9
:108080005420EF000303200083015000050031005D
:10809000C3052400008041001040BA000160EF00D9
:1080A00000000600C005240083814100808141005A
:1080B0001380BA000000060020446F00554D660092
:1080C000502020004241740054546800204565004F
:1080D00045502000524F42004D206100284474005A
:1080E0004245740029206500202D7200204479004B
:1080F00069732000706C4500617945002074500060
:108100006865520020634F006F6E4D0074650D006E
:108110006E740A00732000005420EF0083092400CD
:10812000008041001040BA000160EF00000006002E
:10813000204C00004320000055500000202000008B
:10814000202000002020000020200000202000002F
:10815000202000002D2000004C6900006E6500000A
:108160006172000020430000686700002056000094
:1081700020550000700D00000A0000005420EF00A0
:10818000A30C2400008041001040BA000160EF0001
:1081900000000600204C000043200000444E000078
:1081A00020200000202000002020000020200000CF
:1081B00020200000202000002D2000004C6900003D
:1081C0006E650000617200002043000068670000D7
:1081D00020560000204400006E0D00000A00000040
:1081E0005420EF00230220008301500005003100DD
:1081F000C3102400008041001040BA000160EF006D
:1082000000000600C01024008381410080814100ED
:108210001380BA0000000600204C200043207400A8
:1082200031416F00202020002020610020206200CA
:1082300020206F0020207500202074002D202000B9
:1082400053653100742041004C690D006E650A00D1
:108250006172000020430000686700005420EF00B6
:10826000230220008301500005003100A3142400E4
:10827000008041001040BA000160EF0000000600DD
:10828000A014240083814100808141001380BA0042
:1082900000000600204C20004320740032416F0093
:1082A00020202000202061002020620020206F007C
:1082B00020207500202074002D20200053653200FE
:1082C000742041004C690D006E650A006172000067
:1082D00020430000686700005420EF006302200084
:1082E0008301500005003100831824000080410004
:1082F0001040BA000160EF00000006008018240062
:1083000083814100808141001380BA000000060093
:10831000204C6F00432020004D496D00442069002F
:1083200020206400202072002020610020206E00A8
:10833000202067002D206500536520007420280050
:108340004C6933006E6532006172290020430D00D4
:1083500068670A0020560000207400005420EF00D7
:10836000A31B2400008041001040BA000160EF0010
:1083700000000600204C0000432000004D4100009A
:1083800058200000202000002020000020200000B5
:1083900020200000202000002D2000004C6900005B
:1083A0006E650000617200002043000068670000F5
:1083B00020560000204D0000617800000D0A0000EA
:1083C000000000005420EF00E31E24000080410064
:1083D0001040BA000160EF0000000600204C0000D1
:1083E000432000004D4900004E20000020200000E6
:1083F000202000002020000020200000202000007D
:108400002D2000004C6900006E65000061720000C4
:10841000204300006867000020560000204D000047
:10842000696E00000D0A00000D0A00000000000047
:108430005420EF0043222400008041001040BA0085
:108440000160EF00000006003D3D00003D3D0000E2
:108450003D3D00003D3D00003D3D0000205000003E
:108460006F77000065720000204F00006E2F000043
:108470004F660000662000003D3D00003D3D0000CD
:108480003D3D00003D3D00003D3D00000D0A000067
:10849000000000005420EF0063252400008041000C
:1084A0001040BA000160EF0000000600204100000B
:1084B0004E4100004C4F0000472000004F4E00008E
:1084C00020200000202000002020000020200000AC
:1084D0002D200000416E0000616C00006F670000FD
:1084E0002073000075700000706C0000792000009F
:1084F0006F6E00000D0A0000000000005420EF0025
:10850000A3282400008041001040BA000160EF0061
:1085100000000600204100004E4100004C4F0000CA
:10852000472000004F4600004620000020200000A9
:1085300020200000202000002D200000416E0000BF
:10854000616C00006F670000207300007570000010
:10855000706C0000792000006F660000660D00005E
:108560000A0000005420EF00E32B240000804100AB
:108570001040BA000160EF00000006002057000024
:1085800049460000492000004F4E00002020000016
:1085900020200000202000002020000020200000DB
:1085A0002D2000005769000046690000207000007F
:1085B0006F77000065720000206F00006E0D0000F4
:1085C0000A0000005420EF00E32E24000080410048
:1085D0001040BA000160EF000000060020570000C4
:1085E00049460000492000004F4600004620000098
:1085F000202000002020000020200000202000007B
:108600002D2000005769000046690000207000001E
:108610006F77000065720000206F00006666000042
:108620000D0A0000000000005420EF000332240077
:10863000008041001040BA000160EF000000060019
:1086400020530000442000004F4E00002020000076
:10865000202000002020000020200000202000001A
:10866000202000002D200000534400004361000042
:1086700072640000207000006F77000065720000D7
:10868000206F00006E0D00000A0000005420EF0073
:1086900023352400008041001040BA000160EF0043
:1086A0000000060020530000442000004F46000058
:1086B0004620000020200000202000002020000094
:1086C00020200000202000002D2000005344000046
:1086D0004361000072640000207000006F770000AA
:1086E00065720000206F0000666600000D0A000041
:1086F000000000005420EF00633824000080410097
:108700001040BA000160EF000000060020470000A2
:1087100050530000204F00004E2000002020000099
:108720002020000020200000202000002020000049
:108730002D2000004750000053200000706F000003
:1087400077650000722000006F6E00000D0A0000C7
:10875000000000005420EF00633B24000080410033
:108760001040BA000160EF00000006002047000042
:1087700050530000204F000046460000202000001B
:1087800020200000202000002020000020200000E9
:108790002D2000004750000053200000706F0000A3
:1087A00077650000722000006F660000660D000013
:1087B0000A0000005420EF00C30120008301500094
:1087C00005003100633F2400008041001040BA00E2
:1087D0000160EF0000000600603F2400838141003B
:1087E000808141001380BA0000000600205365001C
:1087F00047206E004F4E20002020700020206F0088
:1088000020207700202065002020720020202000FA
:108810002D206F0053696E00676E0D00616C0A00B9
:10882000204700005420EF00E301200083015000A6
:1088300005003100E3422400008041001040BA00EE
:108840000160EF0000000600E04224008381410047
:10885000808141001380BA000000060020532000F0
:10886000472070004F466F004620770020206500AB
:10887000202072002020200020206F002020660091
:108880002D20660053690D00676E0A00616C0000C0
:1088900020470000656E00005420EF00834524004F
:1088A000008041001040BA000160EF0000000600A7
:1088B00041740000746500006D70000074200000B9
:1088C000746F0000207200006561000064200000E9
:1088D0007061000073740000206500006E64000089
:1088E0000D0A0000000000005420EF00034824009F
:1088F000008041001040BA000160EF000000060057
:108900002A2A00002A20000053650000637400003A
:108910006F72000020640000756D00007020000080
:10892000656E000064650000642000002A2A0000D3
:108930002A0D00000A0000005420EF00834A2400A2
:10894000008041001040BA000160EF000000060006
:108950002A2A00002A20000053650000742000002D
:1089600047500000532000004C4500004420000008
:108970004F6E000020740000696D0000652000004B
:10898000776100007320000025750000206E000054
:108990006F7700003A200000257500000D0A0000E6
:1089A000000000005420EF00C301200083015000AC
:1089B00005003100E34E2400008041001040BA0061
:1089C0000160EF0000000600E04E240083814100BA
:1089D000808141001380BA00000006002A2A20008E
:1089E0002A202500536575007420200047506E0032
:1089F00053206F004C45770044203A004F6620001A
:108A000066202500746975006D650D0020770A00E9
:108A1000617300005420EF00635124000080410086
:108A20001040BA000160EF00000006002A2A000092
:108A30002A200000536500007420000046690000F1
:108A40006E650000204C00006F6300006B2000008A
:108A500053630000616C0000650D00000A00000017
:108A60005420EF00C3532400008041001040BA009E
:108A70000160EF00000006002A2A00002A20000002
:108A8000526500007365000074200000444F000030
:108A9000204C00006F6F0000700D00000A00000005
:108AA0005420EF00C3552400008041001040BA005C
:108AB0000160EF00000006002A2A00002A200000C2
:108AC00054430000205200005443000020440000A2
:108AD0006174000065200000546900006D650000AD
:108AE0000D0A0000000000005420EF00E302200007
:108AF000830150000500310003592400008041002B
:108B00001040BA000160EF00000006000059240088
:108B100083814100808141001380BA00000006007B
:108B20002054720043203A00525425004320640030
:108B300044612C007465200020264D0020546900FB
:108B4000696D6E0065203A002D2025005972640081
:108B50003A252C00642C2000204D53006F6E6500D8
:108B60003A256300642C3A002044250061796400B2
:108B70003A250D00642C0A00204800005420EF0024
:108B8000A35C2400008041001040BA000160EF00A7
:108B9000000006002A2A00002A2000004765000085
:108BA00074200000576100006B6500002F53000027
:108BB0006C650000657000000D0A000000000000F8
:108BC0005420EF00C35E2400008041001040BA0032
:108BD0000160EF00000006002A2A00002A200000A1
:108BE000544300002031000032330000340D0000F7
:108BF0000A0000005420EF004302200083015000CF
:108C00000500310063612400008041001040BA007B
:108C10000160EF00000006006061240083814100D4
:108C2000808141001380BA000000060020543A0001
:108C3000432025003132780033342C00202D2000D1
:108C40002042420079747900653174003A2565004C
:108C5000782C340020423A0079742500653278007F
:108C60003A250D00782C0A0020420000797400009B
:108C7000653300005420EF0063642400008041004D
:108C80001040BA000160EF00000006002A2A000030
:108C90002A200000544300002047000065740000B3
:108CA000204F000070740000696F00006E730000B8
:108CB0000D0A0000000000005420EF00836624002D
:108CC000008041001040BA000160EF000000060083
:108CD00020540000432000004F7000007469000021
:108CE0006F6E0000732000002D2000004869000016
:108CF0003A250000782C0000204C00006F3A00005C
:108D0000257800000D0A0000000000005420EF004C
:108D100023692400008041001040BA000160EF0088
:108D2000000006002A2A00002A2000005443000008
:108D300020520000657600000D0A000000000000CF
:108D40005420EF00C36A2400008041001040BA00A4
:108D50000160EF00000006002054000043200000E6
:108D600052650000762000002D20000052650000B2
:108D700076480000693A0000257500002052000086
:108D8000657600004C6F00003A250000750D00006C
:108D90000A0000005420EF00636D240000804100B1
:108DA0001040BA000160EF00000006002A2A00000F
:108DB0002A2000005443000020410000637100009D
:108DC000204D00006F640000650D00000A000000E7
:108DD0005420EF00436F2400008041001040BA008F
:108DE0000160EF00000006002A2A00002A2000008F
:108DF0005443000020470000657400002057000025
:108E0000616B000065200000526500006173000086
:108E10006F6E00000D0A0000000000005420EF00FB
:108E2000A3712400008041001040BA000160EF00EF
:108E3000000006002054000043200000576100009D
:108E40006B65000052650000617300006F6E0000EA
:108E50003A250000780D00000A0000005420EF00C1
:108E6000A3732400008041001040BA000160EF00AD
:108E70000000060020200000487500006464000027
:108E80006C6500002054000065730000743A000017
:108E9000200000005420EF00637524000080410092
:108EA0001040BA000160EF00000006004F6E0000A5
:108EB0000D0A0000000000005420EF00837624001B
:108EC000008041001040BA000160EF000000060081
:108ED0004F660000660D00000A0A00000000000056
:108EE0005420EF00C3772400008041001040BA00F6
:108EF0000160EF00000006002A2A00002A2000007E
:108F0000456E00007465000072200000536C000084
:108F10006565000070790000204D00006F6400005E
:108F2000650D00000A0000005420EF00037A2400C1
:108F3000008041001040BA000160EF000000060010
:108F40002A2A00002A20000054430000205200007A
:108F500065730000657400000D0A00000000000049
:108F60005420EF00C37B2400008041001040BA0071
:108F70000160EF00000006002A2A00002A200000FD
:108F80004765000074200000536C00006565000018
:108F9000707900002052000061740000650D00002F
:108FA0000A0000005420EF00E37D2400008041000F
:108FB0001040BA000160EF000000060020540000DD
:108FC00043200000536C00006565000070790000CC
:108FD0002052000061740000653A0000257800000E
:108FE0000D0A0000000000005420EF000380240060
:108FF000008041001040BA000160EF000000060050
:109000002A2A00002A200000536500007420000076
:10901000536C00006565000070790000205200006C
:1090200061740000650D00000A0000005420EF008C
:1090300023822400008041001040BA000160EF004C
:10904000000006002A2A00002A20000057720000B3
:1090500069740000696E000067200000534E000034
:109060000D0A0000000000005420EF0003842400DB
:10907000008041001040BA000160EF0000000600CF
:109080002A2A00002A200000476500007420000002
:10909000534E00000D0A0000000000005420EF00B5
:1090A000A3852400008041001040BA000160EF0059
:1090B00000000600534E0000202D00002025000077
:1090C000730D00000A0000005420EF000387240005
:1090D000008041001040BA000160EF00000006006F
:1090E0002A2A00002A20000057720000697400003C
:1090F000652000004461000074650000206F0000DE
:10910000662000004D6100006E7500006661000081
:10911000747500007265000020250000752F0000A6
:10912000257500000D0A0000000000005420EF002B
:10913000238A2400008041001040BA000160EF0043
:10914000000006002A2A00002A20000047650000CF
:10915000742000004461000074650000206F00006E
:10916000662000004D6100006E7500006661000021
:109170006374000075720000650D00000A000000B5
:109180005420EF00C38C2400008041001040BA003E
:109190000160EF00000006004D6100006E750000E8
:1091A00066610000637400007572000065200000B5
:1091B0004461000074650000202D0000202500009F
:1091C000752F0000257500000D0A0000000000004A
:1091D0005420EF00438F2400008041001040BA006B
:1091E0000160EF00000006002A2A00002A2000008B
:1091F000536500006E640000696E00006720000087
:10920000534700002046000072650000712F0000E7
:10921000416D0000700D00000A0000005420EF00B6
:10922000A3912400008041001040BA000160EF00CB
:10923000000006002A2A00002A20000047650000DE
:109240007420000047500000532000004D730000C0
:1092500067200000257800000D0A000000000000D3
:109260005420EF00C3932400008041001040BA0056
:109270000160EF00000006002A2A00002A200000FA
:109280005347000020520000657600000D0A0000E0
:10929000000000005420EF0063952400008041008E
:1092A0001040BA000160EF000000060053470000C4
:1092B0002052000065760000202D000020520000A2
:1092C00065760000486900003A250000782C00000F
:1092D00020520000657600004C6F00003A25000027
:1092E000780D00000A0000005420EF0003982400CD
:1092F000008041001040BA000160EF00000006004D
:109300002A2A00002A2000005347000020530000B2
:10931000494E0000450D00000A0000005420EF00F7
:10932000A3992400008041001040BA000160EF00C2
:10933000000006002A2A00002A20000053470000EF
:1093400020440000430D00000A0000005420EF00FC
:10935000239B2400008041001040BA000160EF0010
:10936000000006002A2A00002A20000053470000BF
:10937000204E00004F490000534500000D0A000038
:10938000000000005420EF00E39C24000080410016
:109390001040BA000160EF00000006002A2A000019
:1093A0002A2000005347000020520000414D0000D9
:1093B000500D00000A0000005420EF00839E24009E
:1093C000008041001040BA000160EF00000006007C
:1093D0002A2A00002A2000005347000020500000E5
:1093E000554C0000534500000D0A0000000000002D
:1093F0005420EF0043A02400008041001040BA0038
:109400000160EF00000006002A2A00002A20000068
:109410005347000020530000514100005552000006
:10942000450D00000A0000005420EF0003A22400B4
:10943000008041001040BA000160EF00000006000B
:109440002A2A00002A200000534700002054000070
:109450004553000054200000493200004320000022
:109460002854000043430000207400006F200000D7
:10947000436100006E630000656C0000292000005D
:109480002E2E00002E0D00000A0000005420EF00D8
:1094900023A52400008041001040BA000160EF00C5
:1094A000000006002A2A00002A200000534700007E
:1094B000205300006C650000657000000D0A00007C
:1094C000000000005420EF00E3A6240000804100CB
:1094D0001040BA000160EF00000006002A2A0000D8
:1094E0002A2000005347000020570000414B000095
:1094F000450D00000A0000005420EF0083A824005E
:10950000008041001040BA000160EF00000006003A
:109510002A2A00002A2000005443000020540000A2
:109520004553000054200000493200004320000051
:109530002854000043430000207400006F20000006
:10954000436100006E630000656C0000292000008C
:109550002E2E00002E0D00000A0000005420EF0007
:10956000A3AB2400008041001040BA000160EF006E
:10957000000006002A2A00002A2000005374000080
:1095800061720000742000004469000073630000F1
:10959000697000006C6900006E6700000D0A000031
:1095A000000000005420EF00E3AD240000804100E3
:1095B0001040BA000160EF00000006002A2A0000F7
:1095C0002A200000537400006F7000002044000047
:1095D0006973000063690000706C0000696E000030
:1095E000670D00000A0000005420EF0003B02400C3
:1095F000008041001040BA000160EF00000006004A
:109600002A2A00002A20000047650000742000007C
:1096100047500000530D00000A0000005420EF00E6
:10962000A3B12400008041001040BA000160EF00A7
:10963000000006002A2A00002A200000496E0000CF
:10964000697400002045000045500000524F0000A2
:109650004D0D00000A0000005420EF0083B32400E9
:10966000008041001040BA000160EF0000000600D9
:109670002A2A00002A200000496E000069740000B8
:10968000204C00006F77000020450000455000008E
:10969000524F00004D0D00000A0000005420EF0062
:1096A000A3B52400008041001040BA000160EF0023
:1096B000000006002A2A00002A200000496E00004F
:1096C0006974000020560000434F00002045000050
:1096D00045500000524F00004D0D00000A000000F0
:1096E0005420EF00C3B72400008041001040BA00AE
:1096F0000160EF00000006002A2A00002A20000076
:1097000054430000204C000065610000726E0000B0
:10971000204F00006E0D00000A0000005420EF00F2
:10972000A3B92400008041001040BA000160EF009E
:10973000000006002A2A00002A20000054430000EE
:10974000204C000065610000726E0000204F000098
:1097500066660000720A0000000000005420EF005E
:10976000A3BB2400008041001040BA000160EF005C
:10977000000006002A2A00002A2000004765000099
:1097800074200000564300004F0D00000A00000046
:109790005420EF00E3012000830150000500310058
:1097A00043BE2400008041001040BA000160EF0079
:1097B0000000060040BE24008381410080814100FA
:1097C0001380BA0000000600564378004F202C009A
:1097D0002D20200042794200743479003A2574002B
:1097E000782C310020423A0079742500333A780011
:1097F00025780D002C200A00427900007432000008
:109800003A2500005420EF00E3C02400008041000E
:109810001040BA000160EF00000006002A2A000094
:109820002A20000047650000742000005443000017
:10983000204C00006F6300006B2000005374000098
:1098400061740000757300000D0A00000000000044
:109850005420EF0043C32400008041001040BA00B0
:109860000160EF00000006004C6F0000636B000019
:10987000205300007461000074750000733A00000A
:10988000257800002C200000564300004F5F0000A8
:1098900044410000433A0000257500000D0A000015
:1098A000000000005420EF00E3C5240000804100C8
:1098B0001040BA000160EF00000006002A2A0000F4
:1098C0002A200000575200004954000045200000A3
:1098D000564300004F200000746F00002045000038
:1098E00045500000524F00004D0D00000A000000DE
:1098F0005420EF0043C82400008041001040BA000B
:109900000160EF00000006002A2A00002A20000063
:10991000524500004144000020560000434F000023
:1099200020660000726F00006D20000045450000B9
:10993000505200004F4D00000D0A000000000000D2
:109940005420EF00C3CA2400008041001040BA0038
:109950000160EF0000000600454500005052000085
:109960004F4D000020440000414300005F560000BE
:10997000434F00003A250000750D00000A0000006A
:109980005420EF00C3CC2400008041001040BA00F6
:109990000160EF00000006002A2A00002A200000D3
:1099A0005365000074200000564300004F0D000076
:1099B0000A0000005420EF0063CE24000080410024
:1099C0001040BA000160EF00000006002A2A0000E3
:1099D0002A2000005365000074200000444100006C
:1099E000430D00000A0000005420EF0003D02400C3
:1099F000008041001040BA000160EF000000060046
:109A00002A2A00002A200000456E0000746500002C
:109A1000726900006E67000020470000505300008C
:109A2000204D00004F4E0000495400004F520000EE
:109A3000206D00006F640000650D00000A0000004A
:109A40005420EF00C3D22400008041001040BA002F
:109A50000160EF00000006002A2A00002A20000012
:109A6000456E000074650000726900006E670000BA
:109A700020560000434F0000204D00004F4E0000D4
:109A8000495400004F520000206D00006F64000038
:109A9000650D00000A0000005420EF0083D524006B
:109AA000008041001040BA000160EF000000060095
:109AB0002A2A00002A200000536500006E6400007E
:109AC000696E000067200000444100004320000050
:109AD00054650000737400000D0A000000000000CF
:109AE0005420EF00C3D72400008041001040BA008A
:109AF0000160EF00000006002A2A00002A20000072
:109B0000436100006E630000656C0000205300009C
:109B1000656E0000740D00000A0000005420EF0084
:109B2000A3D92400008041001040BA000160EF007A
:109B3000000006002A2A00002A20000054430000EA
:109B4000207400006F200000536C00006565000069
:109B5000700D00000A0000005420EF0083DB240099
:109B6000008041001040BA000160EF0000000600D4
:109B70002A2A00002A200000476500007420000007
:109B80004F730000636900006C6C0000617400009A
:109B90006F72000020540000656D000070650000C9
:109BA0007261000074750000726500000D0A00000B
:109BB000000000005420EF0063DE2400008041001C
:109BC0001040BA000160EF00000006004F73000073
:109BD000636900006C6C0000617400006F7200002B
:109BE00020540000656D0000706500007261000087
:109BF00074750000726500003A20000025640000C2
:109C00000D0A0000000000005420EF0003E12400D2
:109C1000008041001040BA000160EF000000060023
:109C20002A2A00002A200000476500007420000056
:109C300052650000677500006C610000746F0000E1
:109C400072200000546500006D7000006572000015
:109C50006174000075720000650D00000A000000CC
:109C60005420EF00C3E32400008041001040BA00FC
:109C70000160EF00000006005265000067750000FB
:109C80006C610000746F00007220000054650000D9
:109C90006D70000065720000617400007572000054
:109CA000653A000020250000640D00000A00000055
:109CB0005420EF0043E62400008041001040BA0029
:109CC0000160EF00000006002A2A00002A200000A0
:109CD000476500007420000053630000616E0000BF
:109CE0004E640000780D00000A0000005420EF00D0
:109CF00023E82400008041001040BA000160EF001A
:109D00000000060053630000616E00004E64000016
:109D1000783A000020250000640D00000A000000D1
:109D20005420EF00C3E92400008041001040BA0035
:109D30000160EF00000006002A2A00002A2000002F
:109D4000557000006461000074650000204E000042
:109D50005620000050610000726100006D73000029
:109D60000D0A0000000000005420EF0003EC240066
:109D7000008041001040BA000160EF0000000600C2
:109D80002A2A00002A2000005769000046690000C6
:109D9000204F00006E200000447500007269000032
:109DA0006E670000204300006861000072670000D9
:109DB000650D00000A0000005420EF0083EE24002F
:109DC000008041001040BA000160EF000000060072
:109DD0002A2A00002A200000576900004669000076
:109DE000204F0000666600002044000075720000ED
:109DF000696E000067200000436800006172000087
:109E0000676500000D0A0000000000005420EF000C
:109E100023F12400008041001040BA000160EF00EF
:109E2000000006002A2A00002A2000004E650000DB
:109E30006F20000052650000636F00007264000034
:109E4000696E0000672000004F6E00000D0A0000E0
:109E5000000000005420EF0063F324000080410064
:109E60001040BA000160EF00000006002A2A00003E
:109E70002A2000004C6900006E650000617200003D
:109E80002063000068670000205600002055000095
:109E90007020000028250000642900000D0A000041
:109EA000000000005420EF00E3F524000080410092
:109EB0001040BA000160EF00000006002A2A0000EE
:109EC0002A2000004C6900006E65000061720000ED
:109ED0002063000068670000205600002044000056
:109EE0006E20000028250000642900000D0A0000F3
:109EF000000000005420EF0063F8240000804100BF
:109F00001040BA000160EF00000006002A2A00009D
:109F10002A2000004C6900006E650000617200009C
:109F2000206300006867000020560000204D0000FC
:109F3000696400002028000033320000290D000071
:109F40000A0000005420EF00E3FA240000804100E2
:109F50001040BA000160EF00000006002A2A00004D
:109F60002A2000004C6900006E650000617200004C
:109F70002063000068670000202E000031200000F0
:109F8000416D0000702000002825000064290000B9
:109F90000D0A0000000000005420EF0083FD2400A3
:109FA000008041001040BA000160EF000000060090
:109FB0002A2A00002A2000004C6900006E6500007B
:109FC000617200002063000068670000202E00001E
:109FD00032200000416D00007020000028250000A4
:109FE000642900000D0A0000000000005420EF006A
:109FF00023002500008041001040BA000160EF00FE
:10A00000000006002A2A00002A2000004C690000F7
:10A010006E65000061720000206300006867000048
:10A02000202E000035200000416D0000702000004F
:10A0300028250000642900000D0A0000000000002F
:10A040005420EF00C3022500008041001040BA00F8
:10A050000160EF00000006002A2A00002A2000000C
:10A060004C6900006E650000617200002063000012
:10A070006867000020310000204100006D70000082
:10A080002028000025640000290D00000A000000BF
:10A090005420EF0043052500008041001040BA0025
:10A0A0000160EF00000006002A2A00002A200000BC
:10A0B0004C6900006E6500006172000020630000C2
:10A0C0006867000020320000204100006D70000031
:10A0D0007320000028250000642900000D0A0000FC
:10A0E000000000005420EF00E3072500008041003D
:10A0F0001040BA000160EF00000006002A2A0000AC
:10A100002A2000004C6900006E65000061720000AA
:10A11000206300006867000020560000204D00000A
:10A12000617800002028000025640000290D00004F
:10A130000A0000005420EF00630A2500008041005F
:10A140001040BA000160EF00000006002A2A00005B
:10A150002A2000004C6900006E650000617200005A
:10A16000206300006867000020560000204D0000BA
:10A17000696E00002028000025640000290D000001
:10A180000A0000005420EF00E30C2500008041008D
:10A190001040BA000160EF00000006002A2A00000B
:10A1A0002A20000053440000436100007264000054
:10A1B000205000006F77000065720000204F000003
:10A1C0006E0D00000A0000005420EF00030F250070
:10A1D000008041001040BA000160EF00000006005E
:10A1E0002A2A00002A200000534400004361000096
:10A1F00072640000205000006F770000657200005C
:10A20000204F0000666600000D0A000000000000FC
:10A210005420EF0043112500008041001040BA0097
:10A220000160EF00000006002A2A00002A2000003A
:10A2300053470000205000006F7700006572000057
:10A24000204F00006E0D00000A0000005420EF00B7
:10A2500023132500008041001040BA000160EF0088
:10A26000000006002A2A00002A20000053470000B0
:10A27000205000006F77000065720000204F000042
:10A28000666600000D0A0000000000005420EF0088
:10A2900023152500008041001040BA000160EF0046
:10A2A000000006002A2A00002A2000004750000073
:10A2B00053200000506F00007765000072200000FE
:10A2C0004F6E00000D0A0000000000005420EF0057
:10A2D00023172500008041001040BA000160EF0004
:10A2E000000006002A2A00002A2000004750000033
:10A2F00053200000506F00007765000072200000BE
:10A300004F660000660D00000A0000005420EF00B8
:10A3100023192500008041001040BA000160EF00C1
:10A32000000006002A2A00002A20000057690000C9
:10A3300046690000205000006F7700006572000041
:10A34000204F000046460000206F00006E200000F5
:10A35000537400006172000074750000700D0000FD
:10A360000A0000005420EF00E31B2500008041009C
:10A370001040BA000160EF00000006002A2A000029
:10A380002A200000576900004669000020500000A4
:10A390006F77000065720000204F00004E20000023
:10A3A0006F6E0000205300007461000072740000A2
:10A3B000757000000D0A0000000000005420EF003E
:10A3C000A31E2500008041001040BA000160EF008C
:10A3D000000006002A2A00002A2000005265000022
:10A3E0006365000069760000696E00006720000068
:10A3F00049500000412000006B65000065700000BE
:10A40000732000005769000046690000204F0000DB
:10A410006E0D00000A0000005420EF00832125008B
:10A42000008041001040BA000160EF00000006000B
:10A430002A2A00002A2000005265000063650000FF
:10A4400069760000696E0000672000004950000036
:10A4500041200000446F0000657300006E2700007B
:10A46000742000006B65000065700000205700003C
:10A4700069460000692000006F6E00000D0A0000B0
:10A48000000000005420EF00E3242500008041007C
:10A490001040BA000160EF00000006002A2A000008
:10A4A0002A2000005769000046690000205400007F
:10A4B00065730000742000004F6E00000D0A00005C
:10A4C000000000005420EF00E3262500008041003A
:10A4D0001040BA000160EF00000006002A2A0000C8
:10A4E0002A2000005769000046690000205400003F
:10A4F0006573000074200000616C0000726500004C
:10A500006164000079200000727500006E6E00002A
:10A51000696E0000670D00000A0000005420EF0083
:10A52000A3292500008041001040BA000160EF001F
:10A53000000006002A2A00002A20000057690000B7
:10A54000466900002054000065730000742000007C
:10A550004F660000660D00000A0000005420EF0066
:10A56000A32B2500008041001040BA000160EF00DD
:10A57000000006002A2A00002A2000005769000077
:10A58000466900002054000065730000742000003C
:10A59000616C0000726500006164000079200000B9
:10A5A0006F660000660D00000A0000005420EF00F6
:10A5B000232E2500008041001040BA000160EF000A
:10A5C000000006002A2A00002A2000005769000027
:10A5D0004669000020540000696D0000656F0000AE
:10A5E00075740000204F00006E0D00000A0000008E
:10A5F0005420EF0043302500008041001040BA0095
:10A600000160EF00000006002A2A00002A20000056
:10A61000576900004669000020540000696D000081
:10A62000656F000075740000204F00006666000032
:10A630000D0A0000000000005420EF0083322500C6
:10A64000008041001040BA000160EF0000000600E9
:10A650002A2A00002A200000536500007420000010
:10A66000576900004669000020540000696D000031
:10A67000656F0000757400003A2000002575000029
:10A68000206D0000696E00007574000065730000A5
:10A690000D0A0000000000005420EF008335250063
:10A6A000008041001040BA000160EF000000060089
:10A6B0002A2A00002A20000057690000466900008D
:10A6C000205000006F77000065720000204F0000EE
:10A6D000464600000D0A0000000000005420EF0074
:10A6E000A3372500008041001040BA000160EF0050
:10A6F000000006002A2A00002A20000057690000F6
:10A7000046690000205000006F770000657200006D
:10A71000204F00006E0D00000A0000005420EF00E2
:10A72000A3392500008041001040BA000160EF000D
:10A73000000006002A2A00002A20000053740000AE
:10A740006172000074200000412F000044200000CE
:10A75000436F00006E7600006572000073690000B0
:10A760006F6E00000D0A0000000000005420EF0092
:10A77000233C2500008041001040BA000160EF003A
:10A78000000006002A2A00002A2000004361000081
:10A790006E630000656C0000204300006D640000E3
:10A7A0000D0A0000000000005420EF00033E2500C9
:10A7B000008041001040BA000160EF000000060078
:10A7C0002A2A00002A20000053650000742000009F
:10A7D000536100006D7000006C65000020520000A5
:10A7E00061740000653A0000202500006325000028
:10A7F000756D0000730D00000A0000005420EF008A
:10A80000A3402500008041001040BA000160EF0025
:10A81000000006002A2A00002A20000053650000DC
:10A820007420000050720000656100006D7000002F
:10A8300020470000616900006E3A000020250000FA
:10A8400075640000620D00000A0000005420EF0053
:10A8500023432500008041001040BA000160EF0052
:10A86000000006002A2A00002A2000004765000098
:10A8700074200000426100007474000065720000E2
:10A8800079200000787800000D0A00000000000028
:10A890005420EF0043452500008041001040BA00DD
:10A8A0000160EF00000006004261000074740000C7
:10A8B000657200007920000041640000723A0000D7
:10A8C000202500003478000020560000616C000054
:10A8D000756500003A200000256400002028000073
:10A8E0003078000025340000782900000D0A0000AF
:10A8F000000000005420EF00E3012000830150001D
:10A900000500310063492500008041001040BA0075
:10A910000160EF00000006006049250083814100CE
:10A92000808141001380BA00000006002A2A6100DD
:10A930002A2074005772690069746F00696E6E0096
:10A940006720200046612E0073742E0020432E00E5
:10A9500068612E0072672E0065200D0054650A00A4
:10A96000726D0000696E00005420EF00E3012000CA
:10A970008301500005003100034D25000080410097
:10A980001040BA000160EF0000000600004D2500F5
:10A9900083814100808141001380BA0000000600DD
:10A9A0002A2A20002A20520057726100697474001C
:10A9B000696E6500672020004C6F2E0077202E0006
:10A9C00042612E0074742E0020442E0069730D0025
:10A9D00063680A0061720000676500005420EF00A0
:10A9E000E30120008301500005003100A350250041
:10A9F000008041001040BA000160EF000000060036
:10AA0000A050250083814100808141001380BA005D
:10AA1000000006002A2A65002A20200057725200F2
:10AA200069746100696E74006720650048692000E0
:10AA300067682E0020422E0061742E0074202E00C4
:10AA400044692E0073630D0068610A00726700009C
:10AA50005420EF0043532500008041001040BA000D
:10AA60000160EF00000006002A2A00002A200000F2
:10AA7000447500006D700000204200006174000009
:10AA80007420000045450000505200004F4D00006A
:10AA9000202A00002A2A00000D0A00000000000001
:10AAA0005420EF0003022000830150000500310014
:10AAB000C3562500008041001040BA000160EF003D
:10AAC00000000600C05625008381410080814100BE
:10AAD0001380BA00000006000D0A2A002A2A2A0064
:10AAE0002A2A2A002A2A2A002A2A2A002A2A2A006E
:10AAF0002A2A2A0020422A0061742A0074652A004A
:10AB000072792A0020530D0074610A0074750000E8
:10AB100073310000202A00005420EF0083592500E3
:10AB2000008041001040BA000160EF000000060004
:10AB30002044000065730000697200006564000035
:10AB40002043000068670000204300007572000089
:10AB5000726500006E7400003A2000002564000059
:10AB60000D0A0000000000005420EF00035C2500E7
:10AB7000008041001040BA000160EF0000000600B4
:10AB80002020000020200000204400006573000009
:10AB9000696700006E2000004361000070610000E2
:10ABA00063690000747900003A2000002564000009
:10ABB0000D0A0000000000005420EF00835E250015
:10ABC000008041001040BA000160EF000000060064
:10ABD0002020000020200000202000002020000075
:10ABE0002020000020200000202000002020000065
:10ABF0004D6F0000646500003A20000030780000CE
:10AC000025340000780D00000A0000005420EF00F9
:10AC1000E30120008301500005003100236225007C
:10AC2000008041001040BA000160EF000000060003
:10AC30002062250083814100808141001380BA0099
:10AC4000000006002020740050616100636B7400F6
:10AC5000204375006F6E730066693A0067752000C7
:10AC600072613000746978006F6E25003A203200FE
:10AC70003078780025320D0078200A00205300003B
:10AC80005420EF00C3642500008041001040BA004A
:10AC90000160EF00000006002020000020200000DE
:10ACA0004D6100006E750000666100006374000075
:10ACB00075720000652000004461000074650000AA
:10ACC0003A200000256400002F250000642F0000BA
:10ACD000256400000D0A0000000000005420EF0071
:10ACE000A3672500008041001040BA000160EF001A
:10ACF0000000060020200000202000004D61000020
:10AD00006E750000666100006374000075720000DB
:10AD10006520000044610000746100003A200000DA
:10AD2000256400000D0A0000000000005420EF0020
:10AD3000236A2500008041001040BA000160EF0046
:10AD4000000006004C61000073740000204D0000FC
:10AD500065610000737500007265000064200000EA
:10AD60004469000073630000686700003A20000037
:10AD7000256400000D0A0000000000005420EF00D0
:10AD8000A36C2500008041001040BA000160EF0074
:10AD90000000060020530000656C000066200000E3
:10ADA000446900007363000068610000726700007E
:10ADB0006520000052610000746500003A20000028
:10ADC0004C6F0000770D00000A0000005420EF00D7
:10ADD000236F2500008041001040BA000160EF00A1
:10ADE0000000060020530000656C00006620000093
:10ADF000446900007363000068610000726700002E
:10AE00006520000052610000746500003A200000D7
:10AE100048690000676800000D0A0000000000009B
:10AE20005420EF00E30120008301500005003100B1
:10AE3000C3722500008041001040BA000160EF009D
:10AE400000000600C072250083814100808141001E
:10AE50001380BA00000006000D0A2A002A2A2A00E0
:10AE60002A2A2A002A2A2A002A2A2A002A2A2A00EA
:10AE70002A2A2A0020422A0061742A0074652A00C6
:10AE800072792A0020532A0074610D0074750A003B
:10AE9000732000005420EF006375250000804100FE
:10AEA0001040BA000160EF00000006002020000002
:10AEB0002020000020200000202000002020000092
:10AEC00020200000205600006F6C0000746100001C
:10AED000676500003A200000256400000D0A0000AC
:10AEE000000000005420EF00E377250000804100BF
:10AEF0001040BA000160EF000000060020200000B2
:10AF00002020000020200000202000002020000041
:10AF100020200000204300007572000072650000D0
:10AF20006E7400003A200000256400000D0A000045
:10AF3000000000005420EF00637A250000804100EB
:10AF40001040BA000160EF00000006002020000061
:10AF5000526500006D610000696E0000696E0000BE
:10AF60006720000043610000706100006369000019
:10AF7000747900003A200000256400000D0A0000EA
:10AF8000000000005420EF00E37C25000080410019
:10AF90001040BA000160EF000000060020410000F0
:10AFA00062730000205300007461000074650000AB
:10AFB000206F0000662000004368000061720000FE
:10AFC000676500003A200000256400002525000088
:10AFD0000D0A0000000000005420EF00837F2500D0
:10AFE000008041001040BA000160EF000000060040
:10AFF00020520000656C00002053000074610000C6
:10B0000074650000206F00006620000043680000A7
:10B0100061720000676500003A20000025640000AE
:10B02000252500000D0A0000000000005420EF005C
:10B0300023822500008041001040BA000160EF002B
:10B0400000000600467500006C6C00002043000004
:10B050006861000072670000652000004361000025
:10B060007061000063690000747900003A200000FC
:10B07000256400000D0A0000000000005420EF00CD
:10B08000A3842500008041001040BA000160EF0059
:10B0900000000600202000002020000020200000EA
:10B0A0002020000020200000204D000061780000DA
:10B0B00020450000727200006F7200003A2000000C
:10B0C00025640000252500000D0A00000000000096
:10B0D0005420EF0043872500008041001040BA0053
:10B0E0000160EF0000000600202000002052000058
:10B0F000756E000020540000696D0000652000009E
:10B10000546F0000204500006D700000747900004D
:10B110003A200000000000005420EF008389250041
:10B12000008041001040BA000160EF0000000600FE
:10B130004368000061720000676900006E670000EC
:10B140000D0A0000000000005420EF00038B2500D2
:10B15000008041001040BA000160EF0000000600CE
:10B1600020200000202000002020000020200000DF
:10B1700020430000796300006C650000204300005C
:10B180006F7500006E7400003A2000002564000016
:10B190000D0A0000000000005420EF00838D250000
:10B1A000008041001040BA000160EF00000006007E
:10B1B000202000002020000020200000202000008F
:10B1C00020420000617400007420000053740000ED
:10B1D00061740000757300003A20000030780000B0
:10B1E00025340000780D00000A0000005420EF0014
:10B1F00023902500008041001040BA000160EF005C
:10B200000000060020200000202000002020000078
:10B210002020000020540000656D000070650000D3
:10B220007261000074750000726500003A20000031
:10B23000253300002E310000660D00000A000000DA
:10B240005420EF00C3922500008041001040BA0056
:10B250000160EF00000006002020000043680000AD
:10B2600061720000676500002054000065720000F4
:10B270006D6900006E610000746900006F6E00006F
:10B280003A200000256400002C20000030780000E7
:10B2900025340000780D00000A0000005420EF0063
:10B2A000A3952500008041001040BA000160EF0026
:10B2B00000000600202000002020000020200000C8
:10B2C0002020000020200000436800006754000098
:10B2D000696D000065430000747200003A200000B0
:10B2E000256400003A250000643A0000256400004F
:10B2F0000D0A0000000000005420EF008398250094
:10B30000008041001040BA000160EF00000006001C
:10B3100020200000202000002020000054680000B1
:10B32000697300004368000067540000696D000005
:10B33000654300006E7400003A20000025640000A0
:10B340003A250000643A0000256400000D0A000060
:10B35000000000005420EF00639B250000804100A6
:10B360001040BA000160EF0000000600202000003D
:10B3700020200000202000002020000020200000CD
:10B380002020000020200000202000005469000040
:10B390006D6500003A200000256400003A25000099
:10B3A000643A0000256400000D0A0000000000005F
:10B3B0005420EF00439E2500008041001040BA0059
:10B3C0000160EF00000006002020000020200000A7
:10B3D00020200000202000004C6900006E65000065
:10B3E0006172000043680000674E0000647800004E
:10B3F0003A200000256400000D0A00000000000053
:10B400005420EF00C3A02500008041001040BA0086
:10B410000160EF00000006002A2A00002A20000038
:10B42000577200006974000065200000457200003A
:10B43000726F0000722000002A2A00002A0D00000E
:10B440000A0000005420EF00E3A225000080410024
:10B450001040BA000160EF000000060057720000C3
:10B4600069740000652000004F4B00000D0A0000C9
:10B47000000000005420EF0063A42500008041007C
:10B480001040BA000160EF00000006002A2A000008
:10B490002A2000005772000069740000696E0000E5
:10B4A00067200000426100007474000065720000B3
:10B4B0007920000044610000746500003A2000001B
:10B4C000256400002F250000642F00002564000083
:10B4D0000D0A0000000000005420EF0083A72500A3
:10B4E000008041001040BA000160EF00000006003B
:10B4F0002A2A00002A200000426100007474000023
:10B50000657200007920000043680000617200004D
:10B510006765000020530000796E00006320000082
:10B5200046430000432000002D3E00002052000052
:10B530004D2E00002E2E00002E2E00000D0A0000C1
:10B54000000000005420EF00E3AA25000080410025
:10B550001040BA000160EF00000006002A2A000037
:10B560002A20000052650000677500006C61000031
:10B57000746F000072790000204400006F6D0000BD
:10B58000616900006E3A000020460000434300005D
:10B590002028000055530000412900000D0A00003A
:10B5A000000000005420EF00E3AD250000804100C2
:10B5B0001040BA000160EF00000006002A2A0000D7
:10B5C0002A20000052650000677500006C610000D1
:10B5D000746F000072790000204400006F6D00005D
:10B5E000616900006E3A00002045000054530000DD
:10B5F0004920000028450000552900000D0A0000E0
:10B60000000000005420EF00E3B02500008041005E
:10B610001040BA000160EF00000006002A2A000076
:10B620002A20000052650000677500006C61000070
:10B63000746F000072790000204400006F6D0000FC
:10B64000616900006E3A000020540000454C000083
:10B6500045430000202800004A610000706100009E
:10B660006E2900000D0A0000000000005420EF00C9
:10B6700083022000830150000500310023B525001E
:10B68000008041001040BA000160EF000000060099
:10B6900020B5250083814100808141001380BA00DC
:10B6A000000006002A2A6F002A206600556E20003E
:10B6B00072657400636F6800676E6500697A2000C8
:10B6C0006564660020656F006E746C0072796C00B2
:10B6D0002E206F004D7577007374690020636E0033
:10B6E000686F67006F733A0065200D006F6E0A0087
:10B6F000652000005420EF0063B825000080410061
:10B700001040BA000160EF00000006003020000089
:10B710002D20000046430000432000002855000073
:10B7200053410000290D00000A0000005420EF00E2
:10B7300023BA2500008041001040BA000160EF00EC
:10B7400000000600312000002D20000045540000BC
:10B75000534900002028000045550000290D000035
:10B760000A0000005420EF00E3BB250000804100E8
:10B770001040BA000160EF00000006003220000017
:10B780002D200000544500004C45000043200000DF
:10B79000284A000061700000616E0000290D000061
:10B7A0000A0000005420EF006302200083015000D3
:10B7B00005003100E3BE2500008041001040BA00C2
:10B7C0000160EF0000000600E0BE2500838141001B
:10B7D000808141001380BA00000006002A2A6C0014
:10B7E0002A20740052652000677574006C616F0038
:10B7F000746F200072794600204443006F6D43004F
:10B80000616920006E3A2800204E55004F545300C5
:10B810002053410045542900202D0D0020640A00CA
:10B8200065660000617500005420EF0003C225002A
:10B83000008041001040BA000160EF0000000600E7
:10B840002A2A00002A200000556E000072650000C0
:10B85000636F0000676E0000697A00006564000095
:10B860002052000065670000756C000061740000E4
:10B870006F72000079200000446F00006D610000CD
:10B88000696E00002E0D00000A0000005420EF0039
:10B8900063022000830150000500310023C625000B
:10B8A000008041001040BA000160EF000000060077
:10B8B00020C6250083814100808141001380BA00A9
:10B8C00000000600546F20002073630065746F0051
:10B8D00020746D0068656D002052610065676E0020
:10B8E000756C6400617420006F725300792045000C
:10B8F000446F54006D612000696E5200206945005C
:10B900007373470075650D0020740A0068650000B8
:10B910005420EF0043C92500008041001040BA00C8
:10B920000160EF0000000600616E0000642000006E
:10B93000656E000074650000722000006F6E0000EC
:10B94000652000006F66000020740000686500003C
:10B95000206600006F6C00006C6F000077690000CB
:10B960006E6700003A0D00000A0000005420EF004E
:10B9700023CC2500008041001040BA000160EF0098
:10B980000000060030200000666F000072200000FA
:10B9900046430000432000002855000053410000AA
:10B9A000290D00000A0000005420EF0003CE2500FE
:10B9B000008041001040BA000160EF000000060066
:10B9C00031200000666F0000722000004554000026
:10B9D000534900002028000045550000290D0000B3
:10B9E0000A0000005420EF00E3CF25000080410052
:10B9F0001040BA000160EF00000006003220000095
:10BA0000666F000072200000544500004C450000A5
:10BA100043200000284A000061700000616E0000B1
:10BA2000290D00000A0000005420EF00030220004E
:10BA3000830150000500310003D325000080410040
:10BA40001040BA000160EF000000060000D325009E
:10BA500083814100808141001380BA00000006000C
:10BA60005468320065203000576920004669630041
:10BA70002053680053496100442072006D756100D5
:10BA80007374630020627400652065006C65720049
:10BA90007373730020740D0068610A006E2000004B
:10BAA0005420EF00C3D52500008041001040BA00AB
:10BAB0000160EF00000006000D0A0000546800005D
:10BAC000652000006E6500007720000053530000E1
:10BAD0004944000020690000733A0000202500005E
:10BAE000730D00000A0000005420EF0003D8250069
:10BAF000008041001040BA000160EF000000060025
:10BB00002A2A00002A200000576900004669000028
:10BB100020500000726F000067650000616D00003A
:10BB2000204D00006F640000652000004F460000BB
:10BB3000460D00000A0000005420EF0083DA2500C3
:10BB4000008041001040BA000160EF0000000600D4
:10BB50002A2A00002A2000005769000046690000D8
:10BB600020500000726F000067720000616D0000DD
:10BB7000204D00006F640000652000004F4E000063
:10BB80000D0A0000000000005420EF0003DD250036
:10BB9000008041001040BA000160EF000000060084
:10BBA0002A2A00002A200000576100006974000062
:10BBB000696E000067200000666F000072200000C0
:10BBC000706F00007765000072200000746F000045
:10BBD0002073000074610000626900006C6900005D
:10BBE0007A6500002E2E00002E0D00000A000000D5
:10BBF0005420EF0043E02500008041001040BA00CF
:10BC00000160EF00000006002A2A00002A20000040
:10BC10005769000046690000204100006C72000076
:10BC20006561000064790000204F00006E0D000087
:10BC30000A0000005420EF0063E22500008041006C
:10BC40001040BA000160EF00000006002A2A000040
:10BC50002A200000436F00006E7300006F6C00002C
:10BC600065200000436F00006E6E000065630000F9
:10BC70007465000064200000746F0000205700000D
:10BC800069460000692000004D6F000064750000E7
:10BC90006C6500000D0A0000000000005420EF0059
:10BCA000A3E52500008041001040BA000160EF00CC
:10BCB000000006002A2A00002A2000004D43000050
:10BCC00020520000657600000D0A00000000000010
:10BCD0005420EF0043E72500008041001040BA00E7
:10BCE0000160EF0000000600204D0000432000002E
:10BCF00052650000762000002D20000052650000F3
:10BD000076480000693A00002575000020520000C6
:10BD1000657600004C6F00003A250000750D0000AC
:10BD20000A0000005420EF00E3E9250000804100F4
:10BD30001040BA000160EF00000006002A2A00004F
:10BD40002A200000536500007420000041630000B9
:10BD5000712000004D6F000064650000204E00005F
:10BD6000656F0000204F00006E0D00000A0000000B
:10BD70005420EF0043EC2500008041001040BA0041
:10BD80000160EF00000006002A2A00002A200000BF
:10BD9000544300002053000065740000205300004D
:10BDA0004E41000050200000506F000077650000F9
:10BDB000722000004F6E0000206F00006E20000017
:10BDC000706F000077650000722000007570000041
:10BDD0000D0A0000000000005420EF0083EF250052
:10BDE000008041001040BA000160EF000000060032
:10BDF0002A2A00002A20000054430000205300009B
:10BE000065740000205300004E41000050200000E7
:10BE1000506F000077650000722000004F66000040
:10BE2000662000006F6E0000207000006F77000039
:10BE30006572000020750000700D00000A0000000F
:10BE40005420EF00C3F22500008041001040BA00EA
:10BE50000160EF00000006002A2A00002A200000EE
:10BE6000434800004B2000004145000052520000B2
:10BE70000D0A0000000000005420EF0083F42500AC
:10BE8000008041001040BA000160EF000000060091
:10BE90002041000045520000527300003A25000086
:10BEA000640D00000A0000005420EF0003F6250096
:10BEB000008041001040BA000160EF000000060061
:10BEC0002A2A00002A2000004745000054200000D4
:10BED0004145000052520000203000000D0A0000D1
:10BEE000000000005420EF00E3F72500008041002F
:10BEF0001040BA000160EF00000006002A2A00008E
:10BF00002A20000047450000542000004145000061
:10BF100052520000204100004C4C00000D0A00006D
:10BF2000000000005420EF00E3F9250000804100EC
:10BF30001040BA000160EF00000006002A2A00004D
:10BF40002A20000047450000542000004145000021
:10BF5000525200000D0A0000000000005420EF00C3
:10BF6000A3FB2500008041001040BA000160EF00F3
:10BF7000000006002A2A00002A2000005245000086
:10BF8000534500005420000041450000525200007B
:10BF90002047000045540000204E00004458000097
:10BFA0000D0A0000000000005420EF0003FE2500F1
:10BFB000008041001040BA000160EF000000060060
:10BFC0002A2A00002A2000005245000053450000A4
:10BFD0005420000041450000525200000D0A0000AC
:10BFE000000000005420EF00E3FF25000080410026
:10BFF0001040BA000160EF00000006002A2A00008D
:10C000002A20000052450000534500005420000043
:10C0100041450000525200002053000045540000EA
:10C02000204E0000445800000D0A000000000000EF
:10C030005420EF0043022600008041001040BA0067
:10C040000160EF00000006002A2A00002A200000FC
:10C0500053450000542000004145000052520000AA
:10C060002047000045540000204E000044580000C6
:10C070003A200000254400000D0A000000000000E6
:10C080005420EF00C3042600008041001040BA0095
:10C090000160EF00000006002A2A00002A200000AC
:10C0A00050500000532000005465000073740000DD
:10C0B000204F00006E0D00000A0000005420EF0029
:10C0C000A3062600008041001040BA000160EF0086
:10C0D000000006002A2A00002A20000048750000FF
:10C0E000646400006C65000020540000657300006B
:10C0F000742000004F6E00000D0A000000000000D8
:10C100005420EF00C3082600008041001040BA0010
:10C110000160EF00000006002A2A00002A2000002B
:10C1200048750000646400006C6500002054000045
:10C1300065730000742000004F460000460D0000AB
:10C140000A0000005420EF00430220008301500049
:10C1500005003100E30B2600008041001040BA00CA
:10C160000160EF0000000600E00B26008381410023
:10C17000808141001380BA00000006002A2A6F0067
:10C180002A206400537465006F702000204E7400F4
:10C19000656F6F0020723A00656320006F724E0079
:10C1A000646965006E676F00206120006E644F0057
:10C1B000207366006574660020410D0063710A00FB
:10C1C000204D00005420EF00E30E260000804100C7
:10C1D0001040BA000160EF00000006002A2A0000AB
:10C1E0002A200000417400006F6D00002033000021
:10C1F0004320000053740000617400007573000058
:10C20000202A00002A2A00000D0A00000000000079
:10C210005420EF0043112600008041001040BA0076
:10C220000160EF0000000600576100006B65000030
:10C2300052650000617300006F6E00005B2000001B
:10C2400025750000205D00000D0A000000000000C0
:10C250005420EF0043132600008041001040BA0034
:10C260000160EF00000006002A2A00002A200000DA
:10C270005465000073740000204C00004544000029
:10C28000732000006F660000660D00000A000000C9
:10C290005420EF0043152600008041001040BA00F2
:10C2A0000160EF00000006002A2A00002A2000009A
:10C2B0005465000073740000204C000045440000E9
:10C2C000732000006F6E00000D0A000000000000E7
:10C2D0005420EF0043172600008041001040BA00B0
:10C2E0000160EF00000006002A2A00002A2000005A
:10C2F0004C45000044730000206F0000666600009B
:10C300000D0A0000000000005420EF000319260071
:10C31000008041001040BA000160EF0000000600FC
:10C320002A2A00002A2000005465000073740000CF
:10C3300020420000757A00007A650000722000003B
:10C340006F660000660D00000A0000005420EF0038
:10C35000231B2600008041001040BA000160EF005E
:10C36000000006002A2A00002A2000005465000070
:10C370007374000020420000757A00007A650000A6
:10C38000722000006F6E00000D0A00000000000027
:10C390005420EF00431D2600008041001040BA00E9
:10C3A0000160EF00000006002A2A00002A20000099
:10C3B00053650000742000006445000042550000F1
:10C3C00047200000466C00006167000073200000F9
:10C3D00025320000780D00000A0000005420EF0014
:10C3E000A31F2600008041001040BA000160EF004A
:10C3F000000006002A2A00002A200000466F0000E4
:10C40000726D000061740000746900006E670000C6
:10C41000202A00002A2A00000D0A00000000000067
:10C420005420EF00C3212600008041001040BA00D4
:10C430000160EF0000000600466F0000726D000012
:10C440006174000020450000727200006F720000ED
:10C450000D0A0000000000005420EF008323260096
:10C46000008041001040BA000160EF0000000600AB
:10C470002051000075690000636B00002046000039
:10C480006F7200006D61000074200000666900009A
:10C490006E69000073680000656400000D0A00000A
:10C4A000000000005420EF00E3252600008041003A
:10C4B0001040BA000160EF00000006002A2A0000C8
:10C4C00020450000525200004F520000202D000075
:10C4D0002072000065740000757200006E65000037
:10C4E0006420000065720000726F0000722000007E
:10C4F000636F00006465000020250000750D0000DA
:10C500000A0000005420EF00E328260000804100CC
:10C510001040BA000160EF0000000600496E000004
:10C52000636F00006D7000006C65000074650000B2
:10C53000206300006F6D00006D6100006E640000FC
:10C540000D0A0000000000005420EF00E30120006D
:10C550008301500005003100032C260000804100BB
:10C560001040BA000160EF0000000600002C260019
:10C5700083814100808141001380BA0000000600E1
:10C580002A2A720020456F00525272004F5220003A
:10C59000202D630020456F00585064004C4F65000B
:10C5A00052452000207225006574750075720D00DB
:10C5B0006E650A0064200000657200005420EF00E0
:10C5C000A32E2600008041001040BA000160EF0059
:10C5D0000000060054590000504500002063000090
:10C5E0006F6D00006D6100006E6400000D0A0000B8
:10C5F000000000005420EF0063302600008041005E
:10C600001040BA000160EF0000000600486500001D
:10C610007861000064650000636900006D610000DE
:10C620006C200000666900006C650000206400005A
:10C63000756D000070200000636F00006D6D0000DC
:10C64000616E0000640D00000A0000005420EF003D
:10C6500023332600008041001040BA000160EF0043
:10C660000000060052450000534500005420000021
:10C670004D430000206300006F6D00006D610000FD
:10C680006E6400000D0A0000000000005420EF005E
:10C6900023352600008041001040BA000160EF0001
:10C6A0000000060053440000204900004E490000ED
:10C6B00054200000636F00006D6D0000616E00008B
:10C6C000640D00000A0000005420EF00033726002C
:10C6D000008041001040BA000160EF000000060039
:10C6E0004E65000077410000726E0000316D000061
:10C6F000734600006C610000672000005B4F000083
:10C700004E5D00000D0A0000000000005420EF0004
:10C7100023392600008041001040BA000160EF007C
:10C72000000006004E65000077410000726E0000B8
:10C73000316D0000734600006C610000672000004E
:10C740005B4F0000464600005D0D00000A0000003F
:10C750005420EF00433B2600008041001040BA0007
:10C760000160EF0000000600436F00006D6D0000E7
:10C77000616E000064200000556E00006B6E0000CA
:10C780006F7700006E2000002D3E00002573000032
:10C790003C2D00000D0A0000000000005420EF00B6
:10C7A000A33D2600008041001040BA000160EF0068
:10C7B0000000060045780000697400002057000062
:10C7C0006946000069200000636F00006E7300007E
:10C7D0006F6C0000652000006D6F00006465000054
:10C7E0000D0A0000000000005420EF000340260066
:10C7F000008041001040BA000160EF000000060018
:10C80000434D0000443E0000000000005420EF00B3
:10C81000030220008301500005003100234226005E
:10C82000008041001040BA000160EF0000000600E7
:10C830002042260083814100808141001380BA009C
:10C84000000006000D0A7300537469006F706700E2
:10C8500020776E0061696D00746965006E676E0017
:10C86000206674006F720D0020490A0050205700A6
:10C8700041646900647246006573690073203E007C
:10C88000617300005420EF00E34426000080410063
:10C890001040BA000160EF00000006000D0A000021
:10C8A0005769000046690000204F000066660000DE
:10C8B0000D0A0000434D0000443E0000000000004F
:10C8C0005420EF00C3462600008041001040BA000B
:10C8D0000160EF00000006000D0A00005265000034
:10C8E0007374000061720000746900006E670000DC
:10C8F0002057000069460000690D00000A5700003B
:10C9000069460000693E0000000000005420EF006E
:10C9100023492600008041001040BA000160EF006A
:10C92000000006000D0A00005749000046490000BB
:10C930003E0000005420EF00634A260000804100C2
:10C940001040BA000160EF000000060057490000E7
:10C95000464900003E0000005420EF00A3022000E2
:10C960008301500005003100834C26000080410007
:10C970001040BA000160EF0000000600804C260065
:10C9800083814100808141001380BA0000000600CD
:10C990002A2A20002A2A3F0020412C00746F200000
:10C9A0006D203F0033433F002076200025646F0058
:10C9B0002E257200642020002A2A3F002A2A3F00E8
:10C9C0000D0A3F000D0A0D00466F0A007220430059
:10C9D00068654D006C7044002C203E0074790000A6
:10C9E000706500005420EF00E34F260000804100F6
:10C9F0001040BA000160EF00000006003D3D00005D
:10CA00003D3D00003D3D00003D3D00003D3D00003E
:10CA10003D3D00003D3D00003D3D00003D3D00002E
:10CA20003D3D00003D3D00000D0A000000000000FB
:10CA30005420EF0043522600008041001040BA000D
:10CA40000160EF0000000600202000002020000010
:10CA500020200000546900006D6500003A200000AD
:10CA6000256400003A250000643A000025640000B7
:10CA70000D0A0000000000005420EF00835426003F
:10CA8000008041001040BA000160EF000000060085
:10CA90002020000020200000202000004461000031
:10CAA000746500003A200000256400002F25000076
:10CAB000642F0000256400000D0A00000000000043
:10CAC0005420EF00C3562600008041001040BA00F9
:10CAD0000160EF0000000600202000004C61000013
:10CAE0007469000074750000646500003A2000005D
:10CAF0002573000020250000630D00000A000000DF
:10CB00005420EF00C3582600008041001040BA00B6
:10CB10000160EF0000000600204C00006F6E000076
:10CB20006769000074750000646500003A20000029
:10CB30002573000020250000630D00000A0000009E
:10CB40005420EF00C35A2600008041001040BA0074
:10CB50000160EF00000006002020000020200000FF
:10CB600020200000484400004F5000003A20000000
:10CB7000253100002E310000660D00000A00000083
:10CB80005420EF00C35C2600008041001040BA0032
:10CB90000160EF000000060020200000416C000052
:10CBA0007469000074750000646500003A2000009C
:10CBB000253400002E310000660D00000A00000040
:10CBC0005420EF00C35E2600008041001040BA00F0
:10CBD0000160EF0000000600536100007465000072
:10CBE0006C6C000069740000657300003A2000005E
:10CBF000256400000D0A0000000000005420EF0032
:10CC0000A3602600008041001040BA000160EF00E0
:10CC1000000006002020000020200000202000004E
:10CC200020460000697800003A20000025640000DA
:10CC30000D0A0000000000005420EF00836226006F
:10CC4000008041001040BA000160EF0000000600C3
:10CC50002047000050530000204D00007367000083
:10CC60003A200000000000005420EF00036426007A
:10CC7000008041001040BA000160EF000000060093
:10CC800020200000202000002020000020200000A4
:10CC90002020000020200000202000002020000094
:10CCA0002020000020200000202000002020000084
:10CCB0002020000020200000202000002020000074
:10CCC000202000000D0000005420EF000367260024
:10CCD000008041001040BA000160EF000000060033
:10CCE0003D3D00003D3D00003D3D00003D3D00005C
:10CCF0003D3D00003D3D00003D3D00003D3D00004C
:10CD00003D3D00003D3D00003D3D00003D3D00003B
:10CD10003D3D00000D0A0000000000005420EF001F
:10CD2000A3692600008041001040BA000160EF00B6
:10CD30000000060020200000505000005354000066
:10CD4000696D0000654500007272000041630000DB
:10CD5000637500006D3A0000202500006C6400003F
:10CD60000D0A0000000000005420EF00036C2600B4
:10CD7000008041001040BA000160EF000000060092
:10CD80002020000020200000202000005050000043
:10CD900053540000696D0000657200004572000088
:10CDA000723A0000202500006C6400000D0A0000AB
:10CDB000000000005420EF00636E26000080410058
:10CDC0001040BA000160EF000000060020200000C3
:10CDD0002020000020200000202000002020000053
:10CDE000564300004F200000416400006A3A0000F2
:10CDF000202500006C640000200D00000A000000E7
:10CE00005420EF00C3702600008041001040BA009B
:10CE10000160EF000000060020200000202000003C
:10CE20002020000020560000434F00002043000057
:10CE3000686100006E670000653A00002025000070
:10CE4000640D00000A0000005420EF000373260068
:10CE5000008041001040BA000160EF0000000600B1
:10CE600020200000202000002020000020200000C2
:10CE700020200000564300004F20000044410000E5
:10CE8000433A0000202500006C6400000D0A0000F9
:10CE9000000000005420EF00637526000080410070
:10CEA0001040BA000160EF000000060020200000E2
:10CEB00020200000564300004F200000496E000073
:10CEC000746500006772000061740000653A00003C
:10CED000202500006C6400000D0A00000000000026
:10CEE0005420EF00C3772600008041001040BA00B4
:10CEF0000160EF0000000600202D0000202D000042
:10CF0000202D0000202D0000202D0000202D0000ED
:10CF1000202D0000202D0000202D0000202D0000DD
:10CF2000202D0000202D0000202D00000D0A000003
:10CF3000000000005420EF00637A260000804100CA
:10CF40001040BA000160EF00000006002020000041
:10CF500020200000202000002020000020200000D1
:10CF6000202000002020000041440000433A00003F
:10CF700020250000640D00000A0000005420EF008E
:10CF8000A37C2600008041001040BA000160EF0041
:10CF900000000600202000002020000020200000CB
:10CFA000202000004144000043460000696C00005E
:10CFB00074650000723A0000202500006C640000D7
:10CFC0000D0A0000000000005420EF00037F26003F
:10CFD000008041001040BA000160EF000000060030
:10CFE0002020000020200000202000002020000041
:10CFF000414400004345000072720000416400009B
:10D000006A3A0000202500006C6400000D0A000050
:10D01000000000005420EF006381260000804100E2
:10D020001040BA000160EF0000000600444100001B
:10D0300043460000696C000074650000722D00001A
:10D04000564300004F5F000044410000433A000097
:10D05000202500006C6400000D0A000000000000A4
:10D060005420EF00C3832600008041001040BA0026
:10D070000160EF00000006002020000020200000DA
:10D080002020000020440000414300005F460000D3
:10D09000696C000074650000723A000020250000F1
:10D0A0006C6400000D0A0000000000005420EF0036
:10D0B00023862600008041001040BA000160EF0086
:10D0C000000006002020000020200000202000009A
:10D0D000202000002020000054430000466C000087
:10D0E00061670000733A000020250000780D000001
:10D0F0000A0000005420EF006388260000804100F1
:10D100001040BA000160EF0000000600202000007F
:10D110002020000020200000505000005345000057
:10D12000766500006E740000436E0000743A0000E3
:10D1300020250000750D00000A0000005420EF00BB
:10D14000A38A2600008041001040BA000160EF0071
:10D15000000006002050000050530000564300001D
:10D160004F53000065740000746C0000656400009B
:10D1700043740000723A000020250000750D000085
:10D180000A0000005420EF00E38C260000804100DC
:10D190001040BA000160EF000000060020200000EF
:10D1A00020200000204C00006F630000616C000034
:10D1B0005F5000005053000043740000723A0000BA
:10D1C000202500006C7500000D0A00000000000022
:10D1D0005420EF00438F2600008041001040BA0029
:10D1E0000160EF0000000600202000002020000069
:10D1F0002020000020470000505300005F50000036
:10D200005053000043740000723A000020250000D3
:10D210006C7500000D0A0000000000005420EF00B3
:10D22000A3912600008041001040BA000160EF0089
:10D230000000060020200000202000002020000028
:10D240004C6F0000737400004C6F0000636B0000B3
:10D2500043740000723A000020250000750D0000A4
:10D260000D0A0000000000005420EF000394260087
:10D27000008041001040BA000160EF00000006008D
:10D280002020000020410000444300005F4C0000CB
:10D29000544100005F450000766500006E74000098
:10D2A000733A000020250000750D00000A00000000
:10D2B0005420EF0043962600008041001040BA0041
:10D2C0000160EF0000000600202000002020000088
:10D2D000202000002020000020200000202000004E
:10D2E00020540000696D0000653A00002025000010
:10D2F000643A0000256400003A250000640D000037
:10D300000A0000005420EF00E3982600008041004E
:10D310001040BA000160EF0000000600205000003D
:10D320005053000045760000656E00007443000015
:10D33000747200003A2000002575000020200000D3
:10D34000205000005053000045760000656E00003C
:10D35000744300006E7400003A2000002575000040
:10D360000D0000005420EF00E39B260000804100E8
:10D370001040BA000160EF00000006002A2A0000F9
:10D380002A2A00002A2A00002A2000004750000014
:10D3900053200000556E00006C6F0000636B0000AE
:10D3A000656400002025000075200000202000009A
:10D3B0002A2A00002A2A00002A2A00002A2A00001D
:10D3C0002A2A00000D0000005420EF00039F2600D1
:10D3D000008041001040BA000160EF00000006002C
:10D3E0000D0A00002A2A00002A200000412F000018
:10D3F00044200000537900006E63000027640000A1
:10D400003A250000750D00000A0000005420EF00CE
:10D4100023A12600008041001040BA000160EF0007
:10D420000000060045520000524F0000523A000032
:10D4300020540000757200006E2000005769000043
:10D4400046690000204F00006E2000004669000081
:10D4500072730000740D00000A0000005420EF00F9
:10D46000A3A32600008041001040BA000160EF0035
:10D47000000006002A2A00002A200000416E000059
:10D48000616C00006F670000204F00006E0D00000F
:10D490000A0000005420EF0063A526000080410030
:10D4A0001040BA000160EF00000006002A2A0000C8
:10D4B0002A200000416E0000616C00006F670000D0
:10D4C000204F0000666600000D0A0000000000000A
:10D4D0005420EF0043A72600008041001040BA000E
:10D4E0000160EF00000006003D3D00003D3D0000F2
:10D4F0003D200000436D0000645400004F0D00000B
:10D500000A0000005420EF00E3A82600008041003C
:10D510001040BA000160EF000000060061740000D6
:10D520002B6E000064680000637000003D31000055
:10D53000000000005420EF0063AA26000080410094
:10D540001040BA000160EF000000060041540000E6
:10D550002B4E000053550000445000003D250000B4
:10D5600034750000000000005420EF0003AC2600DA
:10D57000008041001040BA000160EF00000006008A
:10D5800063720000656100007465000064200000A3
:10D590003C550000445000005265000073650000D7
:10D5A000745300006F6300006B650000743E000060
:10D5B0000D0A0000000000005420EF0083AE26009A
:10D5C000008041001040BA000160EF00000006003A
:10D5D000415400002B4E0000435400004350000013
:10D5E0003D250000732C000025340000750000006C
:10D5F0005420EF0043B02600008041001040BA00E4
:10D600000160EF0000000600456E0000642000008D
:10D610006F66000020730000656E00006469000002
:10D620006E6700002064000061740000612000004B
:10D63000330D00000A0000005420EF0083B22600E2
:10D64000008041001040BA000160EF0000000600B9
:10D650003D3D00003D3D00003D3D000020640000D8
:10D660006F4100006E6100006C6F0000674F0000AA
:10D67000666600000D0A0000000000005420EF0064
:10D68000A3B42600008041001040BA000160EF0002
:10D69000000006003D3D00003D3D00003D3D000016
:10D6A0002044000052440000590D00000A00000010
:10D6B0005420EF0043022000830150000500310098
:10D6C00043B72600008041001040BA000160EF001F
:10D6D0000000060040B726008381410080814100A0
:10D6E0001380BA0000000600575F650049447300CC
:10D6F0004C4565003A537400696E2000655445003E
:10D7000065735200744652006C674F00206F5200E0
:10D710006E2E21002E2E210020532100616D2E003F
:10D72000706C0D0065430A00747200002052000006
:10D730005420EF0043BA2600008041001040BA0098
:10D740000160EF0000000600576900004669000014
:10D7500052780000536900007A6500003A25000005
:10D76000750D00000A0000005420EF0003BC2600E5
:10D77000008041001040BA000160EF000000060088
:10D7800057490000464900005F5200004541000033
:10D79000444900004E470000204400004F4E000066
:10D7A000452000000D0A0000000000005420EF009A
:10D7B00023BE2600008041001040BA000160EF0047
:10D7C000000006005544000050200000434D0000BA
:10D7D000445B000025430000254300005D0D000070
:10D7E0000A0000005420EF00E3BF26000080410043
:10D7F0001040BA000160EF00000006005544000030
:10D8000050200000545800000D0A000000000000E5
:10D810005420EF0043C12600008041001040BA00B0
:10D820000160EF0000000600415400002B4E000094
:10D83000434C00004F530000453D000025310000DF
:10D84000780D00000A0000005420EF0003C32600FA
:10D85000008041001040BA000160EF0000000600A7
:10D860004E6500006F2000005374000061720000DC
:10D87000740D00000A0000005420EF0083C426004D
:10D88000008041001040BA000160EF000000060077
:10D890005443000050200000434D0000445B000052
:10D8A00025430000254300005D0D00000A00000034
:10D8B0005420EF0043C62600008041001040BA000B
:10D8C0000160EF00000006005443000050200000FB
:10D8D000436D0000643D0000303000000D0A000080
:10D8E000000000005420EF00E3C726000080410044
:10D8F0001040BA000160EF0000000600475300002E
:10D90000505F000052780000537400006174000002
:10D910002825000064290000213D00004753000035
:10D92000505F0000525300004C5400005F4F000055
:10D930004B0D00000A0000005420EF0083CA2600AF
:10D94000008041001040BA000160EF0000000600B6
:10D95000447500006D70000062200000436F0000FD
:10D960006D6D0000616E00006420000045520000F3
:10D97000524F000052200000330D00000A0000004A
:10D980005420EF00C3CC2600008041001040BA00B4
:10D990000160EF0000000600447500006D7000009B
:10D9A00062200000436F00006D6D0000616E00009A
:10D9B0006420000045520000524F00005220000039
:10D9C000340D00000A0000005420EF0003CF2600B1
:10D9D000008041001040BA000160EF000000060026
:10D9E000534E0000442000004F4B00000D0A000081
:10D9F000000000005420EF0063D0260000804100AA
:10DA00001040BA000160EF00000006002D2D00005C
:10DA1000534500004E440000206500006E64000085
:10DA2000203200006E6400000D0A000000000000BB
:10DA30005420EF0043D22600008041001040BA007D
:10DA40000160EF00000006002D2D0000534500008E
:10DA50004E440000207300007461000072740000E6
:10DA6000203200006E6400000D0A0000000000007B
:10DA70005420EF0043D42600008041001040BA003B
:10DA80000160EF0000000600535300004E44000008
:10DA900020530000656E0000646900006E6700009E
:10DAA00020660000696C00006520000070610000C5
:10DAB000636B0000657400000D0A000000000000A8
:10DAC0005420EF00C3D62600008041001040BA0069
:10DAD0000160EF0000000600446F00006E6500006A
:10DAE0002072000065610000646900006E6700003C
:10DAF00020660000696C0000650D00000A0000004F
:10DB00005420EF00C3D82600008041001040BA0026
:10DB10000160EF000000060046410000494C000093
:10DB200055520000452000003A540000580D0000F6
:10DB30000A0000005420EF0063DA26000080410054
:10DB40001040BA000160EF0000000600636F0000A3
:10DB50006E6E000065630000746900006F6E000067
:10DB60002069000073200000636C00006F730000E8
:10DB7000656400000D0A0000000000005420EF0062
:10DB8000A3DC2600008041001040BA000160EF00D5
:10DB9000000006003C450000534300003E25000005
:10DBA000632800003078000025780000292000005C
:10DBB0002E2E0000203F000065720000726F0000F2
:10DBC000723F00000D0A0000000000005420EF002A
:10DBD00023DF2600008041001040BA000160EF0002
:10DBE000000006005443000050200000536F000066
:10DBF000636B0000657400002825000064290000A4
:10DC0000204E00006F740000206600006F75000059
:10DC10006E6400000D0A0000000000005420EF00B8
:10DC2000230220008301500005003100A3E22600FA
:10DC3000008041001040BA000160EF0000000600C3
:10DC4000A0E2260083814100808141001380BA0058
:10DC5000000006002A2A20002A202500496E7500AF
:10DC600069746D00696141006C6948007A6920003F
:10DC70006E672E0020422E0061742E0074652E0007
:10DC800072792E0020450D0045500A00524F0000C9
:10DC90004D200000746F00005420EF0083E5260043
:10DCA000008041001040BA000160EF000000060053
:10DCB0004261000074740000657200007920000069
:10DCC00045450000505200004F4D00002049000023
:10DCD0006E69000074690000616C0000697A0000E0
:10DCE000656400000D0A0000000000005420EF00F1
:10DCF00063022000830150000500310023E9260063
:10DD0000008041001040BA000160EF0000000600F2
:10DD100020E9260083814100808141001380BA0000
:10DD20000000060042616900747474006572680046
:10DD30007920200045452500505264004F4D2000B9
:10DD400020666500616972006C65720064206F0076
:10DD5000696E72006974730069612E006C690D0050
:10DD60007A610A00746900006F6E0000207700007D
:10DD70005420EF0043EC2600008041001040BA0020
:10DD80000160EF0000000600257300002530000050
:10DD9000327500002E610000746D0000000000006C
:10DDA0005420EF00C3ED2600008041001040BA006F
:10DDB0000160EF000000060046530000204500000F
:10DDC000525200004F520000203100000D0A0000A6
:10DDD000000000005420EF0063EF260000804100A7
:10DDE0001040BA000160EF0000000600437200001E
:10DDF0006561000074650000642000006669000031
:10DE00007273000074200000666900006C650000F9
:10DE10003A25000073200000617400003A250000DC
:10DE200075730000200D00000A0000005420EF0070
:10DE300023F22600008041001040BA000160EF008C
:10DE4000000006004653000020450000525200002A
:10DE50004F520000203200000D0A000000000000B8
:10DE60005420EF00C3F32600008041001040BA00A8
:10DE70000160EF000000060046530000204500004E
:10DE8000525200004F520000203300000D0A0000E3
:10DE9000000000005420EF0063F5260000804100E0
:10DEA0001040BA000160EF00000006004653000079
:10DEB00020450000525200004F5200002034000064
:10DEC0000D0A0000000000005420EF0003F72600B8
:10DED000008041001040BA000160EF000000060021
:10DEE0004653000020450000525200004F520000EF
:10DEF000203500000D0A0000000000005420EF0053
:10DF0000A3F82600008041001040BA000160EF0035
:10DF100000000600437200006561000074650000A7
:10DF200064200000666F00006C64000065720000F1
:10DF30003A200000257300000D0A000000000000D8
:10DF40005420EF00C3FA2600008041001040BA00C0
:10DF50000160EF0000000600415200004E4D00003D
:10DF6000696E000075740000653A0000202500000D
:10DF7000750D00000A0000005420EF0083FC26000D
:10DF8000008041001040BA000160EF000000060070
:10DF90004653000020450000525200004F5200003E
:10DFA000203600000D0A0000000000005420EF00A1
:10DFB00023FE2600008041001040BA000160EF00FF
:10DFC00000000600465300002045000052520000A9
:10DFD0004F520000203700000D0A00000000000032
:10DFE0005420EF00C3FF2600008041001040BA001B
:10DFF0000160EF00000006004653000020450000CD
:10E00000525200004F520000203800000D0A00005C
:10E01000000000005420EF00630127000080410051
:10E020001040BA000160EF000000060043720000DB
:10E0300065610000746500006420000066690000EE
:10E040006C6500003A200000257300000D0A0000F6
:10E05000000000005420EF0063032700008041000F
:10E060001040BA000160EF000000060020410000EF
:10E070006371000053650000636F00006E64000070
:10E080003A250000752C0000204C00006F63000052
:10E090006B3A0000257800002C2000004C6F000037
:10E0A000636B000043740000723A000025750000A5
:10E0B0000D0000005420EF0063062700008041009F
:10E0C0001040BA000160EF00000006004F6600003B
:10E0D000660D00000A0000005420EF0083072700AF
:10E0E000008041001040BA000160EF00000006000F
:10E0F00059650000730D00000A0000005420EF0075
:10E10000A3082700008041001040BA000160EF0022
:10E11000000006004E6F00000D0A00000000000025
:10E120005420EF00C3092700008041001040BA00CE
:10E130000160EF00000006005365000072690000F6
:10E14000616C0000204E0000756D000062650000EB
:10E15000723A000020250000730D00000A00000044
:10E160005420EF00C30B2700008041001040BA008C
:10E170000160EF00000006004261000074740000BE
:10E1800020430000617000006163000069740000BA
:10E19000793A00002025000064250000250D0000CC
:10E1A0000A0000005420EF00E30D2700008041002A
:10E1B0001040BA000160EF0000000600204200009D
:10E1C0006174000074200000566F00006C74000041
:10E1D00061670000653A000020250000640D000022
:10E1E0000A0000005420EF00E30F270000804100E8
:10E1F0001040BA000160EF0000000600204200005D
:10E200006174000074200000437500007272000009
:10E21000656E0000743A000020250000640D0000C7
:10E220000A0000005420EF00E311270000804100A5
:10E230001040BA000160EF00000006003D3D000004
:10E240003D2000004163000071750000697300000B
:10E2500069740000696F00006E2000003D3D000001
:10E260003D3D00000D0A0000000000005420EF00BA
:10E2700023142700008041001040BA000160EF0025
:10E280000000060020200000536100006D700000B7
:10E290006C6500002052000061740000653A0000C7
:10E2A0002025000063250000756D0000730D00003F
:10E2B0000A0000005420EF00631627000080410090
:10E2C0001040BA000160EF000000060020200000AE
:10E2D00050720000656100006D7000002047000072
:10E2E000616900006E3A000020250000756400009E
:10E2F000620D00000A0000005420EF008318270080
:10E30000008041001040BA000160EF0000000600EC
:10E3100020200000202000002020000041520000AA
:10E32000204D00006F640000653A000020000000EE
:10E330005420EF00431A2700008041001040BA002B
:10E340000160EF00000006002020000020200000F7
:10E35000204E0000656F0000206D00006F6400001B
:10E36000653A0000200000005420EF00031C270045
:10E37000008041001040BA000160EF00000006007C
:10E380004F6E0000202D0000200000005420EF0000
:10E39000231D2700008041001040BA000160EF00FB
:10E3A0000000060052650000636F00007264000008
:10E3B000696E000067200000737400006172000045
:10E3C00074650000642000002D200000475000000C
:10E3D000532000006C6F0000636B00006564000058
:10E3E0000D0A0000000000005420EF000320270069
:10E3F000008041001040BA000160EF0000000600FC
:10E4000052650000636F000072640000696E0000D6
:10E4100067200000737400006172000074650000E2
:10E42000642000002D200000475000005320000011
:10E43000554E00004C4F0000434B00004544000087
:10E440000D0A0000000000005420EF000323270005
:10E45000008041001040BA000160EF00000006009B
:10E4600052650000636F000072640000696E000076
:10E47000672000006E6F00007420000073740000BD
:10E480006172000074650000642000002D2000000F
:10E4900047500000532000006C6F0000636B0000C9
:10E4A000656400000D0A0000000000005420EF0029
:10E4B00023262700008041001040BA000160EF00D1
:10E4C0000000060052650000636F000072640000E7
:10E4D000696E0000672000006E6F0000742000006D
:10E4E0007374000061720000746500006420000015
:10E4F0002D2000004750000053200000554E000022
:10E500004C4F0000434B0000454400000D0A000042
:10E51000000000005420EF0023022000830150007F
:10E5200005003100632A2700008041001040BA0036
:10E530000160EF0000000600602A2700838141008F
:10E54000808141001380BA0000000600456E6E0015
:10E55000616267006C652000642066002D207200F7
:10E5600042756F0074206D00737420006F7073002B
:10E5700070656C006420650077686500696C7000E8
:10E5800065200D0063680A00617200006769000081
:10E590005420EF00432D2700008041001040BA00B6
:10E5A0000160EF0000000600456E0000616200009F
:10E5B0006C650000642000002D2000004275000002
:10E5C00074200000737400006F700000706500001C
:10E5D000640D00000A0000005420EF00832F270084
:10E5E000008041001040BA000160EF00000006000A
:10E5F0003D3D00003D3D00003D3D00003D20000050
:10E600005769000046690000203D00003D3D0000C4
:10E610003D3D00003D3D00000D0A000000000000EF
:10E620005420EF00C3312700008041001040BA00A1
:10E630000160EF0000000600202000002020000004
:10E640002020000020200000205700006946000024
:10E65000693A0000200000005420EF0083332700B7
:10E66000008041001040BA000160EF000000060089
:10E670005769000046690000206100007420000016
:10E680007374000061720000743A00002000000002
:10E690005420EF0043352700008041001040BA00AD
:10E6A0000160EF00000006002057000069460000EE
:10E6B00069200000546900006D6500006F7500005E
:10E6C000743A0000200000005420EF0003372700B8
:10E6D000008041001040BA000160EF000000060019
:10E6E000257500006D20000028720000656D000097
:10E6F000616900006E6900006E6700003A2000004A
:10E70000257500006D2900000D0A000000000000C2
:10E710005420EF0043392700008041001040BA0028
:10E720000160EF000000060020200000417400009E
:10E730006F6D00002049000050200000416400007F
:10E74000723A0000200000005420EF00033B270035
:10E75000008041001040BA000160EF000000060098
:10E760002D2D00002D0D00000A0000005420EF00A8
:10E77000233C2700008041001040BA000160EF00F8
:10E780000000060020200000202000005043000070
:10E79000204900005020000041640000723A00004F
:10E7A000200000005420EF00E33D270000804100DE
:10E7B0001040BA000160EF000000060020200000B9
:10E7C0002020000020200000202000002053000016
:10E7D00053490000443A000020250000730D00005A
:10E7E0000A0000005420EF00E33F270000804100B2
:10E7F0001040BA000160EF00000006002020000079
:10E8000020200000436F00006E6E00006563000072
:10E8100074650000643A0000200000005420EF00FE
:10E82000A3412700008041001040BA000160EF00C2
:10E830000000060049500000202D00003E2000008E
:10E840005769000046690000204F00006E3A000042
:10E85000200000005420EF006343270000804100A7
:10E860001040BA000160EF0000000600436800009D
:10E8700067200000772F00005769000046690000FC
:10E88000204F00006E3A0000200000005420EF00EE
:10E8900023452700008041001040BA000160EF00CE
:10E8A000000006003D3D00003D3D00003D3D0000F4
:10E8B000205300007461000074650000203D0000DA
:10E8C0003D3D00003D3D00003D3D00000D0A0000C3
:10E8D000000000005420EF00634727000080410043
:10E8E0001040BA000160EF0000000600416E000019
:10E8F000616C00006F6700002073000075700000FD
:10E90000706C0000793A0000200000005420EF00F5
:10E9100023492700008041001040BA000160EF0049
:10E920000000060020200000202000002020000021
:10E93000204200006F7800004E7500006D3A000024
:10E9400020250000750D00000A0000005420EF0093
:10E95000234B2700008041001040BA000160EF0007
:10E96000000006003D3D00003D3D00003D20000050
:10E9700046690000726D000077610000726500005A
:10E98000203D00003D3D00003D3D00000D0A00001F
:10E99000000000005420EF00634D2700008041007C
:10E9A0001040BA000160EF000000060020200000C7
:10E9B00020200000202000004D43000020440000E3
:10E9C00061740000653A000020300000392F00001B
:10E9D000333000002F320000300D00000A0000002C
:10E9E0005420EF00C34F2700008041001040BA00C0
:10E9F0000160EF0000000600202000002020000041
:10EA000020200000204D000043200000526500003F
:10EA1000763A000020250000752E00002530000009
:10EA2000327500000D0A0000000000005420EF00C5
:10EA300023522700008041001040BA000160EF001F
:10EA40000000060020200000202000002020000000
:10EA5000205400004320000052650000763A000078
:10EA600020250000752E00002530000032750000C2
:10EA70000D0A0000000000005420EF00835427001E
:10EA8000008041001040BA000160EF000000060065
:10EA90002020000020200000202000002053000043
:10EAA0004720000052650000763A00002025000053
:10EAB000752E000025300000327500000D0A0000A0
:10EAC000000000005420EF00E356270000804100C2
:10EAD0001040BA000160EF00000006002020000096
:10EAE0002020000020200000205300004E200000C5
:10EAF00052650000763A000020250000752E0000C7
:10EB000025300000327500000D0A000000000000F2
:10EB10005420EF0043592700008041001040BA0004
:10EB20000160EF000000060020200000202000000F
:10EB3000205300004E4100005020000052650000AC
:10EB4000763A0000202D00002D2D00000D0A000057
:10EB5000000000005420EF00635B270000804100AC
:10EB60001040BA000160EF00000006003D3D0000CB
:10EB70003D3D00003D2000004D6500007368000031
:10EB8000204E000065740000203D00003D3D000067
:10EB90003D3D00000D0A0000000000005420EF0081
:10EBA000A35D2700008041001040BA000160EF0023
:10EBB000000006002020000020200000202000008F
:10EBC00020200000205300004E410000503A000079
:10EBD000200000005420EF00635F27000080410008
:10EBE0001040BA000160EF0000000600204D000058
:10EBF00065730000682000004E650000742000006E
:10EC000041640000723A00002025000032780000C4
:10EC10002E250000327800002E25000032780000FA
:10EC2000202800002530000034750000290D000068
:10EC30000A0000005420EF006362270000804100BA
:10EC40001040BA000160EF0000000600204D0000F7
:10EC500065730000682000004E650000742000000D
:10EC600041640000723A0000202D00002D2D0000AC
:10EC70000D0A0000000000005420EF00836427000C
:10EC8000008041001040BA000160EF000000060063
:10EC900020200000202000002020000053630000FE
:10ECA000616E00004E640000783A000020250000EC
:10ECB000750D00000A0000005420EF008366270055
:10ECC000008041001040BA000160EF000000060023
:10ECD000534E0000415000002061000074200000ED
:10ECE0005374000061720000743A00002059000063
:10ECF000657300000D0A0000000000005420EF00C2
:10ED0000A3682700008041001040BA000160EF00B6
:10ED1000000006002020000020200000202000002D
:10ED2000534E00004150000020430000683A0000AC
:10ED300020250000750D00000A0000005420EF009F
:10ED4000A36A2700008041001040BA000160EF0074
:10ED500000000600534E00004150000020610000FA
:10ED6000742000005374000061720000743A0000C7
:10ED7000204E00006F0D00000A0000005420EF003C
:10ED8000A36C2700008041001040BA000160EF0032
:10ED9000000006003D3D00003D3D00003D3D0000FF
:10EDA0003D20000047500000532000003D3D000082
:10EDB0003D3D00003D3D00003D3D00000D0A0000CE
:10EDC000000000005420EF00E36E270000804100A7
:10EDD0001040BA000160EF00000006002020000093
:10EDE0002053000061740000656C00006C69000035
:10EDF00074650000733A00002025000064200000C4
:10EE0000280000005420EF00E3702700008041003C
:10EE10001040BA000160EF00000006004C6F0000D7
:10EE2000636B000065640000290D00000A0000000B
:10EE30005420EF0043722700008041001040BA00C8
:10EE40000160EF0000000600556E00006C6F0000CE
:10EE5000636B000065640000290D00000A000000DB
:10EE60005420EF00C3732700008041001040BA0017
:10EE70000160EF0000000600475000005320000032
:10EE80004F660000662900000D0A00000000000027
:10EE90005420EF0043752700008041001040BA0065
:10EEA0000160EF000000060020200000202000008C
:10EEB000202000002020000020540000696D000088
:10EEC000653A000020250000643A00002564000037
:10EED0003A250000640D00000A0000005420EF00F5
:10EEE000A3772700008041001040BA000160EF00C6
:10EEF00000000600415400002B4E0000434C00006F
:10EF00004F530000453D0000257500000D0A00002C
:10EF1000000000005420EF006379270000804100CA
:10EF20001040BA000160EF00000006002A2A00002D
:10EF30002A2000004E6500006F200000526500008E
:10EF4000636F000072640000696E000067200000BB
:10EF5000546500006D7000006F7200006172000067
:10EF6000696C0000792000004F660000660D00000B
:10EF70000A0000005420EF00637C2700008041005D
:10EF80001040BA000160EF000000060020430000BE
:10EF9000686B000020530000796E0000630D0000D4
:10EFA0000A0000005420EF00E3022000830150001B
:10EFB00005003100E37E2700008041001040BA00C8
:10EFC0000160EF0000000600E07E27008381410021
:10EFD000808141001380BA00000006002323430013
:10EFE00023207400537972006E633A002045250097
:10EFF0007272750020232C00232320002C20530044
:10F000005443610053656D00633A700025756C00D0
:10F01000204165006371500053657400633A7200CB
:10F0200025753A002C20250041537500796E0D009E
:10F0300063430A00686B00005420EF0083822700BE
:10F04000008041001040BA000160EF00000006009F
:10F05000537900006E630000204F00004B20000039
:10F060002D200000536100006D7000006C650000F1
:10F0700050740000723A0000257500000D0A00006F
:10F08000000000005420EF00A30320008301500083
:10F0900005003100E3852700008041001040BA00E0
:10F0A0000160EF0000000600E08527008381410039
:10F0B000808141001380BA00000006002020640017
:10F0C00020572000616B4D00652F6900536C6E0066
:10F0D00065653A00703A25002020640053742000D2
:10F0E000617220007420200044612000793A5200AF
:10F0F0002564650020487000723A6500256461004F
:10F10000204D7400696E3A003A25250064206400A1
:10F110002020200020524400756E610020547900A8
:10F12000696D730065200D0048720A003A250000E1
:10F130005420EF00438A2700008041001040BA00AD
:10F140000160EF000000060046530000204500006B
:10F15000525200004F5200000D0A00000000000053
:10F160005420EF00E303200083015000050031002C
:10F17000C38C2700008041001040BA000160EF00FE
:10F1800000000600C08C270083814100808141007F
:10F190001380BA00000006002041200045525300B1
:10F1A00052735000202D7400204E72006478480085
:10F1B0003A253A0064202500417275006E202C002B
:10F1C0002D202000484853003A255000642C74003C
:10F1D000204D72004D3A4C0025643A002C20250049
:10F1E0004163750071202C002D2020004848450007
:10F1F0003A257200642C7200204D3A004D3A2500E9
:10F20000256475002C200D0053530A003A25000098
:10F21000642C00005420EF0063912700008041001F
:10F220001040BA000160EF00000006002A2A00002A
:10F230002A200000447500006D700000622000006C
:10F24000466900006C650000205200006561000006
:10F250006420000045720000726F00007220000000
:10F26000257500000D0A0000000000005420EF008A
:10F2700023942700008041001040BA000160EF0095
:10F2800000000600417400006F6D00002041000086
:10F290002020000020200000763100002E300000E9
:10F2A000312000004653000020450000525200006B
:10F2B0004F5200003A250000303200007500000077
:10F2C0005420EF00C3962700008041001040BA0090
:10F2D0000160EF0000000600417400006F6D000047
:10F2E00020760000312E0000303100002045000063
:10F2F00052520000000000005420EF0083982700C5
:10F30000008041001040BA000160EF0000000600DC
:10F31000417400006F6D000020760000312E000067
:10F3200030310000202000004F4B000000000000A2
:10F330005420EF00439A2700008041001040BA009B
:10F340000160EF00000006003A25000030320000A6
:10F35000752C00004E610000647200003A25000028
:10F36000327800002E250000327800002E250000A3
:10F37000327800002C4200006F7800003A2500002F
:10F3800030340000752C0000495000003A25000080
:10F3900030330000750000005420EF00839D2700EB
:10F3A000008041001040BA000160EF00000006003C
:10F3B0002A2A00002A200000526500007374000011
:10F3C0006F72000065200000446500006661000067
:10F3D000756C0000747300000D0A00000D0A000037
:10F3E000000000005420EF00E39F27000080410050
:10F3F0001040BA000160EF00000006002A2A000059
:10F400002A200000446500006275000067200000AB
:10F41000466C000061670000733A00002025000080
:10F42000327800000D0A0000000000005420EF00B8
:10F4300003A22700008041001000BA00000006006F
:10F44000900100008000000000020000C8000000E1
:10F4500040000000000100006400000020000000E7
:10F46000800000003200000010000000400000009A
:10F47000190000000800000020000000E803000060
:10F4800040010000000500005420EF0003A5270004
:10F49000008041001040BA000160EF00000006004B
:10F4A000000600000C120000181E000024000000DE
:10F4B0005420EF0043A62700008041001040BA000E
:10F4C0000160EF00000006004442000047200000F9
:10F4D000525400004D6F00006E6900004865000046
:10F4E00061640000496E000069280000686800003F
:10F4F0003B6D00006D3D000025320000643A0000C5
:10F5000025320000642900000D0A00000000000000
:10F510005420EF0043A92700008041001040BA00AA
:10F520000160EF0000000600525400004800000097
:10F530005420EF0043AA2700008041001040BA0089
:10F540000160EF000000060052540000440000007B
:10F550005420EF00A3022000830150000500310079
:10F5600043AC2700008041001040BA000160EF006A
:10F570000000060040AC27008381410080814100EB
:10F580001380BA00000006003C4573005252690027
:10F590003E527A00746D650048653A00616425004A
:10F5A0005772640069742C0065422500756664001A
:10F5B00020462C00756C25006C3A640077502C00B6
:10F5C0006F7325003D256400642C0D0072500A0005
:10F5D0006F7300003D250000642C00005420EF00F4
:10F5E000A3AF2700008041001040BA000160EF0087
:10F5F0000000060044420000472000005274000052
:10F600006D480000656100006457000072690000E9
:10F610007465000042750000663A00003A7300000D
:10F62000697A0000653D0000256400000D0A0000B5
:10F63000000000005420EF0063022000830150000E
:10F640000500310063B32700008041001040BA007C
:10F650000160EF000000060060B3270083814100D5
:10F66000808141001380BA00000006003C45730011
:10F67000525269003E527A00746D650057723A002A
:10F68000697425006542640075662C0020462500DB
:10F69000756C64006C3A2C00775025006F73640021
:10F6A0003D252C00642C2500725064006F730D0002
:10F6B0003D250A00642C00005420EF0083B627008B
:10F6C000008041001040BA000160EF000000060019
:10F6D0004442000047200000527400006D570000B3
:10F6E000726900007465000042750000663A00000F
:10F6F0003A730000697A0000653D0000256400004F
:10F700000D0A0000000000005420EF0003B927009C
:10F71000008041001040BA000160EF0000000600C8
:10F7200057690000666900005F520000544D0000F8
:10F730006F6E000069540000782800002920000046
:10F74000636100006C6C0000206100007420000008
:10F75000525400004D2E000053570000204F00006F
:10F76000464600000D0A0000000000005420EF0093
:10F7700023BC2700008041001040BA000160EF0068
:10F78000000006002B2B00002B2B00002B2B000071
:10F790002B2B00002B200000525400004D6F000066
:10F7A0006E690000205700006966000069200000B3
:10F7B0006465000062750000672000002B2B0000CC
:10F7C0002B2B00002B2B00002B2B00002B0D0000FF
:10F7D0000A0000005420EF0063BF270000804100B2
:10F7E0001040BA000160EF000000060057690000F9
:10F7F000466900005374000061740000653D00001C
:10F800005B250000645D00000D0A000000000000A0
:10F810005420EF0043C12700008041001040BA008F
:10F820000160EF000000060067520000544D000028
:10F830006F6E0000694D0000742E000073770000A9
:10F840003D250000640D00000A0000005420EF0078
:10F8500023C32700008041001040BA000160EF0080
:10F860000000060067520000544D00006F6E00005B
:10F87000694D0000742E000074780000466C000092
:10F88000616700003D250000640D00000A000000D3
:10F890005420EF0043C52700008041001040BA000B
:10F8A0000160EF00000006005544000050460000D3
:10F8B0006C6700003D250000640D00000A00000098
:10F8C0005420EF00C3C62700008041001040BA005A
:10F8D0000160EF0000000600536500006C66000048
:10F8E0005465000073740000204300006D64000044
:10F8F0003A200000257800002C2000002578000028
:10F900000D0A0000000000005420EF0003C927008A
:10F91000008041001040BA000160EF0000000600C6
:10F920003A530000656C00006654000065730000E7
:10F93000744300006D6400003D3C00002530000071
:10F94000325800002C200000253000003258000002
:10F950002C20000025300000325800002C20000030
:10F9600025300000325800003E2000000D0A000043
:10F97000000000004200F8003600F8005400F800D3
:10F98000801F7800200020000C000900B01F7800C4
:10F9900010C0B3003FF3B700DB51E2000B003200B0
:10F9A000DA51E20003003200DA71ED00E67C040077
:10F9B0000000000007E2A900044020004410880075
:10F9C000042C2F003410880007E2A800C751E20081
:10F9D0000A003200C48D80006120E100030036007F
:10F9E000B831ED00FE7C040000000000B831EF00EB
:10F9F00010C0B300C8F1B700C771EF00B653E20002
:10FA000009003200C953E20007003200C973ED005B
:10FA1000C953E20004003A0010C0B300CFF3B700AE
:10FA2000CED3BF00C9F3B7002E33ED002E13E20092
:10FA300004003A0010C0B30034F3B70054002000B3
:10FA4000749988003233ED003213E20004003A006A
:10FA500010C0B30035F3B700240320009499880048
:10FA6000EF72ED00EF52E2001D003A0040C6B30015
:10FA7000EFF2B70010C0B30036F3B7007153E200E5
:10FA8000010032007173ED003A73ED003A53E20069
:10FA90000C003A00B0C0B3003AF3B7003B53E200A9
:10FAA00005003A003D73EF00E4152000649A8800D9
:10FAB000607D04000000000010C0B3003DF3B700FB
:10FAC0003B73EF00F551E20005003200F571ED00E7
:10FAD000F551E20002003A0010C0B300F7F1B700A0
:10FAE0000068A900A00120000C0009004F10780058
:10FAF0004F0078005400F9003600F9004200F90088
:10FB0000004006004200F8003600F8005400F800FB
:10FB1000801F7800200020000C000900B01F780032
:10FB20006153E200030032006433EF006633EF00FC
:10FB300011E1A9006413E200090032006433ED0012
:10FB400063CEAE000300370065CEA900AC7D040093
:10FB50000000000065CEA800E87D04000000000061
:10FB60006613E200180032006633ED0065CEA9008E
:10FB70006613E20012003A006353E2000D00320007
:10FB80006373ED00149B80004822DE00E4CFB200D6
:10FB900002003A00F0CFB30063F3B7006813F80037
:10FBA0006413F9006A13F8006613F900E07D04009D
:10FBB000000000006433EF006633EF0011E1A9009C
:10FBC000E87D04000000000065CEA90011E1A90055
:10FBD00000E8A900A00120000C0009004F107800E7
:10FBE0004F0078005400F9003600F9004200F90097
:10FBF00000400600851F7800C500200003000900B2
:10FC0000B51F780000F0A6000C0037000000EA00E5
:10FC10000480A00004F0A60008003700801F7800D0
:10FC2000D00220002322AF00FEFF370024A2B7003D
:10FC30004F0078000480A1000860ED008002EB0016
:10FC4000800378008404780004F0A1000404E0003C
:10FC500006003A0009F0A700020037000500200066
:10FC60000F003700050020000D003700E64252006B
:10FC70000A0039000003200009F0A600000220005D
:10FC80002322AF00FEFF370024A2B7008502E9005F
:10FC9000FBFF3B0055002000010037008402780084
:10FCA000640020000580A7000402E80005E0A00031
:10FCB00009F0A70005F0A00008712200110009005A
:10FCC0008883D800A67E020000000000810378002F
:10FCD000883E2000110009008883D800A67E02001B
:10FCE0000000000081037800480620001100090090
:10FCF0008883D800A67E02000000000081037800FF
:10FD0000A8002000110009008883D800A67E020008
:10FD1000000000000980A60005003700D002200086
:10FD20002322AF00FEFF370024A2B7000980A10004
:10FD30000003200000C04000500188002322AF00D3
:10FD4000FEFF370024A2B700200037000603200082
:10FD50000000E0000E003A0005E0A60016003700A3
:10FD60000402E9000524E100020032004200AF0075
:10FD7000000006000000E00005003A0005E0A600D3
:10FD80000D00370005F0A600060220000A0037002B
:10FD900005E0A1000980A6000700370000057800F3
:10FDA000D00220002322AF00FEFF370024A2B700BC
:10FDB0000980A1000A007800004043002322AF0020
:10FDC000FEFF370024A2B700000006002501200036
:10FDD00003000900CF127800CF027800000006006F
:10FDE0004200F8003600F8005400F800801F780048
:10FDF000200020000C000900B01F78002148A90055
:10FE0000348EA8001551E2001E003200F0898000F7
:10FE10003E31EC0080027800E4AB24000483420011
:10FE200048C2BF0000439800F08980003E31EC00DA
:10FE300080027800E4AB24000483420048C2BF0083
:10FE400000439800F08980003E31EC008002780089
:10FE5000E4AB24000483420048C2BF000043980082
:10FE6000108A8000F48980000020E100030039003E
:10FE700010C0B3002FF1B7003E31EF000282040042
:10FE8000000000004B50E2003B003A0048C2BF00B7
:10FE900091F6B700C08980003831EC00800278000C
:10FEA000E4AB24000483420091D6BF00004B7800ED
:10FEB00091F6AF00020037004F50E2000900320017
:10FEC000C08980003831EC0080027800E4AB240067
:10FED0000483420048C2BF0000439800AA7F040088
:10FEE0000000000048C2BF0091F6B700C089800042
:10FEF0003831EC0080027800E4AB24000483420037
:10FF000091D6BF00004B780084B480004822DE0008
:10FF1000C3082000041CE1000E0031009456E200EA
:10FF20000C003A0050C0B3003AF3B700040EA8002A
:10FF3000042EA900142EA800140EA90004CEA800B7
:10FF400004EEA900040A2000448F880010C0B3000A
:10FF50004FF0B700C08980003831EC008002780093
:10FF6000E4AB24000483420048C2BF000043980071
:10FF7000CE7F04000000000048C2BF0091F6B70029
:10FF800048C2BF0091F6B70048C2BF0091F6B70063
:10FF9000C489800063024200C48988003031EC00CB
:10FFA0006150E200080032006410E20006003200F6
:10FFB0006430ED006410E20003003A0010C0B300AA
:10FFC0004BF0B7006170EF009176EF00C4898000BC
:10FFD000036524000418E10016003E003831EF00EC
:10FFE0003411F8003211F900249180004822DE001B
:10FFF0006424E1000B003A009556E200050032004F
:020000040001F9
:1000000010C0B30091F6B7009576EF000E800400A3
:100010000000000010C0B30095F6B7001680040081
:100020000000000010C0B30091F6B7002A80040061
:1000300000000000C08980003211E30005003A0092
:10004000908980003411B4009089880020C0B300EA
:1000500091F6B7009156E200EA0032003031EF002D
:100060005070EC0084828000C4C3B20020003A00CB
:100070005070EF005170EC00848280004822DE0056
:10008000C4C3B2001A003A005170EF005270EC0085
:10009000948280007824E10015003A005270EF004D
:1000A0005370EC00A48280000960EF00E307210098
:1000B000030042000002780014407800948280001F
:1000C0004822DE000024E1000900360010C0B30021
:1000D00053F0B7005470EC00A48280006C24E1005F
:1000E0000300360010C0B30054F0B7005570EC00A8
:1000F00084B480004822DE006124E10002003A005E
:1001000050D0BF00FDF0B7005050E20009003200AF
:10011000848280006F24E100060032008482800027
:100120007E24E100030032008482800024C3B200F8
:1001300000003A007650E200B20032007750E20050
:10014000B0003A008D53E200AE003200A4B480004B
:100150006224E1006D003A005050E20006003200D7
:10016000848280007424E1000300320084828000D5
:1001700084C2B20063003A002322AF00FEFF3700C2
:1001800034052000241188002322AF00FEFF370031
:1001900004052000241188002322AF00FEFF370051
:1001A000D403200024118800C089800004002000AE
:1001B000FA7D0200000000005100200001007800DC
:1001C0000160EF0000020200000000008100E80072
:1001D0002322AF00FEFF370024A2B70080002000DA
:1001E0001008E600F5FF370091D6BF000000FB00C5
:1001F00004002000FA7D0200000000002322AF006E
:10020000FEFF3700D4002000241188002322AF0015
:10021000FEFF3700A4002000241188003611F800EA
:100220003C11F9003811F8003A11F9005B70EF0049
:1002300051D0BF005CF0B70052D0BF005DF0B700F6
:1002400053D0BF005EF0B70054D0BF005FF0B700DE
:1002500055D0BF0060F0B70051D0BF005AF0B700D2
:100260006830EF006C10F8006A10F90063D0BF002E
:1002700072F0B7007370EF00848280007424E10094
:1002800009003A0040C1B3005BF0B7006E10F800FF
:100290006A10F90074D0BF0072F0B7007370EF00FD
:1002A00068810400000000008482800084C2B200E3
:1002B00007003A0080C2B3005BF0B7007010F8008E
:1002C0006A10F90075D0BF0072F0B7007370EF00CC
:1002D00010C0B30078F0B70010C0B30077F0B700DB
:1002E0005BD0BF0059F0B7003811F8009616F9003E
:1002F000C48980000412B100348388006610F800BD
:100300009816F90002820400000000002322AF00CA
:10031000FEFF370034042000241188002322AF00A0
:10032000FEFF370084062000241188002322AF003E
:10033000FEFF3700D40320002411880094D6BF00AC
:100340000000FB0004002000FA7D02000000000015
:1003500051002000010078000160EF001A02020045
:10036000000000008100E8002322AF00FEFF3700FC
:1003700024A2B700800020001008E600F5FF370037
:10038000C089800004002000FA7D02000000000007
:10039000B1002000010078000160EF001A020200A5
:1003A000000000008100E8002322AF00FEFF3700BC
:1003B00024A2B700E00020001008E600F5FF370097
:1003C00091D6BF000000FB0004002000FA7D02006F
:1003D000000000002322AF00FEFF3700D400200001
:1003E000241188002322AF00FEFF3700A400200064
:1003F00024118800348EA90010C0B3009AF6B7000B
:10040000190037003631EC004500090000000000FB
:10041000348EA9004500090000000000A4B480004B
:100420006224E100080031004822EF004822EF007A
:100430004822EF000148A9002148A8009476EC006A
:1004400034820400000000009476EF004C50E2007B
:10045000050032003754E200030032003631EF006D
:100460003831EF003774EF000148A900A0012000E7
:100470000C0009004F1078004F0078005400F9007C
:100480003600F9004200F900004006004200F80082
:100490003600F8005400F800801F7800200020008B
:1004A0000C000900B01F78000000000000000000F0
:1004B00000000000FC27A900A00120000C0009009A
:1004C0004F1078004F0078005400F9003600F90012
:1004D0004200F900004006004200F8003600F80033
:1004E0005400F800801F7800200020000C00090054
:1004F000B01F7800000000000000000000000000B5
:10050000FC87A900A00120000C0009004F10780012
:100510004F0078005400F9003600F9004200F9005D
:100520000040060000A0FE0048C2BF00AAA8F800D4
:10053000E0FF9F00AAA8F9004822EF004822EF0040
:100540004822EF000148A9002148A80006C8A900D8
:100550000080FE00004006004200F8003600F8006F
:100560005400F800801F7800200020000C000900D3
:10057000B01F780008A2AF00030037009B76EF00A1
:100580000842AF009BF6A8009BD6BF000160EF00B9
:100590009B76EC004DF1B700648A80004822DE00B3
:1005A00003082000041CE10058003900648A800020
:1005B0004822DE0004C8B20003003A004CF1B70044
:1005C0004083040000000000A6A8F8004F00780057
:1005D00000C0B300801F7800A6A8F9000862AF0031
:1005E0000D003700801F78000040E800A6A8F80042
:1005F000E0FF9F00A6A8F9004F007800F40F20004C
:100600000024E10002003A000C8304000000000016
:10061000EE82040000000000A6A8F8004F00780059
:1006200000C0B300801F7800A6A8F9000822AF0020
:100630000D003700801F78000040E800A6A8F800F1
:10064000E0FF9F00A6A8F9004F007800F40F2000FB
:100650000024E10002003A0034830400000000009E
:10066000168304000000000008C2AE00010037003D
:1006700008C2A9000782A80000C2BF004CF1B70061
:100680004D51E20004003A00A031EF00A231EF002A
:100690008683040000000000648A80004822DE0097
:1006A0006124E10019003900648A80004822DE00DC
:1006B00004C8B20015003200648A80004822DE00BF
:1006C000614052000080FB000160EF00E414210053
:1006D000840240004CD1BF0080429800048D80000D
:1006E0006120E10008003900048D800061005200A3
:1006F000748A80004822DE000400E10002003A0013
:1007000014002000148D8800A031EC000208A9001C
:10071000A00120000C0009004F1078004F00780065
:100720005400F9003600F9004200F90000400600CC
:100730005202AE00FEFF37005202F8009216F90096
:10074000B01280005222A900000006004200F8000A
:100750003600F8005400F800801F780020002000C8
:100760000C000900B01F780040978000E832EC00D0
:10077000B49C80000400400080027800988302004E
:1007800000000000804A7800449780004351200018
:100790000418E10001003E00E832EF005202AE0012
:1007A0002B00370040978000E832EC00B49C8000BA
:1007B00004004000800278009883020000000000DE
:1007C000804A780044978000435120000418E100DB
:1007D00001003E00E832EF005202AE001C0037007C
:1007E00040978000E832EC00B49C80000400400098
:1007F000800278009883020000000000804A7800A0
:1008000044978000435120000418E10001003E009D
:10081000E832EF005202AE000D0037004097800032
:10082000E832EC00B49C80000400400080027800B4
:100830009883020000000000804A780044978000FE
:10084000435120000418E10001003E00E832EF00AF
:100850000A48A900A00120000C0009004F107800F0
:100860004F0078005400F9003600F9004200F9000A
:1008700000400600B202AE00FEFF3700B202F800F0
:100880009216F900B0158000B222A90000000600FF
:100890004200F8003600F8005400F800801F78008D
:1008A000200020000C000900B01F7800ADD2BF006E
:1008B000AD72EC000080FB000160EF00642B2100B2
:1008C000840240003A84020000000000804A780060
:1008D000649580004822DE0003032000041CE10030
:1008E00001003E00AD72EF00B202AE000F00370013
:1008F000ADD2BF00AD72EC000080FB000160EF00E4
:10090000642B2100840240003A84020000000000B1
:10091000804A7800649580004822DE0003032000AE
:10092000041CE10001003E00AD72EF000B08A900BD
:10093000A00120000C0009004F1078004F00780043
:100940005400F9003600F9004200F90000400600AA
:100950004200F8003600F8005400F800801F7800CC
:10096000200020000C000900B01F78000268A900D8
:10097000A00120000C0009004F1078004F00780003
:100980005400F9003600F9004200F900004006006A
:100990000000E0004220AF000C00370047170900BC
:1009A00000000000FE3F090000000000FE3F0900BB
:1009B00000000000FE3F090000000000FE3F0900AB
:1009C000000000000000E900F4FF3A00000006000B
:1009D000851F78000425F8000A25F9000625F8008F
:1009E0000C25F900402881006000E1001E0036005F
:1009F0005028810090427800602881000002780031
:100A000014407800002CE1000C00320050288100D6
:100A1000904278006028810000027800144078003D
:100A2000002CE10003003D0000C0EB001C85040029
:100A30000000000010C0B3000C00370050288100F7
:100A40000000E80050288900602881000000E800CC
:100A500060288900402881000000E90040288900C2
:100A6000F2840400000000000060EF00CF02780074
:100A700000000600277EEF00020EAF00277EEC008C
:100A80002A7EEF0002CEAF002A7EEC0004CEA80042
:100A90007400200044F1880044F180006020E100EF
:100AA0000E00350026DEBF0002E0B70028DEBF00E2
:100AB0000100A50003003900040EA80064850400AD
:100AC00000000000040EA90004CEA90004CEA80076
:100AD000283EED004C85040000000000658EA80053
:100AE000658EA900275EE20003003200040EA80014
:100AF0007E85040000000000040EA9002A5EE200CA
:100B00000300320004CEA8008A8504000000000023
:100B100004CEA900000006004970EF0049D0BF00D4
:100B200026FEB7003A850200000000000000060023
:100B30008404210014C0A00049D0BF0026FEB700E5
:100B40003A8502000000000000000600851F7800C2
:100B500050C0B300D2F3B700949E8000330220004F
:100B6000041CE1000900360000003700949E80005C
:100B70000960EF000320210083024200804AEB005D
:100B8000D273EC00AC8504000000000050C5B30037
:100B900000F2B70030C2B30001F2B70050C4B30096
:100BA00002F2B700A0CAB30003F2B70010C1B3004D
:100BB00004F2B70010C0B30005F2B700C0D1BF0007
:100BC00006F2B70010C0B30009F2B700CF027800F8
:100BD000000006005B70EF005C70EF005D70EF00DE
:100BE0005E70EF005F70EF006070EF001571EF0056
:100BF0004B70EF006170EF00F4F321002483880054
:100C00005070EF00FD70EF003031EF003631EF0033
:100C10003831EF00E431EF0000000600EA85020001
:100C2000000000004C70EF00B473EF00B573EF00EC
:100C30009073EF008E73EF008F73EF008D73EF00F2
:100C40008B73EF008C73EF001571EF002F71EF00C5
:100C50004471EF00FB71EF004031EF003E31EF00D7
:100C60004E70EF005872EF0000000600851F7800FC
:100C7000C500200003000900B51F780000F0A600A1
:100C80000C0037000000EA000480A00004F0A60079
:100C900008003700801F7800D0022000B322AF0088
:100CA000FEFF3700B4A2B7004F0078000480A10017
:100CB0000860ED008002EB00800378008404780077
:100CC00004F0A1000404E00006003A0009F0A700C7
:100CD00002003700050020000F003700050020004B
:100CE0000D003700E64252000A00390000032000E0
:100CF00009F0A60000022000B322AF00FEFF37007B
:100D0000B4A2B7008502E900FBFF3B0055002000BC
:100D10000100370084027800640020000580A700ED
:100D20000402E80005E0A00009F0A70005F0A0001B
:100D300008712200110009008883D800E2860200B1
:100D40000000000081037800883E200011000900A7
:100D50008883D800E286020000000000810378004A
:100D600048062000110009008883D800E2860200AE
:100D70000000000081037800A80020001100090095
:100D80008883D800E2860200000000000980A600E7
:100D900005003700D0022000B322AF00FEFF37006D
:100DA000B4A2B7000980A1000003200000C04000E9
:100DB00050018800B322AF00FEFF3700B4A2B70095
:100DC00020003700060320000000E0000E003A007B
:100DD00005E0A600160037000402E9000524E10042
:100DE000020032004200AF00000006000000E000F8
:100DF00005003A0005E0A6000D00370005F0A6004A
:100E0000060220000A00370005E0A1000980A600C4
:100E10000700370000057800D0022000B322AF00A1
:100E2000FEFF3700B4A2B7000980A1000A007800D5
:100E300000404300B322AF00FEFF3700B4A2B7006A
:100E4000000006002501200003000900CF127800F1
:100E5000CF02780000000600FD71EF00FF71EF0087
:100E6000FE71EF00F571EF00E673EF00DA33EF008B
:100E7000D8F3EF00C673EF00BA73EF00BB73EF0057
:100E800010C0B300BCF3B700FC73EF00FE73EF00BB
:100E900084B580004822DE006324E1001D00390093
:100EA0000000370001002000010078000160EF0021
:100EB00002080200000000008100E800B322AF0039
:100EC000FEFF3700B4A2B700E00020001008E600E3
:100ED000F5FF3700000020000400200036860200E5
:100EE00000000000B322AF00FEFF3700D405200051
:100EF000A4158800B322AF00FEFF3700D400200005
:100F0000A4158800B322AF00FEFF3700A400200024
:100F1000A4158800FA73EF00FB73EF00FD73EF0078
:100F2000C671EF00FF73EF0084B580004822DE0039
:100F30006224E1001D00390000003700010020009C
:100F4000010078000160EF00BA0302000000000019
:100F50008100E800B322AF00FEFF3700B4A2B70063
:100F6000400120001008E600F5FF370000002000D7
:100F7000040020003686020000000000B322AF000B
:100F8000FEFF3700D4052000A4158800B322AF006F
:100F9000FEFF3700D4002000A4158800B322AF0064
:100FA000FEFF3700A4002000A4158800F171EF00B7
:100FB000E831EF0030C0B300B9F3B700CE71EF00F5
:100FC000BE73EF00B673EF00B773EF00F973EF0075
:100FD000F873EF00E873EF0084B580004822DE006C
:100FE0006124E1001D0039000000370001002000ED
:100FF000010078000160EF003403020000000000EF
:101000008100E800B322AF00FEFF3700B4A2B700B2
:10101000A00020001008E600F5FF370000002000C7
:10102000040020003686020000000000B322AF005A
:10103000FEFF3700D4052000A4158800B322AF00BE
:10104000FEFF3700D4002000A4158800B322AF00B3
:10105000FEFF3700A4002000A4158800DC33EF0059
:10106000DE33EF00E773EF00A033EF00E832EF006C
:10107000EA32EF00A631EF00DE71EF00D971EF0028
:10108000ED71EF00E371EF00B033EF00F40F2000DB
:10109000749D88009833EF0004302400B49C8800CD
:1010A00000000600AB73EF00AC73EF009573EF0028
:1010B000A673EF00A773EF00A873EF00A973EF000A
:1010C000AA73EF00F873EF0000000600851F780098
:1010D00004022C0004708800C43C2C00847088003A
:1010E000E40023000471880004702F0084718800DC
:1010F00004302000047288000410200084728800EC
:10110000F408220004738800042EEF00142EEF0070
:10111000041028002471880014042400A47188009D
:10112000442EEF0004102000A4728800642EEF000B
:101130008C85020000000000C4572100C481880093
:10114000D4572100B481880064582100E4818800CC
:1011500074582100D4818800E4572100048288005B
:10116000F4572100F481880021E2A90051E2A9008E
:10117000546EA90054042000343A88004407A900A2
:101180004427A9004447A9004467A9004487A9004F
:1011900044C7A90044E7A9004827EF003000200019
:1011A0003174200082072000A309200082487800C3
:1011B00083487800804878001000200021742000C7
:1011C000620420007305200082487800834878007C
:1011D00080487800E602AF00FEFF370098850200E5
:1011E00000000000C47DEF0024EE800033022000E8
:1011F000041CE1000800360024EE80000960EF00C6
:10120000A325210083024200804AEB00C47DEC004C
:10121000F48804000000000010C0B3005AF2B700C8
:1012200000C1B3005CF2B700A68502000000000018
:10123000040028006470880084202000E470880086
:1012400004102600E4718800040420006472880001
:10125000140820006473880014002000D4718800F2
:10126000040320005470880004002800D471880012
:10127000140A20001454880004012A0064548800D1
:10128000C573EF00C673EF00C773EF00C873EF00BC
:10129000A431EF00F0C1B3007FF0B700C0C1B300CC
:1012A00080F0B700F0C1B30081F0B700E0C1B30037
:1012B00082F0B700F0C1B30083F0B700E0C1B30023
:1012C00084F0B700F0C1B30085F0B700F0C1B300FF
:1012D00086F0B700E0C1B30087F0B700F0C1B300FB
:1012E00088F0B700E0C1B30089F0B700F0C1B300E7
:1012F0008AF0B700C471EF005570EF007670EF0010
:101300007770EF007970EF006830EF007870EF00D1
:101310009073EF008E73EF008F73EF007B70EF0020
:10132000D48380004822DE0083032000041CE100F7
:1013300008003600D48380004822DE00430C2100E0
:1013400083024200804AEB007B70EC00908904002D
:10135000000000004F70EF007B70EF004A71EF005B
:101360004B71EF004871EF004971EF00C571EF005C
:1013700010C0B30048F0B7007F73EF008633EF0072
:101380007E73EF005833EF005633EF005433EF0015
:101390004A73EF004B73EF007A73EF007B73EF003B
:1013A0007673EF007073EF006F73EF00C071EF00A2
:1013B000CF71EF00D071EF00BD73EF0010C0B3002C
:1013C00038F3B70040C1B30039F3B700A231EF00E2
:1013D0006173EF00E41029001482880014828000F9
:1013E0006500520020828800540020007499880013
:1013F000A400200084998800240320009499880088
:1014000040C6B300EFF2B7003573EF003673EF005C
:101410003473EF005C33EF0010C0B300F4F1B70099
:10142000EA31EF000771EF000E86020000000000B5
:101430002C8702000000000052880200000000001B
:10144000F671EF00EB73EF00F771EF00F673EF004A
:10145000EC71EF00E631EF00FE73EF009473EF00E4
:10146000E673EF00ED73EF00EE71EF00EF71EF0048
:10147000F071EF00B0C0B300F2F1B700444D2000AE
:10148000049F8800044B2000149F88004E33EF0017
:101490005A33EF006C73EF00C4122000148A8800E6
:1014A000AA72EF009273EF00CD71EF00F371EF00BD
:1014B000A831EF00AA31EF006373EF006433EF004F
:1014C0006633EF006833EF006A33EF004770EF00D8
:1014D0007173EF00B572EF00E772EF008A73EF00EF
:1014E000EC72EF002472EF00AD72EF00B472EF0007
:1014F000ED72EF00EE72EF0010C0B300BBF1B70069
:10150000BA71EF0020C0B300BCF1B7003D73EF002B
:10151000C0C0B3003AF3B700E4152000649A880015
:101520003B73EF00A0C0B3003CF3B7003E73EF0085
:1015300000C5B30041F3B7004273EF004373EF00FF
:1015400004FA2000749A88005233EF0000C5B300FB
:1015500048F3B7004773EF006073EF004573EF0087
:101560006273EF005F73EF0010C0B3005EF3B7006B
:10157000AD73EF00B273EF00B373EF00CC71EF0007
:101580009173EF00B431EF00A0C5B30073F3B7005F
:101590007273EF00A0C0B30077F3B7007873EF0069
:1015A00050C0B30074F3B7007573EF00DC71EF0047
:1015B000DB71EF007973EF0040C0B30025F2B70094
:1015C0005772EF005872EF004D70EF0010C0B3007B
:1015D00059F2B7004A70EF006270EF00010020007E
:1015E000010078000160EF00980C0200000000008C
:1015F0008100E800B322AF00FEFF3700B4A2B700BD
:10160000900120001008E600F5FF370003000900F4
:10161000B01280000A48A90003000900B01580003C
:101620000B08A9002168A8002A48A8002B08A800D8
:101630000208A9002208A800C3E8A80004CEA90057
:1016400004EEA900346EA800CB71EF00A031EF00CA
:10165000C028EF002068A9000421EF00F437220021
:101660001408880004012A00240888000068A900E2
:101670002068A8001021EF00F437220064088800D9
:1016800004002A008408880020E8A80011E1A900CD
:10169000CF02780000000600851F780084B5800026
:1016A0004822DE006224E10011003900E5C2B300E7
:1016B000D0022000B322AF00FEFF3700B4E2B70033
:1016C000B562EF000A60ED004220AE00F8FF37007F
:1016D000B322AF00FEFF3700D4002000A41588001D
:1016E000B322AF00FEFF3700A4002000A41588003D
:1016F00084B580004822DE006224E1000C0039003D
:1017000001002000010078000160EF00700202007B
:10171000000000008100E800B322AF00FEFF3700A8
:10172000B4A2B700D00120001008E600F5FF370092
:10173000AB76EF00CF027800000006004C8B020071
:101740000000000010C0B300B0F6B70084B5800000
:101750004822DE006124E1001D0039000100200064
:10176000010078000160EF003A0202000000000072
:101770008100E800B322AF00FEFF3700B4A2B7003B
:10178000A00020001008E600F5FF3700E0D1BF0000
:101790000000FB000400200036860200000000006C
:1017A000B322AF00FEFF370004022000A41588001A
:1017B000B322AF00FEFF3700D4022000A41588003A
:1017C000B322AF00FEFF3700E4032000A415880019
:1017D000E0F1EF0084B580004822DE006124E100E2
:1017E00015003900B322AF00FEFF370004022000CD
:1017F000A4158800E0D1BF000000FB000400200019
:101800003686020000000000310020000100780050
:101810000160EF0058020200000000008100E800B3
:10182000B322AF00FEFF3700B4A2B700A000200033
:101830001008E600F5FF3700E2F1EF0000000600B7
:1018400021B6210002002000370009008058EB007B
:1018500004302300B4DC880004502300C4DC88007A
:10186000000006003E7BEF00403BEF00000006005A
:1018700018DEBF00C951E30001003A00380037000C
:10188000C9D1BF00C4F080000024E1001800360078
:10189000248EA800630109000000000025EEA900C5
:1018A0006301090000000000C9D1BF0019FEB700A4
:1018B00019DEBF00C4F080000024E10009003600FA
:1018C000248EA9004500090000000000248EA80015
:1018D0004500090000000000197EEC00588C04004F
:1018E00000000000248EA900A68C04000000000067
:1018F000248EA900630109000000000025EEA90064
:10190000630109000000000018DEBF0019FEB700E7
:1019100019DEBF00448E80004822DE000024E10072
:1019200009003600248EA8004500090000000000D0
:10193000248EA9004500090000000000197EEC007B
:10194000888C040000000000248EA90063010900B7
:101950000000000025EEA80018DEBF00C9F1B700A6
:1019600000000600040EA800042EA90004EEA80042
:1019700004CEA900142EA800140EA9000000060031
:10198000F0FF2F000862AE000500370009C2AF006B
:10199000FEFF37001110880009C2AF00FEFF3700BC
:1019A0000000200009E2AF000000E800000006008F
:1019B0000862AE00040037000622A8000622AF002D
:1019C000FEFF3700030037000602A8000602AF0042
:1019D000FEFF370021C2B300C08C020000000000EF
:1019E00020DEBF0002E0B700C08C02000000000053
:1019F0008040EB00C08C0200000000000862AE00D6
:101A0000040037000622A8000622AF00FEFF3700C0
:101A1000030037000602A8000602AF00FEFF3700F1
:101A200031C2B300C08C02000000000000000600BC
:101A3000F0FF2F000862AE00110037003210800066
:101A40007F016100FDFF3A000662A8000100A700C7
:101A500006A2A9000100A60006A2A800321080007C
:101A60007F016100FDFF3A000682A8000822AE0057
:101A7000FEFF37000010800008C2AF0008C2A900B6
:101A800000000600840421001480A00049D0BF009B
:101A900026FEB7003A8502000000000010C0B30027
:101AA000CAF1B70000000600010020000100780024
:101AB0000160EF00C00C0200000000008100E8009F
:101AC000B322AF00FEFF3700B4A2B70080012000B0
:101AD0001008E600F5FF37000040EB000004E000CE
:101AE0000C00320001002000010078000160EF00CE
:101AF000E60C0200000000008100E800B322AF0005
:101B0000FEFF3700B4A2B700800020001008E600F6
:101B1000F5FF3700101EAE000C003700010020005A
:101B2000010078000160EF00FC0C020000000000E2
:101B30008100E800B322AF00FEFF3700B4A2B70077
:101B4000000120001008E600F5FF3700103EAE004F
:101B50000C00370001002000010078000160EF0058
:101B60001A0D0200000000008100E800B322AF005F
:101B7000FEFF3700B4A2B700F00020001008E60016
:101B8000F5FF370010DEBF00634060000004E00096
:101B90000C00320001002000010078000160EF001D
:101BA000380D0200000000008100E800B322AF0001
:101BB000FEFF3700B4A2B700000120001008E600C5
:101BC000F5FF3700105EAE000C003700010020006A
:101BD000010078000160EF00560D020000000000D7
:101BE0008100E800B322AF00FEFF3700B4A2B700C7
:101BF000D00020001008E600F5FF370010DEBF001F
:101C0000654060000004E0000C003200010020008C
:101C1000010078000160EF00720D0200000000007A
:101C20008100E800B322AF00FEFF3700B4A2B70086
:101C3000E00020001008E600F5FF370010DEBF00CE
:101C4000664060000004E0000C003200010020004B
:101C5000010078000160EF008E0D0200000000001E
:101C60008100E800B322AF00FEFF3700B4A2B70046
:101C7000A00020001008E600F5FF370010DEBF00CE
:101C8000674060000004E0000C003200010020000A
:101C9000010078000160EF00A60D020000000000C6
:101CA0008100E800B322AF00FEFF3700B4A2B70006
:101CB000100120001008E600F5FF370010DEBF001D
:101CC0006B4060000004E0000C00320001002000C6
:101CD000010078000160EF00C60D02000000000066
:101CE0008100E800B322AF00FEFF3700B4A2B700C6
:101CF000C00020001008E600F5FF370010DEBF002E
:101D00006C4060000004E0000C0032000100200084
:101D1000010078000160EF00E00D0200000000000B
:101D20008100E800B322AF00FEFF3700B4A2B70085
:101D3000F00020001008E600F5FF37000000060064
:101D400010C6B30094F0B70040C7B30095F0B700D9
:101D5000F0C6B30096F0B700D0C6B30097F0B70056
:101D600000C3B30098F0B70000C3B30099F0B70008
:101D700000C3B3009AF0B70000C3B3009BF0B700F4
:101D80009C70EF0000000600040EA900042EA900BC
:101D9000142EA900140EA90004EEA90004CEA90077
:101DA0000000060020C0B300BFF1B700DE71EF00F5
:101DB000E832EF00EA32EF00E773EF00265EE20060
:101DC00003003A00000037009E8B02000000000074
:101DD000E873EF0084B580004822DE006124E10052
:101DE0001D003900000037000100200001007800CC
:101DF0000160EF0034030200000000008100E800F1
:101E0000B322AF00FEFF3700B4A2B700A00020004D
:101E10001008E600F5FF3700000020000400200055
:101E20003686020000000000B322AF00FEFF37003C
:101E3000D4052000A4158800B322AF00FEFF3700B0
:101E4000D4002000A4158800B322AF00FEFF3700A5
:101E5000A4002000A4158800B773EF00BB73EF0047
:101E6000BA73EF0000000600267EEF00D28E02005B
:101E700000000000000006008404210014F0A0000F
:101E800049D0BF0026FEB7003A85020000000000DE
:101E90000000060004CEA80004EEA9002C87020072
:101EA00000000000F651E20002003200000037009E
:101EB0001F003700348F020000000000E973EF00BC
:101EC000EE71EF00EF71EF00EC73EF00A0C1B30013
:101ED000F5F1B700EB73EF00F771EF00245EE2005D
:101EE000020032000000370025CEA8003C8F02001F
:101EF00000000000544EA800546EA800401F2000AF
:101F0000C884020000000000DF71EF00C671EF001E
:101F100051E2A8005342A80003000900B01280005B
:101F20000A48A9002A48A80004CEA90004EEA90086
:101F300000000600851F780010C4B300A8F0B700A9
:101F400040C5B300A9F0B700B0C2B300AAF0B70013
:101F500070C5B300ABF0B70010C4B300ACF0B7006D
:101F6000D0C3B300ADF0B700D273EF00949E8000F1
:101F70007324E1003800310000003700949E800097
:101F8000664242000440780000E0B7000080FB0099
:101F90000160EF00840A210084024000949E8000CA
:101FA0000960EF004309210003004200904A7800D5
